:020000040800F2
:1000000000500020C98B0008758C00082977000873
:10001000758C0008758C0008758C000800000000C5
:10002000000000000000000000000000758C0008C7
:10003000758C000800000000758C00081977000816
:10004000758C0008758C0008758C0008758C00088C
:10005000758C0008758C0008758C0008758C00087C
:10006000758C0008758C0008758C0008758C00086C
:10007000758C0008758C000881760008758C000866
:10008000758C0008758C0008758C0008758C00084C
:10009000758C0008758C0008758C0008758C00083C
:1000A000758C000895750008758C0008A57500080A
:1000B000857500087575000865750008C976000823
:1000C000C1760008C5760008BD760008758C00086A
:1000D000758C00083D760008B5750008758C000821
:1000E000758C0008758C0008758C000800000000F5
:1000F0000000000000000000000000000000000000
:0C01000000000000000000005FF808F1A3
:100110002DE9F04F674B684C99B023600023636072
:1001200005F0D2FF18B903F02DFE05F0EFFF03F044
:100130001FFA00230893614C09930A934FF4E013CC
:100140000B9323685E4943F480338A7B2360A36961
:10015000894643F01003A361236803F40033099335
:10016000089B01330893099B1BB9089BB3F5A06F4B
:10017000F2D12168514B11F4003101D0022315E076
:10018000186840F0010018600891236803F002032A
:100190000993089B01330893099B1BB9089BB3F58E
:1001A000A06FF2D12368980739D501230A93454BF4
:1001B000454E1968454F41F010011960196821F04A
:1001C00003011960196841F00201196063686360F6
:1001D00063686360636843F4806363603C4B1968E1
:1001E00021F0704119603B49B161616821F47C11D3
:1001F0006160196841F000411960FB6823F4004315
:10020000FB60BB68190449BF334B4FF4E013B36183
:100210004FF480130B930A9B012B01D117E0FEE7EB
:10022000022B18D16AB10B9BB3F5801F02D14FF49A
:10023000A01305E00B9BB3F5E01F02D14FF40013B0
:100240000B9362680B9B134343F4803302E06368B3
:1002500043F460136360236843F080732360226873
:10026000164B9201FBD55A6822F003025A605A6875
:1002700042F002025A606368104A03F00C03082B34
:100280000693F8D15168154B01F00C01042903D0F5
:10029000082904D00F4A00E0B2691A602AE05168C8
:1002A0005068C1F38341C50301F102011AD40C4A1D
:1002B0001EE000BF5D23000808050020001002407A
:1002C000A40F002000200240100000200010014078
:1002D0000410014000127A00001BB70080000020CB
:1002E00000093D00526812F4003FB26918BF52087D
:1002F000514319606268DFF848A3C2F30312324425
:1003000092F81CB01A6818AD22FA0BFBC3F800B0C3
:10031000BB4B4FF00008CAF80C30A369B94843F052
:100320000103A361636A43F080736362A36943F0CE
:100330001C03A3614FF6FF7325F82C3D29468DF869
:10034000368002F04FFBB048294602F04BFB2946AD
:10035000AE4802F047FBAE4B28465A6842F00072A6
:100360005A6006F027FC0D9BAA4AAB48B3FBF2F398
:100370004FF47A728360BBFBF2FBA84B0BF1FF32A8
:100380005A60F0228AF823200722C3F808806420EC
:100390001A6001F0D4FEA022A14841460AF0B9FD3E
:1003A000E369424643F00703E361A36943F4006352
:1003B00043F00C03A361984B4FF0000803F10C01CC
:1003C00002F8018001320E2AF5D1FF229A76DA7600
:1003D0001A775A77934B4FF0100A0FCB85E80F002E
:1003E000A3690D9843F01003A361A3690EA943F01C
:1003F0001003A3614FF400533B614FF480433B6112
:1004000002F0F0FA10A90F9802F0ECFA404606F05C
:10041000F7FE854FD9F808B041460BF40063524609
:10042000384605930AF075FD042302223B7007212C
:1004300001231BF4004F8DF832208DF83380ADF886
:1004400030A0BB70F97008D01220ADF830003B71BD
:100450007B71BB71F971904600E0984669480CA920
:1004600001F092FB059B93B1022367480CA9ADF8FC
:10047000303001F089FB092301223B73BA7308F184
:100480000103072287F80D80FA735FFA83F8636926
:10049000664843F001036361A369DFF890A143F468
:1004A0000073A36106F00FFB614B00240D93614BB9
:1004B000B8F1010F0E930CBF2346802312934FF423
:1004C000807313934FF4806314932023294615936C
:1004D00050464FF4005316930F94CDF8408011947A
:1004E000179406F0D2FADAF80030B8F1010F43F0B1
:1004F0000103CAF80030504B98BF00215A6888BFEA
:10050000012122F4702222F4807242EA01225A6010
:1005100099684A4A20460A4042F4602242F00202A8
:100520009A60D96A08F1FF3221F47001D2B241EA2F
:100530000252DA62012339188A78002A5AD03A5CCA
:100540005C1C092A91F803E0E4B23B4911D9A2F1FD
:100550000A0505EB45054FF0070C0CFA05FC0EFAF1
:1005600005FED1F80C8028EA0C0C4CEA0E05CD6093
:100570000EE002EB42054FF0070C0CFA05FC0EFAF8
:1005800005FED1F8108028EA0C0C4CEA0E050D612E
:10059000062B29490ED8013B03EB83034FF01F0EB6
:1005A0000EFA03FE9A404D6B25EA0E0545EA02035A
:1005B0004B6320E00C2B0ED8073B03EB83034FF07B
:1005C0001F0E0EFA03FE9A400D6B25EA0E0545EA52
:1005D00002030B630FE00D3B03EB83034FF01F0E91
:1005E0000EFA03FE9A40CD6A25EA0E0545EA02039B
:1005F000CB6200E01C460430102823D023469AE743
:100600000005FA0500080140000C014000100140FF
:100610000000014040420F000805002010E000E00B
:10062000580E002098CB0008DC0300200800024090
:100630004C240140EC03002000240140FDF7F1FFB1
:1006400000ED00E0A84B9A6842F480729A609A68C4
:1006500042F001029A609A6842F008029A60996832
:10066000A14A0807FBD4936843F0040393609E4AB1
:10067000936813F00403FAD19168B9F8E60041F4E5
:10068000A0019160994A50B9B2F9E83033B9B2F992
:10069000EA30D3F1010338BF002300E0034613F032
:1006A000010340F0898086F82C3000B207F0F6FC98
:1006B0008F4907F047FD8D4E0546B6F9E80007F073
:1006C000EDFC8B4907F03EFD0446B6F9EA0007F061
:1006D000E5FC874907F036FD804628460AF048FECB
:1006E000064628460AF0B8FE074620460AF040FEB5
:1006F000054620460AF0B0FE044640460AF038FEA1
:10070000814640460AF0A8FE31468046484607F03A
:1007100019FD31468346404607F014FD49460590D1
:10072000384607F00FFD41460790384607F00AFDAE
:1007300029468246484607F005FD6E490862414653
:1007400005F1004007F0FEFC6A4A214650629462BF
:10075000079807F0F7FC0146059807F0EBFB654B9F
:100760002146D862504607F0EDFC0146584607F096
:10077000DFFB60490863294607F1004007F0E2FC0F
:100780005C4A21465063584607F0DCFC014650465F
:1007900007F0CEFB574B21469863059807F0D2FC33
:1007A0000146079807F0C6FB5249C8632846314600
:1007B00007F0C8FC4F4A10644F4DDFF860912B687A
:1007C0004A4C43F00A032B60D9F800304B4E49489D
:1007D000B3F852B00023B4F8EE8094F8ED703370A3
:1007E000436406F0F7FC002800F00781444B454ABB
:1007F000B8F1BB0F1A60444A444E5A60444ADA606A
:1008000001D9012312E0B8F1610F01D902230DE0F3
:10081000B8F1290F01D9032308E0B8F1130F01D96A
:10082000042303E0B8F1090F07D9052386F82D301A
:100830002B6843F001032B600CE00623F6E7092F39
:100840000ED097B1334B1B78002B40F08180002FE6
:100850007AD01F46304B0022022F1A70EFD104E0ED
:100860002B6823F002032B60ECE7DFF888804FF061
:1008700000094146C1F8449006F0ACFC0028E1D0E4
:1008800006210DAB68200A4606F0C2FD9DF8373000
:100890009DF839C003F001035B000CF0010C43EA42
:1008A0008C0C9DF8353003F001035CEA030A09D093
:1008B000BAF1010F02D188F8489034E0BAF1020F82
:1008C0000BD12DE00CAB68200C21012206F0A0FD1D
:1008D0009DF8303013F00F0301D105208EE0042B7A
:1008E0001ED188F848A01EE000240140A40F00207B
:1008F00035FA8E3C080500200C0200204E02002034
:1009000038020020F97000085F6F00081000002016
:1009100090C1793D5D160020B6020020340200200F
:10092000012388F84830B04BB04A1A60B04A5A6088
:10093000B04A92F84820002A14BF6E226F221A7221
:10094000AD4B02221A707DE72B6823F002032B6067
:100950002B680DF1600823F004032B60002308F8D6
:100960002C3D1E200A210122434606F051FD18B1FC
:100970009DF83430482B03D02B6823F008032B60FC
:1009800094F8E2300BB19D4A137094F8E3300BB148
:100990009B4A137094F8E4300BB19A4A13702B6899
:1009A000990702D5904B1B689847974B914F1B684E
:1009B00098472B6813F0080F1CD00FFA8BF34FF0F9
:1009C000640A93FBFAF94846049307F067FB049B1B
:1009D00083460AFB193000B207F060FB8B4907F031
:1009E000B1FB0146584607F0A5FA894907F0AAFB72
:1009F000F86405E00023FB6402E0032001F0E8FB5B
:100A0000844B4FF480425A614FF400521A614FF008
:100A10000A0A9946D9F80C30192083F48043C9F8A2
:100A20000C30D9F80C300AF1FF3A83F40053C9F8BE
:100A30000C3001F084FB192001F081FB1AF0FF0A51
:100A4000DFF8D0B1E6D14FF40053CBF810304FF4BB
:100A50008043CBF81030704BDFF8E8A11B6893F9A6
:100A60000C0007F01BFB6D4907F06CFB0AF080FCE3
:100A70008346BAF8000007F011FB594607F062FB05
:100A80000AF0ACFC664B1880BAF8000007F006FBD1
:100A90000146644807F00AFC634907F007FC5A4B1B
:100AA00038655E49D86807F04DFB604907F04AFB9E
:100AB0005F4B627918605F4B5F491A705F4B01EBC7
:100AC000C202527C7B655E4B1A60A268920644BFEC
:100AD00001221A602B681B0740F1FF804FF480430E
:100AE000C9F81430322001F02AFB002111221E2007
:100AF00006F0B6FA012160221E2006F0B1FA642049
:100B000001F01DFB4FF0000A404606F029FBD346DA
:100B10004FF00A0C5346022101221E200493CDF807
:100B20000CC006F09DFA322001F009FB404606F0A9
:100B300017FBBDF93410BDF93600049BBDF9382010
:100B40000B448842B8BF014692449142B8BF0A465E
:100B500012F5805F8344DDF80CC00BDDD9F80C2062
:100B6000BCF1010C82F48042C9F80C20D3D10121E0
:100B7000059101E0002005901E200021122204931F
:100B800006F06EFA049B4FF00A0C022101221E208F
:100B90000493CDF80CC006F063FA322001F0CFFACE
:100BA000404606F0DDFABDF93410BDF93600049B6D
:100BB000BDF938205B1A8842B8BF0146C2EB0A0A69
:100BC0009142B8BF0A4612F5805FC0EB0B0BDDF80F
:100BD0000CC039DDD9F80C20BCF1010C82F4804244
:100BE000C9F80C20D1D131E0A40200204947000807
:100BF000216F0008080500205D1600204E0200202D
:100C0000B60200205A160020380200208988883C4D
:100C10000000204100100140F002002035FA8E3C17
:100C2000140300200AE81C4100401C46BD378635ED
:100C3000EC0200200005002098CB0008B40F002033
:100C4000FC0400200000002000220592DFF8CCC147
:100C50001846CDF80CC007F021FA0146674807F0A6
:100C600025FB20F000403063584607F017FA014694
:100C7000624807F01BFB20F000407063504607F00D
:100C80000DFA01465E4807F011FB20F00040B0630A
:100C9000002170221E2006F0E3F9012120221E20EF
:100CA00006F0DEF9022100221E2006F0D9F96420A8
:100CB00001F045FA059BDDF80CC03BB94FF07E53BF
:100CC000CCF83030CCF83430CCF838304FF48043A6
:100CD000C9F810304B4B01221A704B4E4B4BB346A8
:100CE000336005F029FE3068494B0590FF21184616
:100CF00016220AF00EF9002202702A68DFF814E1C9
:100D0000012112F0020F8EF80010734604D04170DA
:100D10000321197002218170550704D519784D1CE3
:100D20001D700325455412F00A0F0CD01A780421C7
:100D30008154511CC9B205254554D11C0232197089
:100D4000D2B206218154A268910604D519784D1CAF
:100D50001D70072545546179082901D00E2904D159
:100D600019784D1C1D700B25455419784D1CEDB29A
:100D70001D700C234354530705D5264B02311970BF
:100D8000234B10215955234B12261978465494F8B9
:100D900041614D1CEDB2002E0CBF002602F0010691
:100DA0001D7026B102311970194913264E5596054A
:100DB00004D51A78511C1970152383541648002144
:100DC00098220AF0A6F8144D05F1980A95F84A30D1
:100DD000002B30D1059999464A68002603230096D6
:100DE0000120314606F0DAF80346C8B9B9F1000F20
:100DF00024D14FF496424FF00109EEE700406F46D0
:100E000001C05E462C020020B8040020CC10002057
:100E1000BF040020BE0400201804002010000020A1
:100E2000284631464C2204930AF073F8049B2B6049
:100E3000012385F84A304C355545C7D1B64BDBF810
:100E40000020197A02290AD0187D022806D08D07C1
:100E500005D400F0020000F0FF0108B10C3359681E
:100E6000AE4DA96531B9009102209268032306F0C6
:100E700095F8A8654046002114220AF04AF86379E3
:100E80000E2B01D0082B02D101238DF83F30A3682F
:100E9000A348C3F38041C3F340028DF83A10A1493F
:100EA0008DF83920C3F380128DF83B200968C3F315
:100EB00040328DF83420C3F3C03200318DF8362033
:100EC000C3F3C02218BF01218DF83720C3F30042BD
:100ED0008DF83C208DF83D1003F0010201688DF87B
:100EE000352091F8B011B4F8E000C1F380018DF81D
:100EF0003E10ADF84200B4F8DE104FF47A70ADF851
:100F00004400D804ADF8401004D5874BB3F8DA306C
:100F1000ADF84430B1F5FA7F84BF0023ADF844301A
:100F2000B4F81A318149ADF8463094F8223185F889
:100F30005C30002385F85D304B709DF83F30002B0E
:100F400014BF0223002302B10133794A4FF0000895
:100F500002EB8303D3F8C830C1460593059931F8F5
:100F600008304FF6FF718B42DAB20AD195F85D3046
:100F700085F85F306F4B1F78162F40F03F810024BB
:100F80002EE16D4C9DF838104FEA021A544419B105
:100F9000911E012940F20F819DF8361011B1012AEE
:100FA00000F009811B0A022B05D19DF8341000299D
:100FB00008BF002303E0012B08BF9DF835309DF8E2
:100FC0003D1039B19DF83F1021B9A2F10801012966
:100FD00098BF04239DF83E1031B19DF83F1019B918
:100FE000043A032A40F2D080012B39D1FF2387F83D
:100FF000A43087F8A530A3680026E27B6068ADF8CE
:1010000030300CA9022387F8A860C7F8B4408DF8E7
:1010100033308DF8322087F860607E66BE66FE66EB
:10102000C7F8A06087F8A66087F8A76001F0DAFC2F
:10103000414A217B52F80A00324600F079FC2046F2
:1010400005F004F93D4B3E49C7F8B8303D4BC7F8B1
:10105000C060C7F8BC3020460A1D03F091FBAAE02F
:10106000022B36D15FFA89F21C20424336494FF0F9
:10107000000B8E18012086F8019086F802B086F8E1
:101080000AB08854A168E27B6068ADF83010F46063
:101090000CA98DF832208DF8333001F0A3FC264BDB
:1010A000217B53F80A005A4600F042FC204605F026
:1010B000CDF8264BC6F818B03361254B2046736136
:1010C00006F1100106F1140203F05AFB09F10109BF
:1010D00071E0032B56D19DF83A20BDF8443032B16F
:1010E00095F85E60204608214FF6FF723CE0BDF89F
:1010F000402095F85E60B2F5FA7F2FD91549204659
:10110000B1FBF2F292B2082105F052FA05EB860625
:10111000C6F88801104B2EE01000002008050020C2
:1011200034020020FC040020A40F002065050020EC
:1011300098CB00080005002058DE0008CD170008F5
:10114000C0050020A9180008B00500202D1B0008CC
:101150009D17000800127A00C9180008934920461C
:10116000B1FBF2F292B2012105F022FA05EB8606FC
:101170008F4BC6F88801C36095F85E30013385F85F
:101180005E3018E0042B16D1BDF84230874A204665
:1011900092FBF3F20121BDF8463092B297F85D6000
:1011A00005F006FA97F85D3007EB86060133C6F8BE
:1011B000B80187F85D3008F10208B8F11C0F7FF420
:1011C000CDAED3E67B4E98E80F00264486E80F00AC
:1011D000794B10341A78C02C02F101021A7008D031
:1011E0006B6D0021185903EB040807F03FF9002844
:1011F000E8D0724EB368D9041DD418E070486E4A26
:1012000000EBC70393F810E0D3F814C082F800E0B5
:10121000BCF1000FEDD000247445EADA654E2301DD
:101220001E4463440FCB013486E80F00F4E7082F17
:10123000644C28D129E0604B93F80090B9F1010F7C
:10124000F5D9614C4FF00008C84504F11004EEDAFE
:1012500054F8100C4FF07C5106F074FF4FF07C51A5
:1012600044F8100C54F8140C06F06CFF4FF07C514D
:1012700044F8140C54F80C0C06F064FF08F1010853
:1012800044F80C0CE0E70E2F03D1237843F0100351
:1012900002E0237823F01003237005F0ABF84B4AEB
:1012A0004B484C494C4B02604C48C5F89C3201609D
:1012B0000023B6F81A01C5F89812A5F8A23285F8ED
:1012C000A432C5F8A822464958520233242BFAD139
:1012D000444B1A60B3681A0740F1B680374B0022BE
:1012E00093F81831042B00F2A980DFE803F0030320
:1012F0002A4F9300012B4FF003013B4A08D185F898
:10130000AC12072185F8AE3285F8AD120C2308E047
:10131000022385F8AC32002385F8AE3285F8AD1291
:101320000723137000230093102001232F494FF44B
:10133000E13205F033FE2E4BC5F8B002C5F8B432E9
:1013400078E001232B4A2C4900931020052305F057
:1013500025FEC5F8B8020746B6F81A0106F09EFE4B
:10136000264906F0EFFE264906F0E2FD07F0D6F822
:101370000023244A98500433402BFAD1224B1022E8
:10138000C5F8B432184B381C1A7054E0009201238F
:101390004FF4E13210201D4905F000FE1C4BC5F84A
:1013A000BC02C5F8B432102242E000BF40420F0038
:1013B000B9180008E006002034160020A40F002011
:1013C00098CB00081A020020E8060020A40700209D
:1013D0000C040020B410002070CC0008FC00002099
:1013E0006203002000020020D5040020B51F000881
:1013F00039150008A0860100C9200008CDCCCC3FDB
:101400000000B0441C010020ED1500085120000828
:10141000DD150008009201234FF4E1321020384915
:1014200005F0BCFD374BC5F8C002C5F8B432082240
:10143000354B1A70003018BF012028B9082001F080
:101440004EFA0023C5F8B432B2682F4B12F4804F25
:1014500004D0082119702D49C5F8B41242F20101D7
:10146000114002F0010002F4005741B1284AC5F8CA
:10147000B4220FB108221A7008B10C221A701A781F
:10148000043A5A7000F07CFD224B18607379052BEA
:1014900003D1214B4FF4C8721A80204B4FF47A725B
:1014A0001A80237843F0080323701D4B1A7822F02A
:1014B00002021A70B3689B071ED51A4B1A4A1C46C3
:1014C0001A6000F065FC282000F039FE069A013A07
:1014D0000692F6D12168154B48781D780246012303
:1014E000954203D30133082B0244F9D1104A1370FB
:1014F0008A7853430F4A138019B0BDE8F08F00BFBC
:1015000001200008C9150008D5040020191600089C
:10151000251600085C030020B802002058160020A1
:101520005C160020D0030020A8100020CD0300206E
:101530007C000020CE0300201E4B2DE9F0431A78DA
:101540001D460AB31C4B07781E781C4B93F800C04D
:1015500002231B4A03F10108D45C344104F00F0458
:10156000BC420CD20B2C0AD812F8039012F8088057
:1015700002EB840209EA0C0408EB04241461023330
:10158000102BE6D100232B7003788B420FD90C4B24
:1015900093F8400060B10B4A890012780B44186937
:1015A00002B1400800F5777080B2BDE8F0830020FA
:1015B000BDE8F08300010020B4070020B50700203B
:1015C000CC070020B607002007299ABF024B33F84A
:1015D00021000020704700BFDC010020024B53F8BF
:1015E0002100C0F3CF0070478401002008B5074BED
:1015F00053F8210006F04EFD054906F0A3FD05490C
:1016000006F098FC06F08AFF80B208BD1C0100209D
:101610000000203F00005C44014B33F8110070478C
:1016200062030020024B03EB4101B1F84200704716
:10163000CC070020032810B5114B0FD8114A1268AF
:1016400094888C420AD2D2888A4207D9012202FAAF
:1016500000F093F85A20104383F85A0093F85A3058
:101660000F2B0CD1064B002283F85A20064B998889
:1016700008B2142802DD1439998010BD9A8010BD7B
:10168000CC070020E4080020A4070020024B9A8821
:1016900001329A80704700BFA4070020074B1A68E8
:1016A000074B1178B3F9040053780B4403EB830321
:1016B0009842D4BF00200120704700BFE4080020FA
:1016C000A4070020064BB3F90400064B1B681B78E7
:1016D00003EB83039842D4BF00200120704700BF72
:1016E000A4070020E408002010B50446FFF7EAFF35
:1016F000002814BF2046002000F0010010BD024B5E
:1017000001221A72704700BFA4070020014B187A0B
:10171000704700BFA4070020034BB3F90400D0F1C9
:10172000010038BF00207047A4070020014B0022B1
:101730009A807047A4070020016B0346C26810B569
:10174000406941B1196C541A005D013918BF0A464D
:10175000C0B21A6410BD196A405C0131B1FBF2F4E9
:1017600002FB1412C0B21A6210BD026B03691AB1F7
:101770005168013B026C02E0C169026A013B881AB0
:101780001840C0B27047436B13B190F844007047E3
:10179000826A436AD31A58425841704710F80A3C8B
:1017A0000133DBB20A2B00F80A3C0CD910F8123CCA
:1017B00033B910F8131C044A02EB4102A2F842307C
:1017C000002300F80A3C7047CC070020334A10B5CC
:1017D000136C90681944081A40F68C239842916063
:1017E000D060516013463CD9127893F945108A4273
:1017F0000BD1111F082908D893F84610182901D8D1
:10180000013103E083F8442002E0002183F8461010
:1018100093F944108A421CD1204991F84710C1B174
:10182000002191421E4806DA03EB8104246920F866
:1018300011400131F5E7511E00EB410116308142A4
:1018400003D0002421F8024FF9E716490878013047
:10185000087083F84520002201211A7083F8471090
:1018600010BD92F84710B9B1A0F2EF2440F2DA515E
:101870008C4208D811780B2905D80B1D0131117045
:1018800042F8230010BD002283F847209918043243
:101890000020302A0861F9D110BD00BF6805002082
:1018A0000E080020E8090020024B1A6C0132114496
:1018B0001964704768050020024B53F820301B68FC
:1018C0001980704790060020074BA1F57A7153F8F4
:1018D00020304FF47A701A681B894B4393FBF0F366
:1018E0009BB21380704700BF9006002038B50C688B
:1018F0000546204609F04EFB214602462868BDE811
:10190000384009F04FBB094BDA68D10709D4DA68CF
:10191000520708D4DB6813F0100F0CBF042003201B
:101920007047012070470220704700BF002002402E
:101930007C4B70B51B78012B0CBF0325002599BB90
:10194000048C24F001042404240C0484038B048CF0
:101950009BB223F0F30343F0010343EA0515724BF6
:10196000A4B2984215D003F50063984211D0B0F1AB
:10197000804F0ED0A3F5983398420AD003F58063C8
:10198000984206D003F58063984218BF24F00A04F9
:1019900001D124F0020444F00104224305830284AF
:1019A000038B23F00C033AE004293FD1048C5E4BF7
:1019B00024F010042404240C0484018B048C21F4EE
:1019C00040710905090D41F480719842A4B241EAC1
:1019D000053512D003F5006398420ED0B0F1804F68
:1019E0000BD0A3F59833984207D003F58063984253
:1019F00003D003F58063984207D124F0200444F01B
:101A0000100444EA021292B204E024F0A00444F06C
:101A10001004224305830284038B23F440631B04D8
:101A20001B0C0383038B9BB2038370BD0829018CBD
:101A300037D121F480710904090C0184838B048C53
:101A40009BB223F0F30343F0010343EA0515364B41
:101A5000A4B2984212D003F5006398420ED0B0F1C0
:101A6000804F0BD0A3F59833984207D003F58063DD
:101A7000984203D003F58063984207D124F40074A0
:101A800044F4807444EA022292B204E024F4206414
:101A900044F48074224385830284838B23F00C03F7
:101AA00038E021F480510904090C0184838B068CF1
:101AB00023F440731B051B0D43F4807343EA053583
:101AC000194BB6B2984212D003F5006398420ED07B
:101AD000B0F1804F0BD0A3F59833984207D003F5AF
:101AE0008063984203D003F58063984207D126F4BF
:101AF000005646F4805646EA023292B205E047F6B6
:101B0000FF54344044F48054224385830284838B01
:101B100023F440631B041B0C8383838B9BB283835E
:101B200070BD00BF64050020002C014038B510F8DE
:101B30000E2C044650F8043C52B9012200F80E2C39
:101B400020F80C1C197B18680222BDE83840EFE62B
:101B500030F80C2C20F80A1C891A89B220F8081CCD
:101B6000084A10F80F0C002502EB4002A2F84210C0
:101B700004F80E5C1868197B2A46FFF7D9FE04F8B2
:101B8000065C38BDCC070020CB78F0B5DA0648BF3C
:101B90008A78098803F00F0548BF154311F0FF0F3D
:101BA0001DD0046800220127974007EA0106BE42C3
:101BB00011D197004FF00F0C0CFA07FC05FA07F74C
:101BC00024EA0C04282B44EA070401D1466102E010
:101BD000482B08BF06610132082AE4D10460FF29BE
:101BE0001FD94468002202F108060127B74007EA1E
:101BF0000106BE4211D197004FF00F0C0CFA07FC02
:101C000005FA07F724EA0C04282B44EA070401D15B
:101C1000466102E0482B08BF06610132082AE2D182
:101C20004460F0BD2DE9F843564B0C460168013A7B
:101C3000D9658188A3F86010072A42D8DFE802F04E
:101C4000040A101822292F35B3F85C202280B3F83B
:101C50005E2013E0B3F85E202280B3F85C2005E03C
:101C6000B3F85C2052422280B3F85E20524205E075
:101C7000B3F85E2052422280B3F85C206280B3F851
:101C800060301DE0B3F85C2052422280B3F85E2041
:101C900012E0B3F85E202280B3F85C200CE0B3F8C9
:101CA0005C202280B3F85E2005E0B3F85E2052424B
:101CB0002280B3F85C2052426280B3F860305B420D
:101CC000A380314B1B78002B5AD1B4F9000006F0E9
:101CD000E5F98046B4F9020006F0E0F90746B4F9E8
:101CE000040006F0DBF9294D06462968404606F057
:101CF00029FAE9688146384606F024FA0146484642
:101D000006F018F9A9698146304606F01BFA01462B
:101D1000484606F00FF909F061FB696820804046EB
:101D200006F010FA29698146384606F00BFA01469A
:101D3000484606F0FFF8E9698146304606F002FAA7
:101D40000146484606F0F6F809F048FBA9686080AD
:101D5000404606F0F7F969698046384606F0F2F920
:101D60000146404606F0E6F8296A0746304606F086
:101D7000E9F90146384606F0DDF809F02FFBA080AE
:101D8000BDE8F883CC0700203C0000202805002097
:101D900010B5194B93F86220511C83F86210174953
:101DA00002F007024878164903EB420331F810109D
:101DB000A3F8641000231846124A9A5A02331044BA
:101DC000102B80B2F8D1C00806F068F90E4906F071
:101DD000B9F90E4906F06AFA0D4B04461B681878EB
:101DE00006F05CF90146204606F0ACF906F096FBD9
:101DF000084B187010BD00BFCC070020DC0300208A
:101E0000EC030020300800203333534000F07F45BE
:101E1000D0030020CD030020034B1B68DA79511C4E
:101E2000D9711344187A7047B004002010B5FFF739
:101E3000F3FF0446FFF7F0FF04EB002080B210BD73
:101E4000F0B5137C012B29D80C255D43144C0133CC
:101E500005EB040C9CF8086030421DD02D5D1DB1CF
:101E6000012D14BF022501250E4C4E7B04EB0514F9
:101E7000277B3740B7420FD14F686668B7420BD314
:101E80008F68A668B74207D815709460C2F804C07E
:101E9000D16013741046F0BDDBB2D3E70020F0BD73
:101EA0001000002030D100082DE9F0478278C67874
:101EB0001E4BC2F1640802EB820C54425FFA88F8B0
:101EC0004FEA4C0CC6F16409A4B203F11807A5B29D
:101ED00028B2002804DC002D14BF1546012500E0BF
:101EE000454600FB00FA6D430AFB06FA9AFBF5F53E
:101EF0004D4468434FF00A0A90FBFAF0604480B208
:101F000058800D88B1F802A000B2C5EB0A0A00FBA8
:101F10000AF04FF47A7A90FBFAF0054423F8025F56
:101F20000A34BB42A4B2D2D1BDE8F087AA03002094
:101F300010B544780078002303FB03F1193961439D
:101F400001F6C4115943414340F6C41291FBF2F12A
:101F5000034A22F813100133072BEDD110BD00BF47
:101F60008C03002010B5044C2068FFF7E1FF2068C7
:101F70000249BDE8104097E7880300207410002054
:101F800010B5094A094913688C6812689342F8D160
:101F9000074A106811684FF47A725043001BB0FB77
:101FA000F1F002FB030010BDA00F002010E000E0E4
:101FB0001005002038B5104C0123054684F8403048
:101FC000FFF7DEFF636F41F28832C31A9342A367C3
:101FD00084BF002384F87C3094F87C30EDB20F2B62
:101FE0006067E55403D1054B01221A7038BD024ADF
:101FF000013382F87C3038BDCC070020000100207E
:1020000010B50446FFF7BCFF0E4B41F28831D3F800
:102010008020C3F88000821A8A42C3F8842084BFDB
:10202000002283F8882093F88830074A142BD45470
:1020300003D1064B01221A7010BD024A013382F807
:10204000883010BDCC070020C5010020C40100204D
:1020500010B50446FFF794FF174AD2F88C30C2F847
:102060008C00C31AB3F57A6F84BF002382F89030D6
:1020700092F8903023B9A82C1CD110490B7006E0BF
:10208000022B02D10E490C7001E0242B01D80D491E
:10209000CC540133DBB282F89030094A12785200F6
:1020A0000532934206D1044B002283F89020034B63
:1020B00001221A7010BD00BFCC0700205C01002077
:1020C000820100205D01002038B50446FFF758FF6B
:1020D000124B40F6C411D3F89420C3F89400821A2E
:1020E0008A4284BF002283F8982093F898200AB986
:1020F0000F2C11D10A480021017052B1094D182A44
:10210000154405F8014C04D1012283F8981002709F
:1021100038BD013283F8982038BD00BFCC070020BD
:10212000010100200201002038B50446FFF728FF16
:102130000546FFF725FF401BA042FAD338BD10B576
:1021400004462CB14FF47A70FFF7EEFF013CF8E73C
:1021500010BD2DE9F04106460F4690460025EBB232
:10216000434512D20024E3B2B34209D2084B3846A9
:10217000DA68013482F40052DA60FFF7E0FFF2E738
:102180003C20FFF7DCFF0135E9E7BDE8F08100BF47
:10219000001001400B490B7813F0010F03F004020B
:1021A0000AD072B9980707D443F004030B70064BAA
:1021B0001A88064B1A8070471AB90220FF210122A3
:1021C000C7E770475C16002030030020C6030020DC
:1021D00040F2DB1568430C4C08B54FF48043636153
:1021E0004FF400532361851EE368284683F480433F
:1021F000E360E36883F40053E360FFF7A0FF192076
:10220000FFF79DFFF0E700BF0010014008B503682D
:102210001B68984708BD064B10B504462146186850
:10222000FFF7F4FF034B1B689A7954409C7110BD73
:10223000B4040020B004002038B5044624200D4624
:10224000FFF7E9FF4D20FFF7E6FF002C084C0CBF1D
:102250003E202120FFF7DFFF2368002228469A71E5
:10226000FFF7D9FF236893F84900BDE83840D2E76B
:10227000B004002001460020DEE7F8B50E4E0F4CFA
:102280000F4DC1B20746306884F89910FFF7BEFFC2
:102290002B6894F899109A7930684A409A71C7F37C
:1022A000072184F89910FFF7B1FF2B6894F8991073
:1022B0009A794A409A71F8BDB4040020CC070020F6
:1022C000B0040020F8B51B4D1B4C1C4F0646C1B294
:1022D000286884F89A10FFF799FF3B6894F89A10E1
:1022E0009A7928684A409A71C6F3072184F89A10AF
:1022F000FFF78CFF3B6894F89A109A7928684A4057
:102300009A71C6F3074184F89A10FFF77FFF3B6884
:1023100094F89A109A7928684A409A71310E84F894
:102320009A10FFF773FF3B6894F89A109A794A4025
:102330009A71F8BDB4040020CC070020B00400203E
:1023400010B5441E14F8011F21B1034B1868FFF7A4
:102350005DFFF7E710BD00BF60050020014B186866
:1023600054E700BF20090020054B1B6803EBC000A9
:1023700090F9063019420CBF01204FF0FF30704732
:10238000E80800200A4B1A6802EBC002D379FF2B41
:1023900007D008490978994203D9074A32F813004F
:1023A00004E00728D4BF908840F2DC5000B27047A8
:1023B000E8080020D5040020620300202DE9F04F3A
:1023C0000C68836889B0D0F800A0D0F80480064675
:1023D000204603938B4608F0CBFF0746204609F0C2
:1023E0003BF8DBF804408146204608F0C1FF054673
:1023F000204609F031F8DBF8082004461046019227
:1024000008F0B6FF019A8346104609F025F83946D0
:102410000290584605F096FE39460490029805F061
:1024200091FE59460590484605F08CFE02990690AB
:10243000484605F087FE29460790584605F082FE7B
:102440000146504605F07EFE21468346069805F07B
:1024500079FE0146059805F06DFD0146404605F000
:1024600071FE0146584605F065FD214683460498F5
:1024700005F068FE0146079805F05AFD01460398ED
:1024800005F060FE0146584605F054FD30600299A3
:1024900005F1004005F056FE0146504605F052FE9B
:1024A00021468346079805F04DFE0146049805F045
:1024B0003FFD0146404605F045FE0146584605F001
:1024C00039FD21468346059805F03CFE01460698F5
:1024D00005F030FD0146039805F034FE01465846EC
:1024E00005F028FD21467060504605F02BFE294678
:1024F000044609F1004005F025FE0146404605F07E
:1025000021FE0146204605F015FD394604462846C1
:1025100005F018FE0146039805F014FE014620461A
:1025200005F008FDB06009B0BDE8F08F2DE9F84F67
:102530002E4E04463768384608F01AFF05463846DE
:1025400008F08AFF76688046304608F011FF83461F
:10255000304608F081FFD4F80490064629464846E4
:1025600005F0F0FDA76882464146384605F0EAFDD1
:102570000146504605F0DCFC21688246584605F0CD
:10258000E1FD41460446484605F0DCFD314605F0D4
:10259000D9FD0146204605F0CDFC314604463846BB
:1025A00005F0D0FD294605F0CDFD0146204605F099
:1025B000C1FC0146504608F0DDFF0D4905F0C2FDA3
:1025C0000C4905F073FE0C4B196805F0B3FC0B4980
:1025D00005F06CFE08F002FF83B21A0444BF00F558
:1025E000B4739BB218B2BDE8F88F00BF1803002087
:1025F0000000E144DB0F4940540500200000204169
:10260000034B1A78510744BF22F004021A70704736
:102610005C16002070B5FFF755F838B3144C237AD8
:102620000BB9A38070BD134D2E78C6F38000FFF761
:102630005BF890B1104B46F002061A680F4B5189B7
:102640002E7019805189598052899A800C4A1268DB
:102650005288DA80E3880133E380FFF71FF810B96E
:102660002B785B0702D4BDE87040C9E770BD00BF9E
:10267000A40700205C160020A007002062030020B1
:10268000E40800202DE9F04102780346202A00F1F9
:102690000100F9D0092AF7D02D2A02D10346414D75
:1026A00004E02B2A08BF03464FF07E551E46002447
:1026B000334616F8012BA2F13007F9B209290DD8DB
:1026C0003949204605F03EFD0446384605F0E6FC53
:1026D0000146204605F02EFC0446E9E72E2A17D1D4
:1026E000314F334616F8010B3038C2B2092A0FD8E1
:1026F00005F0D4FC394605F0D9FD0146204605F029
:1027000019FC29490446384605F01CFD0746E8E750
:102710001A7802F0DF02452A38D15A782D2A02D1E0
:102720000233012604E02B2A14BF013302330026B2
:10273000013B002713F8012F303AD1B2092903D801
:102740000A2101FB0727F5E7B7F59A7F28BF4FF469
:102750009A77B8464FF07E51B8F1070F07D908466F
:10276000124905F0EFFCA8F108080146F4E707F06C
:10277000070737B108460C4905F0E4FC013F014664
:10278000F7E72EB1204605F091FD04E04FF07E51B1
:10279000204605F0D7FC0146284605F0D3FCBDE8ED
:1027A000F08100BF000080BF0000204120BCBE4C73
:1027B000F0B50124B0FBF4F58D4201D34C43F9E7A9
:1027C0000026DCB1B0FBF4F504FB1500B4FBF1F41A
:1027D0001EB9002D01DC002CF3D1092D03F10107F6
:1027E0005FFA85FC04DD002A0CBF5725372500E081
:1027F000302565441D7001363B46E2E71C70F0BD94
:10280000F0B50124B0FBF4F58D4201D34C43F9E758
:102810000026DCB1B0FBF4F504FB1500B4FBF1F4C9
:102820001EB9002D01DC002CF3D1092D03F10107A5
:102830005FFA85FC04DD002A0CBF5725372500E030
:10284000302565441D7001363B46E2E71C70F0BD43
:1028500070B50646B6FBF2F40846154614B120469C
:10286000FFF7F6FF05FB1464024B1B5D00F8013B0C
:1028700070BD00BF38DF00082DE9F041069C002B39
:1028800006460F460CBF4FF020084FF03008234695
:1028900013F8011B09B9154603E0002AFBDD013AD4
:1028A000F6E7002D04DD30464146B847013DF8E724
:1028B00014F8011B11B13046B847F9E7BDE8F081C3
:1028C00080EAE073A3EBE0738B4206DB002801DDB6
:1028D000401A704702D00844704700207047034BED
:1028E0009A6822EA00009860704700BFA40F002099
:1028F0002DE9F041038A87890446BFB20D461F4087
:10290000002F36D0B7FA87F34FF00042DA40D243B7
:1029100091B21B3B21821740042BF1D8DFE803F072
:10292000221F1C1903006B6A33B103F1FF38002327
:102930001FFA88F86B6203E0B4F82C801FFA88F85D
:102940002E6A002EDCD033683046414698477668C0
:10295000F7E72868A18E08E06868218F05E0A8687D
:10296000A18F02E0E868B4F84010036889B2984784
:10297000C6E7BDE8F0810C4B800A98420CD003D822
:10298000B0F5801F0ED00BE0084B984206D04933BB
:10299000984205D1002070470220704703207047FD
:1029A000FE20704701207047010010000200100057
:1029B000044B53F820301BB107289CBF1B681980BB
:1029C000704700BFC006002010B5054C00202188CC
:1029D000FFF7EEFF61880120BDE81040E8E700BF87
:1029E000620000202DE9F0410F88002347FA03F22E
:1029F000D2072BD58A7803F0070512F0100F18BF05
:102A000091F803C002F00F0618BF46EA0C06AD00AD
:102A10004FF00F0C0CFA05FC06FA05F5DC0850F82F
:102A20002480282A28EA0C0C45EA0C0540F824509A
:102A300005D101229A40C46824EA020205E0482A2E
:102A400004D101229A40C4682243C2600133102B92
:102A5000CCD1BDE8F08100BF08B503F057FB00F012
:102A600087FDBDE808400F2014210122FFF771BB4C
:102A7000A04A2DE9F04F13689F4903F59C439F4DF1
:102A800020330B60AB6885B013F4807F174604D009
:102A90009B4B1B681B681B699847AB6842F201049B
:102AA0001C405CB9974E337873B1954B1B681B681B
:102AB0001B68984703F00EFC347005E0924B1A78BF
:102AC00001321A7003F006FCAB68DA0405D58F4BAF
:102AD0001B68DB0701D4FFF793FD8D4B3C6818683A
:102AE000037C83B18B4A013B32F91300A0F57A7065
:102AF000B0F57A7FA8BF4FF47A7020EAE07005F055
:102B0000CDFA85492FE0AA68170435D57E4A516869
:102B1000611A002930DB04F59C41203151607F4966
:102B20004E797F4931F81660417CB6B296FBF1F0E0
:102B3000117A013101F00F0111720A4450721846E6
:102B4000784A9A5C01331044102B80B2F8D100B25D
:102B500090FBF3F000B26428A8BF642020EAE07084
:102B600005F09CFA704905F0A1FB704905F0EAFAFE
:102B700005F0D4FC6E4B1880AB68DE0510D56D4BAC
:102B80009C426D4C08D923681B681B6A984718B98A
:102B900023681B685B6A984723681B685B699847D2
:102BA000AA68564BD404B5F8DC100AD55948B3F8D6
:102BB0001A31B0F90620581A82420ADD19448A42B5
:102BC00005E05449B3F81C31B1F906209A42C0F22D
:102BD000C1830122002395F823A195F82411B5F8AB
:102BE0001C41B5F81E619B464A4F4FEA9B0BF85EAD
:102BF0000233A042C4BF6BF07F0B5FFA8BFBB04285
:102C0000B8BF4BF0400B082BEED13F4C637E5B45C9
:102C100004D1A37EF92B03D8013300E00023A3766F
:102C2000464B84F819B093F80080384F9946B8F1B4
:102C3000000F14D13B68D80707D582B9404B1B78E9
:102C4000DB070CD5FFF7A6FA09E03D4B1B785E07C2
:102C500005D511B1FFF7D4FC01E0002AFAD0A37E1C
:102C60002949142B374E40F0A280354B1AF1000A47
:102C70001B7818BF4FF0010A03F0040303F0FF02B2
:102C800093B1B8F1000F00F09280BBF15F0F02D159
:102C9000FFF7B6FC8BE0BAF1000F00F08880BBF1C3
:102CA0007D0F40F08480F3E7BBF1570F0BD1264B2B
:102CB0004FF47A721A80254B1B6813F0080376D103
:102CC000234A138073E0AB68580749D5BBF15A0F0C
:102CD00046D1204B187818B11A7001221E4B54E0CF
:102CE000CA7E1E4B82F00102CA760AB104224CE071
:102CF00006224AE05016002004020020A40F002003
:102D000000020020F80000206808002004040020D1
:102D1000FC0000206203002000007A44DC03002055
:102D2000EC030020710800200000C84200C07F446E
:102D3000D8040020404B4C00B00700204C0000207D
:102D40005C16002034020020581600200C020020DF
:102D500030030020E5020020E7020020E602002008
:102D6000BBF15D0F00F09C82BBF15B0F00F09A821B
:102D7000BBF15E0F0BD1032295E2BBF1A70F40F030
:102D8000B282AE4B1A7842F004021A700FE0BBF127
:102D9000560F01D1FFF760FE99F80030002B00F0CC
:102DA0009982BBF16F0F40F08E82FFF7F3F9AB68A9
:102DB0005B0732D5E37EA3B1A14B1B78580710D532
:102DC000A048A14BB0F90620B3F81C319A4208DDA7
:102DD0003B6813F0010304D19C4A322111809C4AC4
:102DE000D3763B68D9030AD59A4B1A782AB99A4AFE
:102DF000127812B9954A3221118001220CE0964BCB
:102E00001A7852B18E4A127802F0040202F0FF01E1
:102E10001AB91970914B01221A70D6F8009000234C
:102E200009F1750A3B6009F1770698460AF1020339
:102E300003EB080113F808204B7816F8010C9A42AE
:102E40000AD2314602F080FA30B116F8023C012273
:102E50009A403B6813433B6008F10408B8F1A00FA7
:102E600006F10406E2D17E4B1B7843B13B68DFF8E4
:102E7000088213F0020F7B4E40F0A18196E109F227
:102E80001512019209F58B769846019A16F8010CF5
:102E9000531C03EB080113F808204B789A4229D2FF
:102EA000314602F051FA28B396F802C030796E4BE1
:102EB0000CF1FF3C4FF00C090CEB4C0C09FB00F93A
:102EC0009C44634B96F803B003F11C0A0AEB09011A
:102ED0004A6862450ED000220AF809B08A600122D1
:102EE00002FA00F093F84C20C1F804C022EA000076
:102EF00083F84C0008F10608B8F1480F06F1060601
:102F0000C3D15A4B5A4A1E68D2F800A0DFF86C8130
:102F10004FF000099B46D8F80030002B00F03D81AF
:102F20001978002900F03981D8F80420C2EB0A0290
:102F3000002A0CDB0AF5FA72C8F80420012202FA12
:102F400009F294F84C0020EA020284F84C2018F8A8
:102F5000040C5A780430C0B2002A40F0E580394AA7
:102F600032F910000190B5F81A01019A00F1C80C6D
:102F7000624501DD9B7814E0019AC838824202DA8A
:102F80009B785B420DE0012303FA09F394F84C208F
:102F900022EA030384F84C300AF5FA73C8F80430C7
:102FA000FBE094F84C2042FA09F2D20700F1F580D8
:102FB000002B304ACCBF02200120013910700A29B1
:102FC00000F2E380DFE801F0060F1B28315C6E8021
:102FD000929CA60032781344FA2BA8BFFA2323EA66
:102FE000E373337007E072781344642BA8BF642343
:102FF00023EAE37373703046FEF79AFFC5E0F27878
:1030000030461344642BA8BF642323EAE373F370B0
:10301000216DFEF749FFB8E032791344642BA8BF55
:10302000642323EAE3733371AFE072791344642BB2
:10303000A8BF642323EAE3737371A6E01A02002099
:103040005C16002062030020A40F0020CC020020A8
:1030500068080020E4020020E5020020E7020020CA
:103060005B160020C403002050D100088803002014
:10307000A00F0020E60200200C020020880800209B
:10308000616D4A781A44C82AA8BFC82222EAE272AF
:103090004A700A781344C82BA8BFC82323EAE373F5
:1030A0000B7072E0616DCA7A1A44C82AA8BFC822A0
:1030B00022EAE272CA728A7A1344C82BA8BFC823D4
:1030C00023EAE3738B7260E0616D4A7D1A44C82A7B
:1030D000A8BFC82222EAE2724A750A7D1344C82BAF
:1030E000A8BFC82323EAE3730B754EE0626D9178A5
:1030F0000B44C82BA8BFC82323EAE373937044E0B2
:10310000626D117B0B44C82BA8BFC82323EAE3736D
:1031100013733AE0626D917D0B44C82BA8BFC8239E
:1031200023EAE373937530E0012A2ED19B784FF4A4
:10313000966292FBF3F38F4A32F91000B0F5617F8B
:1031400005DB40F633029042B8BF024601E04FF47F
:103150006172A2F5617292FBF3F3DBB2864A581CEE
:103160000C29107011D194F858209A420DD0042BDC
:10317000824A28BF02230A2184F8583001FB032326
:103180000633CBF80030FEF7EDFE012303FA09F316
:1031900094F84C20134384F84C3009F10109B9F13B
:1031A000040F08F10C087FF4B6AE5FE6AB68D805F3
:1031B00014D5734B1B681B689B68984770B1D8F88F
:1031C00000309B070AD5338813F001020CD16D49FA
:1031D00043F00103E26522660B8006E0338801229A
:1031E00023F00103338000E000223B68590710D52B
:1031F0007AB1328822F0010102F0020289B292B261
:10320000318052B9E26522665E4A41F002011180C6
:1032100003E0328822F00202328032885A4912F0EA
:10322000030F4FF4804014BF48610861D8F80010C4
:1032300011F00A0F21D0DF0609D554070AD442F055
:1032400004023280514A1188514A118002E022F072
:10325000040232809806328806D5510607D44949BF
:1032600042F040020A8002E022F0400232805A0618
:1032700003D5464A1188474A118013F4006F3388FA
:1032800014BF43F4807323F4807333806B79082B6D
:1032900001D00E2B6AD1338823F04003338065E0E0
:1032A000012200E002225FFA82F808F1FF3385F87C
:1032B0006C3602F02BFF00F05BF902202821424619
:1032C000FEF747FF73E5BAF1000F03D0BBF17E0FA5
:1032D0003FF46BADBBF1970F7FF44FAD2E4B4FF426
:1032E000C8721A8063E50023BBF1BB0F039301D1C1
:1032F000022304E0BBF1B70F04D14FF6FE73ADF823
:103300000E300CE0BBF1BE0F01D1022305E0BBF192
:10331000BD0F7FF44CAD4FF6FE73ADF80C30336843
:10332000BDF80C10B3F854200A44A3F85420BDF89B
:103330000E10B3F856200A44A3F8562002F0E6FE19
:1033400000F016F90F2014210122FEF702FF0023DE
:10335000A3762CE5114B00220021DA651A665A6625
:103360009A66DA6619675967996733E405B0BDE86C
:10337000F08F00BF62030020E60200200C16002040
:10338000B0070020C40300200010014030030020DB
:10339000DA040020C6030020B802002068080020DC
:1033A00000230E49DAB2595C4F2903D001330A2BAE
:1033B000F7D11A460A4B83F82821002283F82921E5
:1033C0004FF4E132C3F82C21C3F83021C3F8342183
:1033D000C3F83821522283F83C2170475DDF000892
:1033E000A40F002007B5064B06480093064B074A7A
:1033F0001968074B02F055FD03B05DF804FB00BFF0
:1034000091DD000867DF0008840000207CDD0008F3
:1034100088DD000810B50446204607F0BBFD10F01B
:10342000FF0F06D10C4B0D481978BDE8104002F093
:1034300038BD204607F003FE02280CD8064B0A22AE
:103440001870074B074C02FB0030074B0630186022
:10345000FEF788FDE0E710BDC008002083DF00080C
:103460000C160020B9E1000888030020234B70B53A
:1034700019684FF47A73B1FBF3F1214B21481A78A4
:10348000214B224D1B7802F00CFD214B214819687D
:10349000214B2E68B1FBF3F102F003FD00241F4B1A
:1034A000E2B253F8221049B1012303FA02F2324288
:1034B00002D01B4802F0F5FC0134F0E72A689207BD
:1034C0000DD5184A1848127803EB8203196A02F0E6
:1034D000E8FC164B197A11B1154802F0E2FC1548C8
:1034E000FEF72EFFBDE87040134B14481A88144BAA
:1034F00092B219884FF4D26302F0D3BCA00F00201F
:10350000CD03002094DF00087C0000200C02002086
:1035100080000020D2DF000840420F0074D1000874
:10352000F0DF00085D160020F4DF0008A402002090
:10353000FEDF0008D5E50008BC04002002E000081A
:103540006003002010B50748FEF7FAFE0024064B82
:1035500006481A19E15852680C3402F0A2FCD82C23
:10356000F5D110BD34E00008C0D100084AE00008E1
:103570002DE9F84302F0A8FD10B90A20FEF728FE55
:10358000A64D4FF4D2622846A54907F0B9FC95F83C
:103590006C364FF4DA72022B84BF002385F86C3648
:1035A00095F86C369F4E02FB035303F5A87393F80E
:1035B00050203360022A84BF002283F8502093F801
:1035C0005030994A13700A2202FB0353974A03F2C0
:1035D0006E631360AB6842F201021A403AB944F2DA
:1035E00008021A401AB98D4A43F400539360AB683D
:1035F000DB0703D54FF40050FFF771F9AB685F04A8
:1036000009D50820FFF76BF94FF40050FFF767F971
:103610000120FFF764F9AB681C0706D54FF4005092
:10362000FFF75DF90120FFF75AF9AB6898040ED552
:103630004FF40040FFF753F94FF40060FFF74FF9E4
:103640004FF48030FFF74BF94020FFF748F9784CF2
:10365000784B27461C6003F06FF9774B04F1180292
:1036600001201A6003F008F90146012002F0F4FC81
:10367000002849D0022003F0FFF80146022002F0A2
:10368000EBFC002840D0202003F0F6F80146202073
:1036900002F0E2FCAB68190601D5002834D01020F6
:1036A00003F0EAF80146102002F0D6FCAB681A07D6
:1036B00000D548B3042003F0DFF80146042002F0EF
:1036C000CBFC30B9082003F0D7F80146082002F0FF
:1036D000C3FCAB685B0503D400231A46194609E016
:1036E0000028F9D110E079B90121C00708D40C33C2
:1036F000182B0BD051481844007A8407F5D5F2E70F
:103700000132D2B2022AF2D9FFF74AFEFEF72AFCB2
:103710004B494C4B366819604B4B06F10409C3F812
:10372000009006F1750200238846D15C39B9D018A3
:103730008478C078844202D2444B197002E004338A
:10374000A02BF2D1424A434B1A603278424B012AF5
:1037500003D0022A03D0414A02E0414A00E0414A34
:10376000414C1A6006F5D3732360404B00229A80C7
:103770003F4B404A06F5D771136006F5B37262609D
:10378000A3F12202A2602E333B4A236106F5D873CF
:103790001160A361C4F80C806761B5F8F00004F013
:1037A00079FC2062B5F8F20004F074FC96F8583009
:1037B00004F11C02237796F874306062637795F801
:1037C0002531C4F82C9084F828302C4BC4F838806C
:1037D0001A602B4B06F160021A6006F16403236342
:1037E00006F25D136363B6F8620104F057FC01460C
:1037F000244804F05BFD244904F0A4FC234B244935
:103800001860F06D04F09EFC01464FF07C5004F00F
:103810004DFD204B1860BDE8F88300BFA40F0020C9
:1038200000F8000834020020C008002088030020AF
:10383000B4100020FC000020B8040020100000207C
:1038400074100020B8080020BC0800204C000020A4
:10385000981000205002002074000020F949000850
:103860005D4C0008D54D0008E4080020A4070020A6
:103870009C100020BC02002004050020F002002063
:103880004C030020000061444C3D0F44F80400202C
:10389000DB0F49403C03002010B50446204607F0EA
:1038A00079FB10F0FF0F07D10B4B0C4893F86C1607
:1038B000BDE8104002F0F5BA204607F0C0FB022830
:1038C00008D8054B064C83F86C0602F01FFCFFF786
:1038D0004FFEE3E710BD00BFA40F002087DF000804
:1038E000B9E100082DE9F04F7F4985B0054607F0A2
:1038F00019FB7E49002828460CBF0124072407F045
:1039000011FB7B490028284608BF022407F00AFB68
:10391000002808BF0424E10740F1B380754802F095
:10392000C0FA0020FFF75EFD734F744802F0B9FA49
:10393000734802F0B6FA7A79724B734803EB82034C
:10394000D3F8201102F0ADFA3869002104F08EFDA1
:1039500000285CD13D460646D5F81080002140463F
:1039600004F084FD00284ED1013668483146D5F870
:1039700014B0D5F818A0D5F81C9002F092FA404681
:10398000002104F07DFD10B1614802F08AFA694619
:10399000404602F0F7FF01465E4802F082FA5846C0
:1039A000002104F06DFD10B1594802F07AFA694621
:1039B000584602F0E7FF0146564802F072FA5046B8
:1039C000002104F05DFD10B1514802F06AFA694629
:1039D000504602F0D7FF01464E4802F062FA4846D0
:1039E000002104F04DFD10B1494802F05AFA694631
:1039F000484602F0C7FF0146474802F052FA0C2E33
:103A000005F11005A8D14548711C02F04AFA444856
:103A100002F047FA434DD7F8088055F8041F19B152
:103A2000414802F03EFAF8E70D46404B53F8256056
:103A300056B10123AB4013EA080F03D03C4831468E
:103A400002F02FFA0135F0E73A4802F02AFA31463F
:103A50007B1893F8103104AA1344374A8A5C013169
:103A6000082903F8102CF3D10023344869468DF857
:103A7000083002F016FA324802F013FA402002F041
:103A8000D7F9A2071AD52F4802F00BFA2E4802F0F8
:103A900008FA2E48FFF700FF2D4802F002FA2B48E3
:103AA00002F0B8F82B4802F0FCF9284802F026F999
:103AB000234802F0F6F9802002F0BAF963070FD527
:103AC000254802F0EEF9254802F0EBF91F48FFF710
:103AD000A1FC1B4802F0E5F94FF4807002F0A8F950
:103AE00005B0BDE8F08F00BF52E00008C9EC000847
:103AF00059E000085FE00008A40F00206DE0000816
:103B00007FE0000874D100088BE0000896E0000810
:103B100088E10008FBDF00084DE000089EE0000897
:103B2000B0E00008F0D20008C0E00008F4D20008BD
:103B3000CEE00008DBE0000841E50008E7E000080F
:103B4000D5E50008F0E0000803E10008B9E100084D
:103B500011E100081BE100082AE100083BE1000830
:103B60002DE9F047784B86B01A789A46DFF8EC9149
:103B7000BAB901238AF80030744BD9F8002059688B
:103B8000914204D019690C33914218BF00230221DD
:103B900059726F4B6F48DA63FEF7D2FB6E48FEF73F
:103BA000CFFBD9F8000003685B689847002800F055
:103BB000C7806A4B664C186803689B689847092859
:103BC000014601D03F2853D14FF00008266C644FC6
:103BD00045462EB163483968324607F0E3F910B91B
:103BE000B84605B93D46604B0C379F42F1D3EDB165
:103BF000D5F800E0D8F800C0236C55481EF80370D3
:103C00001CF80310B94211D15A1C51B92D2B08D8F8
:103C1000026403442027024483F8447082F844106D
:103C200004E0234483F844702264E5E7236C0BB17D
:103C3000454512D04D48FEF783FB454509D855F858
:103C40000C0BFEF77DFBD9F800000921FEF7DEFA28
:103C5000F3E74148FEF774FB0026236C9E42A0D296
:103C6000404BD9F80000995DFEF7D0FA0136F4E731
:103C7000236C33B904283DD104F1440002F0D6FB93
:103C80005EE00C2801D13A4886E70A2901D00D29C7
:103C90004CD13848FEF754FB236CE218002382F81D
:103CA000443094F84420232A17D00493324B2D4EED
:103CB000009303A82A4912220C23039607F0C3F9A4
:103CC000054638B1006807F065F90130AB6830444B
:103CD000984702E02948FEF733FB224800213022B2
:103CE00007F017F9002323649AF80030002B7FF4C3
:103CF00055AF25E00C28C6D07F2903D151E72F2BE3
:103D00003FF64FAFA1F12002D2B25E2A3FF649AF93
:103D100013B920293FF445AF5A1C2264D9F800009A
:103D20001C4484F84410FEF771FA3AE77F29E6D183
:103D3000013B23640022234483F8442010482EE7EB
:103D400006B0BDE8F08700BF5B1600201000002021
:103D5000E40800204DE1000885E10008600500202E
:103D6000C0D100082809002098D200088AE1000884
:103D70008FE10008D5E50008ED1800089AE1000879
:103D8000B6E100082DE9F04FBB4ABC4C85B0106885
:103D9000516802AB03C3DFF8089300214FF4D262ED
:103DA000204607F0B6F804F5A873C9F80030B44B04
:103DB0000025DFF8F0B21D7004F26E63CBF800301E
:103DC00003236371A3604FF41673A4F8F030FA2351
:103DD000A4F8F2302A23A4F8EE304FF4FA73A4F8D2
:103DE000F630202384F8F4306E2384F804312B233A
:103DF00084F80531212384F806314FF4C873A4F800
:103E0000083140F24C43A4F81C3140F26C73A4F822
:103E10001E31192384F8253140F27E43A4F8D030B6
:103E200040F23A73A4F8D2304FF47A73A4F8D43045
:103E300040F27E53A4F8D63040F2EA53A4F8D830CA
:103E400040F2B45301273226552240F2DC514FF0A4
:103E50001E0AA4F8DA304FF47A532270A4F81A112B
:103E6000A4F8DE3084F8EC7084F821A184F8247181
:103E700084F82771A4F8DC60A4F8E0608DE80600FF
:103E8000FFF78EFA40F6AC53A381D9F800304FF01B
:103E900028081720A573187683F80EA083F80FA0C2
:103EA00058761D7083F8048083F805800B20019AF2
:103EB0001872142058721875502098776420D8779B
:103EC0004FF0080E782083F813E05873DFF8D8C15C
:103ED0006C484FF00E0E9A7183F80AE02D224FF0D5
:103EE0005A0E4FF00A0A1A74DE715A7783F80BE003
:103EF000DA7583F821709D765D74DD769D741D778B
:103F000083F815A083F80C80C3F824C0D863186424
:103F10004FF08240D8624FF07C5098635A48C3F803
:103F200028C05864594A5A48DFF880C100991A637A
:103F30005A639864C3F84CC084F86EE64FF0410EA3
:103F400084F87066A4F8761684F86FE684F87256E2
:103F500084F8735684F8715684F874569A664D4AFC
:103F60000421DA664C4A83F858101521D86583F885
:103F70007470A3F85450A3F85650A3F8525083F825
:103F8000608083F8618083F864101A67434802F008
:103F90005BFCD9F800604FF44873A6F86231C8237F
:103FA00086F8A7314FF49663A6F8A83140F2D933CA
:103FB000A6F8AA3140F6430386F86071A6F8AC3142
:103FC00086F85D5186F85E5186F85F8186F8645107
:103FD00086F8A6A133465F464FF47F72A3F86621A8
:103FE0004FF4FA62A3F8682102A940F2DC52A3F868
:103FF0006A214A5D013583F86C21082D4FF0FF02DC
:1040000083F86D2103F10803E6D1012386F8AE3170
:1040100086F8AF3186F8B0310023E2181033002162
:10402000C02B164D1161F8D1314605F541704FF4A2
:10403000DA7206F065FF314605F597604FF4DA72E3
:1040400006F05EFF3B6805F5CF625968186803C249
:10405000198922F8021B1968C5F88216596851603F
:104060001B891381012385F85433022385F8083511
:1040700005B0BDE8F08F00BF44D30008A40F0020B6
:10408000C00800208FC2753DCDCC4C3D9A99193F98
:104090000000A040F6287C3F3D0A773FBAE10008C7
:1040A000340200208803002000002040000040402F
:1040B00008B50548FEF744F9FFF764FE02F026F85C
:1040C000BDE8084002F0DFB8C3E100082DE9F04F79
:1040D000AE4E85B03778032F14D9AD4BAD48B3F948
:1040E0000410B0F904200029B8BF49426FF06303FF
:1040F0005B1A9A4204DB01F164039342A8BF1346A2
:1041000083801FE0012F1DD8A34BA44C1B78013BDB
:10411000142B00F2DF81DFE813F09100DD01DD01F7
:1041200068009F00DD01DD012F01DD01DD01DD0102
:10413000DD01DD01BD00DD01DD01DD01DD01DD01B0
:104140009F01B601924B9649B3F806A0914B0968BE
:10415000B3F80280B3F80090B3F904B0914C029127
:104160000025BD4204F11004CED20FFA8AF003F00C
:1041700095FF54F8101C03F0E5FF03460FFA88F092
:10418000019303F08BFF54F8081C03F0DBFF019B45
:104190000146184603F0CEFE03460FFA89F001935C
:1041A00003F07CFF54F80C1C03F0CCFF019B01468C
:1041B000184603F0BFFE029A034692F900000193ED
:1041C00040420BFB00F003F069FF54F8041C03F0BD
:1041D000B9FF019B0146184603F0ACFE04F078F9E4
:1041E000714B23F815000135BBE702210420FEF7CF
:1041F000BBF8684D0121AF8878431FFA80F804208E
:10420000FEF7B2F86D8800FB05801FFA80F80420E5
:10421000FEF7B8F84044208102210520FEF7A4F8FB
:104220007843012187B20520FEF79EF800FB057058
:1042300087B20520FEF7A6F838440BE005200121DF
:10424000FEF792F8534B9D88684385B20520FEF730
:1042500099F8284460813DE1544B00201D68FEF729
:1042600091F8DFF8608195F90630B8F9022032271D
:10427000534393FBF7F3184420800120FEF782F8A4
:1042800095F90E30B8F90020534393FBF7F7384403
:1042900060801FE1464B1B7813F0040F454B02D1A1
:1042A0001B689B880BE01968394A0B88B2F9062015
:1042B00049889A4203DB9142B4BF0B461346E3811F
:1042C000E289394B394F1A803B4B1B681D7845B347
:1042D0000220FEF757F83A68B2F91030518A984236
:1042E00003DB0BB29842B8BF0346344909684889DA
:1042F000C3EB000E274B0FFA8EFED9880FFA81FC14
:10430000F44501DA0D4401E001DD4D1BDD8092F939
:104310001620B3F906305343642293FBF2F318449A
:10432000A080274B1B88DB050CD5194B1A88D7F8C2
:104330000090E28022819A88184F62815B88032571
:10434000A38101E0134BF1E709EBC50393F90630B4
:10435000B7F90680284608FB03F8642398FBF3F8B6
:10436000A7F80680FEF70EF801354044072DF880C7
:1043700007F10207E8D1ADE00D4B1B7813F0040FF5
:104380000C4B21D11B689B882AE000BF341600200B
:104390009A03002058090020000500206200002038
:1043A00004050020E006002036160020E808002062
:1043B0005C160020F0080020F4080020F808002017
:1043C000C4030020200300201968AD4A0B88B2F90D
:1043D000062049889A4203DB9142B4BF0B4613463C
:1043E000E381E289A74BA84D1A80A84B03201B88C4
:1043F0000121DF0503D5FDF7B7FFA14F02E0FDF76F
:10440000B3FFA34FB7F80280022100FB08F01FFAA8
:1044100080F90320FDF7A8FF3F88012100FB0790EA
:10442000E8800420FDF7A0FF00FB08F002211FFA3E
:1044300080F80420FDF798FF00FB07802881032007
:10444000FDF7A0FFE3881844E0800420FDF79AFF01
:104450002389184420813DE001210420FDF784FFD9
:104460008B4D6F88784387B204202781FDF78AFF40
:104470003844208101210520FDF776FF2D8868430F
:1044800085B26581E2E6824B0325B3F80490984635
:1044900028460221FDF768FF00FB09F0012187B2E1
:1044A0002846FDF761FFC5F106035B0838F81330B5
:1044B00000FB037087B224F815702846FDF762FFF1
:1044C000384424F815000135072DE1D16C4BDA880A
:1044D0006C4B1A806F4DDFF8E491AB6813F0200F3E
:1044E00034D00020FDF74EFF208080460120FDF7EC
:1044F00049FF694B644F1B6860801A0626D5674BDD
:104500001B681B7813F0020F654B23D0D9F800C04D
:10451000B3F900109CF90E209CF906C0B3F90230E3
:104520004A43CCF1000C03FB0CF3322192FBF1F275
:104530006FF0310C92B293FBFCFC9444E04493FB8B
:10454000F1F1A7F800800A4410447880D9F80010EF
:10455000002319E0D9F80010B3F902C091F9062040
:10456000B3F900300CFB02FC32229CFBF2FCE0446D
:10457000A7F8008091F90E104B4393FBF2F2E3E7AA
:10458000E2520233102B0CD0E05E31F9232001EB14
:10459000830790427F88F3DB3AB28242A8BF02468B
:1045A000EEE73E4B1B681B785B0704D43549347833
:1045B000088801231BE03B4B00241F780423043FA1
:1045C000FFB25FFA87F84FFA88F2D4420BD4364A2A
:1045D00003F10109381932F813105FFA89F9C0B2F2
:1045E000FEF7E6F94B460134042CECD1DEE7A3429A
:1045F00008D231F9132000B28242A8BF104680B21F
:104600000133F4E7294B4FEA44081A68AB6803F416
:1046100080550395244D03F01009254BB5F906602C
:10462000244D1B782F68244D03F00403DBB2D5F82A
:1046300000C002930023434562D0B2F802A004B246
:10464000544505DD0F4CC0EB0A0A1D5B55441D5354
:10465000039D0C4C002D33D07D8931F903A0AE426F
:10466000CBBFBCF802509588B2F802B0BCF800B0DD
:10467000AA4503DBDA45B4BF55465D46E55238E04E
:104680009A0300203616002062000020C403002098
:1046900058090020A40F002004040020FC0800207A
:1046A000200300206705002062030020F00800209E
:1046B0005C160020F8080020EC080020E808002024
:1046C00031F903A01588B2F802B0AA4503DBDA4538
:1046D000B4BF55465D46E55204EB030ABC89A642C9
:1046E00007DAB9F1000F01D1148800E09488AAF824
:1046F0000040029C14B9044C1C5BCC5202339AE774
:1047000005B0BDE8F08F00BFDC0400200C4B07B5FE
:104710001B68196819B10B4A9069014391619A8825
:104720009868ADF8042002228DF8072004220DEBD2
:1047300002018DF80620FEF755F903B05DF804FB81
:104740004C0500200010024010B50A4C23681BB134
:10475000FFF7DCFF00232360074B1B7813B1012B0D
:1047600003D010BD4FF4006201E04FF48052034BC0
:104770001A8010BD4C0500205005002000000020CC
:10478000F8B50468054620460E461746FEF7F3F8CE
:10479000032845D82B7B9B089AB246B94FF0020CF0
:1047A0000CFA03F3A18989B221EA0303A3810A2148
:1047B00001FB00211B4B43F82160043143F82170B9
:1047C00046B12A7B0225920805FA02F2A1890A4322
:1047D00092B2A281282202FB003000F12002EFF306
:1047E0001286502383F312880023C1180D6915B176
:1047F00015600A6904320433102BF6D100231360CC
:10480000F3B283F31188036A23B1A3899BB243F007
:10481000010304E0A38923F001031B041B0CA38103
:10482000F8BD00BF580E002070B5046D4279A38911
:1048300002F0040123F400531B041B0C0546866898
:1048400086B0A38101F0FF0021B14FF480604FF4E6
:10485000005100E0014612F0010F14BF04230023B1
:1048600012F0020F1CBF43F008039BB212F0080FB6
:10487000228A18BF0C2392B222F4405211432182A3
:10488000A28992B222F4B05222F00C0210430343E8
:104890009BB2A381A38A01A823F440731B041B0CC1
:1048A000A38202F087F91949049A039B8C4208BF3E
:1048B0001346A2891921594312B2002AB4BF7600C7
:1048C000B600B1FBF6F16423B1FBF3F2120110095B
:1048D00003FB1011A08900B2002806DAC9003231AA
:1048E000B1FBF3F303F0070305E009013231B1FB3B
:1048F000F3F303F00F031A4392B22B6D22819A89CE
:1049000092B242F400529A8106B070BD0038014064
:10491000417189E7816087E730B51049104A0C780A
:10492000104B84B19C6815680444A54214D31268E6
:1049300000209A600C4A0870117809B10139117091
:1049400001221A7330BD98681468C830844203D3BA
:104950001268012008709A6030BD00BF1104002069
:10496000A00F002058090020E602002037B51D4D99
:104970008DF807306B7B8DF8062002AA8DF80400B5
:104980008DF805101A4412F8042C443AD2B20F2ABA
:1049900009D81549022B31F8124008D894B12046A5
:1049A000FFF7BAFF0EE0022B4FF0C804F7D90F4B08
:1049B0001A68AB68121B934204D20A4A002353734D
:1049C0000B4A13702B7B012B00D04CB96B7B022B55
:1049D00002D8044A01335373064A00232B73137021
:1049E00003B030BD580900204CD30008A00F0020B0
:1049F000E6020020110400202DE9F04F8BB009934E
:104A00008A4B0792B3F90220B3F90030002AB8BFED
:104A10005242002BB8BF5B429A42B8BF1A46844B41
:104A200003921B88814603F00302069203F0020200
:104A300003F0010392B205930023089219461E4623
:104A4000184604931F461A46069C002C41D0022AA1
:104A50003FD0764C079F0D5F7C426D00A54203DB83
:104A60003C46A542B8BF2C46724DDDF824A031F972
:104A700005C03AF90150CCEB040404EB050C99F89D
:104A80000750642405FB0CF595FBF4F599F81B40E1
:104A90006FF004076743BD4205DB04EB8404A542C5
:104AA000B4BF2F462746644D5C59644442F2107CE3
:104AB0006445A8BF6446DFF898C16445B8BF644642
:104AC0005C5199F811506C4324130494069C012CFA
:104AD0003BD05A4D55486D5E594C85EAE576A6EBBC
:104AE000E576B6F5206F085E19F802C053F8048029
:104AF0001DDC022A15D05026464396FBFCFC0426FA
:104B000095FBF6F5C5EB0C0CE0444E4EB8F57A5F1C
:104B1000A8BF4FF47A58B045ACBF44F80380E650C4
:104B200007E080EAE076A6EBE076642EE3DD002580
:104B3000E550434C1E597D2496FBF4F609EB020424
:104B4000A47A6643402496FBF4F6089CB4B1022A8A
:104B500068D0DDF80CA0DDF810B00AFB00F40AFB09
:104B600006F8CAF5FA7505FB074405FB0B854FF4FB
:104B7000FA7C94FBFCF495FBFCF506E0059C002C0C
:104B800050D0022A4ED0049D3C46DFF8B0C04FF012
:104B9000040B31F80CC00FFA8CF898FBFBFADFF825
:104BA000B4B012F80BB00BFB0AFA6FF04F0B9AFB84
:104BB000FBFAA244CDF804A0DFF89CA0042431F94C
:104BC0000AB021F80AC0CBEB08080AF1080C98FBE0
:104BD000F4F80AF114041C5953F80CB00AF1140A41
:104BE000A34453F80C40C34443F80A40164CDDF884
:104BF00004A0145D013204FB0BFB20249BFBF4FB9F
:104C0000CBEB050B114DDA44032A43F80C8021F855
:104C100005A003F1040301F102017FF415AF0BB00D
:104C2000BDE8F08F35460446AFE700BF9A03002089
:104C3000C403002020030020C408002054030020E7
:104C4000CC08002080C1FFFFA803002058090020E5
:104C5000F0D8FFFFA2030020680900202DE9F04FE3
:104C600089B00793524B0291B3F904300192039338
:104C7000504B06461B8803F0010103F002039BB270
:104C800004934D4B0691B3F800A04FF6FF714FEA25
:104C90001A13B1FBF3F1002305911D461946022DAD
:104CA00008D1029FDDF80CC07C791B340CFB04F4A6
:104CB000641129E03E4C019A31F9048057424FEAD1
:104CC0004804BC4203DB1746BC42B8BF27463B4CF6
:104CD000DDF81CC00C5F3F1B3CF901403A19069CF3
:104CE0007CB9029C277907F11B0408FB04F4049F9C
:104CF00024114FB190F811C00CFB02F704EB2724EC
:104D000002E0C479544324112D4FDFF8C48031F9F7
:104D100007C004279CFBF7FCCCEB040C0AFB0CF44B
:104D200096F80AB053F80870E4120BFB0474254F90
:104D3000B4F5001FA8BF4FF40014BC42B8BF3C46F6
:104D4000214F10F80590DA5943F8084043F807C09E
:104D5000C2EB0C0809FB0CF9DDF814C001350CFBA3
:104D600008F807F10C0C1837DA5953F80CB04FEA71
:104D7000A818934453F80C20C344DA51377D032D0F
:104D800007FB0BF74FEA272707EBE91707EB64341C
:104D90000E4F43F80C80CC5306F1010601F10201DD
:104DA00003F104037FF47BAF09B0BDE8F08F00BFCF
:104DB0009A030020C4030020600300202003002089
:104DC000540300200000E0FF88090020580900205B
:104DD000CC0800202DE9F04F89B00793714B814634
:104DE00018880492039103F055F96F4903F0AAF96A
:104DF000029002994FF07E5003F058FA002406907A
:104E00004E462546A046B8F1020F684B0BD10399D8
:104E1000B3F904004A790A32504303F03FF9644978
:104E200003F044FA35E0049A5F5F53429F4203DB8C
:104E300013469F42B8BF3B465E4AAA5E9B1A079A3A
:104E4000505F184403F02AF95B4903F02FFA5B4BDB
:104E50008346B3F800A01AF0010F04D0D9F844102B
:104E600003F070F915E0039B18791430784303F0D0
:104E700015F94F4903F01AFA1AF0020F074609D044
:104E8000D9F84810584603F05DF90146384603F05A
:104E900051F807464A4BDFF84CB1585F03F0FEF873
:104EA000484BD96803F04EF982465146384603F024
:104EB0003FF8316A074603F045F9029905903846F4
:104EC00003F040F9F16A03F03DF954F80B1003F0D8
:104ED00031F83D49074603F0D3FA30B938463B492B
:104EE00003F0ECFA10B1394F00E0374F4BF8047083
:104EF000DFF8F4B0504654F80B1003F019F844F8FA
:104F00000BA0069903F01EF90BF10C03E2580BF10C
:104F1000180B54F80B10824610460192009303F0D0
:104F200009F8514603F006F8019A009B44F80B205B
:104F300044F803A0264903F0B9F9B16B03F002F974
:104F40002449824603F09CFA38B95046224903F0BE
:104F5000B5FA20B1DFF880A001E0DFF878A005986D
:104F6000394602F0E7FF514602F0E2FF06F036FA5A
:104F70001A4BB0F57A7FA8BF4FF47A709842B8BF49
:104F8000184608F10108164BB8F1030FE85204F176
:104F9000040405F1020506F104067FF434AF09B0FC
:104FA000BDE8F08F60030020BD3786359A030020EE
:104FB000000048422003002000002041C4030020DC
:104FC000540300203802002000007AC300007A4316
:104FD00000004040000096C30000964318FCFFFF0D
:104FE00058090020D8080020AC090020F0B5934CE7
:104FF000934A23689D8AADB2E9B211F0010F36D011
:10500000198821F400610904090C1980198889B2F2
:1050100041F480611980002182F86810894908787C
:105020008949B8B192F8690018B988480078FF2812
:1050300010D1012082F8690085480078022804D147
:10504000188880B240F400601880097841F00101AE
:10505000198216E1097801F0FE0119827B4B1B7859
:10506000FF2B00F00E81FF2382F8683009E18F07E3
:1050700040D5BFF35F8F76490878C0B2012816D1BA
:10508000704D2D789DB192F8695085B1198821F441
:1050900080610904090C1980BFF35F8F198B19888F
:1050A00082F86A0089B241F4007119801DE0188B02
:1050B000BFF35F8F087802280CD16248007848B1AE
:1050C00092F8690030B1198821F480610904090C53
:1050D0001980D0E00978032907D15A49097821B10C
:1050E00092F86910002940F0C680998889B241F48D
:1050F0008061C5E04E0764D5012182F86A105149EC
:10510000097800293ED092F8691000293AD0504918
:1051100092F8680009784F4D022919881FD921F4A7
:1051200080610904090C19801F8A2E68C1B2FFB280
:1051300040B23754188880B240F4007018808B1C3D
:1051400082F86830236828681D8A013149B2EDB2BF
:105150004554998889B241F4806199802CE089B2E4
:1051600041F4007119801E8A2D68C1B2F6B240B2B6
:105170002E541B8A481C40B2DBB203312B5482F8F8
:10518000681019E092F8691011B93349097851B1E2
:10519000198889B241F40071198092F8683001339E
:1051A00082F8683008E0198889B241F4807119806A
:1051B000234B012183F8691021680B88D805FCD4A2
:1051C0005FE001F0400101F0FF06214809B32149E9
:1051D000B3F810C00F6892F868105FFA8CFCCDB27B
:1051E0006E1C49B2F6B207F801C082F86860077811
:1051F00076B2F11C8F4205D1998821F480610904AF
:10520000090C99800378B3423BD1023582F868508B
:1052100037E0290635D592F868104DB26F1C1FD0C3
:105220000E4E01313668C9B2755D82F86810EDB274
:105230001D82007849B2884223D11CE0500E002024
:1052400068090020430E0020400E0020410E00207F
:105250004C0E0020480E0020420E0020440E00207C
:10526000144982F868600978C9B21982124909782C
:1052700009B9017829B9998821F480610904090CD8
:1052800099800E4B92F9681018780D4B421C914290
:105290000FD1002283F8692093F86A3033B1226875
:1052A000938823F440731B041B0C9380054B00224E
:1052B0001A70F0BD410E0020430E00204C0E00205D
:1052C000680900204D0E002070B50E4620211546BD
:1052D00005F053FE0446B8B1441C204605F0AFFE6D
:1052E000B0F5617F05DB40F634039842A8BF18464D
:1052F00001E04FF461701923A0F5617090FBF3F0A9
:1053000030702B7801332B702046202105F035FEBC
:105310000446B8B1441C204605F091FEB0F5617F0B
:1053200005DB40F634039842A8BF184601E04FF46D
:1053300061701923A0F5617090FBF3F070702B7809
:1053400001332B70204670BD104B043033F9103000
:10535000B3F5617F05DB40F633029342A8BF1346E5
:1053600001E04FF4617308781922504300F2833052
:10537000984208DA4878504300F283309842B4BF2C
:105380000020012070470020704700BF620300200A
:105390000D4B0278D9684378C943C1F30221C1F1AA
:1053A000040103FA01F1094B0901C9B21A4482F858
:1053B000001302780120510902F01F0200FA02F2E4
:1053C00043F82120704700BF00ED00E000E100E05D
:1053D000F8B5074605F0DEFD044638B91A4B1B4800
:1053E0005A791B4B013A53F8221028E038461949E4
:1053F000224605F0D7FD60B91748FCF7A1FF174C0E
:1054000054F8041F19B1164800F04BFDF8E7154891
:1054100005E000250E4B53F8256026B91248BDE87B
:10542000F840FCF78DBF38463146224605F0BAFDFC
:1054300001350028EED1044B0C485D713146BDE8C2
:10544000F84000F02EBD00BFA40F002056E5000874
:1054500098D200085FE300086AE5000894D20008CB
:10546000F0DF0008D5E500087DE5000892E50008BA
:1054700037B582880446836810060D4606D529494B
:105480004FF4DA7091F86C1600FB0133D10504D5A6
:1054900025490A20097800FB013302F03F02042A63
:1054A00012D006D8012A0DD0022A2FD193F900106C
:1054B0002DE0102A0AD0202A0AD0082A26D1B3F9D2
:1054C000001024E0197822E0198820E019681EE015
:1054D0006946186801F056FA0146144800F0E1FCEC
:1054E000F5B1E06802F0DAFD694601F04BFA0146D9
:1054F0000F4800F0D6FC206902F0D0FD694601F0AB
:1055000041FA01460A4800F0CCFC09E000210948B4
:1055100000F0C7FC25B10848E168226900F0C1FC31
:1055200003B030BDA40F0020C0080020FBDF00083E
:10553000FADF0008A8E50008A4E500082DE9F0411D
:10554000002407462546104B3946E65804EB03086D
:10555000304605F05BFD58B10C48314600F0A1FC27
:1055600040460021FFF784FF094800F09AFC01350E
:105570001434B4F5166FE6D125B90648BDE8F041FC
:10558000FCF7DEBEBDE8F0811CD400087BE8000813
:10559000D5E50008ABE500082DE9F74F044605F016
:1055A000F9FC054620B1012818D123782A2B15D102
:1055B0005548FCF7C5FE0024544B5548E618E15801
:1055C00000F06FFC30462946FFF752FF1434514873
:1055D000FCF7B6FEB4F5166FEED192E020463D2101
:1055E00005F0CBFC002800F08780034613F8012C5F
:1055F000202A01D1013BF9E7451C2846C4EB030AE8
:1056000005F01DFD83462846FDF73CF800260546BB
:1056100014237343DFF8F49053F8097003EB09087F
:10562000384605F0B7FC03461A4620463946019332
:1056300005F0B8FC019B002855D15FFA8AF29A4226
:1056400051D1D8F80C0002F029FD0146284602F09D
:105650002BFF002845D0D8F8100002F01FFD0146AE
:10566000284602F017FF00283BD0B8F804309B060C
:105670004FF0140303FB0696B28858BF5D4614062C
:105680002946B36806D524484FF4DA7490F86C06BE
:1056900004FB0033D00504D520480A24007804FB1D
:1056A000003302F03F02042A0BD004D8013A012A49
:1056B0000CD819700AE0102A05D0202A05D0082A33
:1056C00004D1198002E0196000E01D6039461448D9
:1056D00000F0E7FB3046002103B0BDE8F04FFFF7D4
:1056E000C7BE104803E00136782E91D10E4803B0B2
:1056F000BDE8F04FFCF724BE204603B0BDE8F04FF4
:105700001CE703B0BDE8F08FC3E500081CD4000817
:105710007BE80008D5E50008A40F0020C0080020A1
:10572000D8E50008E3E50008ABE500087FB50446CE
:1057300005F030FC082824D100231F49E25C0968E9
:105740001144497801F00301022908BF203AE254CC
:105750000133082BF1D10025665D1848314605F06C
:105760000CFC28B101356019314605F006FC18B172
:105770001348FCF7E5FD1CE0082DEDD1204601F0B3
:1057800063F81048FCF7DCFD00230F4A04A91A4413
:1057900092F810210A440949595C0133082B02F898
:1057A0000C1CF2D10023094801A98DF80C3000F03F
:1057B00078FB04B070BD00BF8800002041E5000800
:1057C00003E6000823E60008A40F00204DE00008CF
:1057D0002DE9F04389B0044605F0DCFBC6B2002E8B
:1057E0006CD18B48FCF7ACFD8A4C2069002102F09B
:1057F0003DFE40BB01368848314600F052FB20692F
:1058000004A901F0BFF80146844800F04AFB606932
:1058100004A901F0B7F80146804800F042FBA069F6
:1058200004A901F0AFF801467C4800F03AFBE069BA
:1058300004A901F0A7F80146794800F032FB0C2ECC
:1058400004F11004D1D10025764C2F462B464FF0A1
:105850000008B04504F1100415DA184654F8101C7D
:1058600002F068FB54F80C1C8146284602F062FBEB
:1058700054F8081C0546384602F05CFB08F10108A4
:105880004B460746E5E76848019302950397FCF706
:1058900057FD002401ABE058644920F0004002F0BD
:1058A0000DFE634B634A0434002814BF10461846AB
:1058B000FCF746FD0C2CEDD15F4891E020465F4996
:1058C000052205F06FFB38B9524B0022034410301B
:1058D000C0281A61F8D197E020465949042205F002
:1058E00061FB06462046002E40D1202105F045FBF5
:1058F000002800F08980451C284605F04BFB344603
:105900008046504B53F824600EB94F4868E0284653
:1059100031465FFA88F205F045FB671C20BB3D4B22
:105920000021C2181030C02811619C46F7D1474BA6
:10593000002403EBC702D2F804E09846BEF1000F42
:1059400004D14348314600F0ACFA55E018F837303E
:105950009C42F6DA23010CEB0305103573440FCBA0
:10596000013485E80F00F1E73C46CAE705F067FB24
:10597000461E0B2E074643DC2046202105F0FDFA8B
:10598000054640B1451C2846FCF77CFE214B3F01F3
:10599000D851012400E004462846202105F0EDFA04
:1059A000054640B1451C2846FCF76CFE194B0134F6
:1059B00003EB061358612846202105F0DEFA054660
:1059C00040B1451C2846FCF75DFE124B013403EB49
:1059D000061398612846202105F0CFFA18B91D4812
:1059E000FCF7AEFC10E00130FCF74CFE094B032C39
:1059F00003EB0616F061F2D11748FFF7E9FE03E06A
:105A000016480C2100F04DFA09B0BDE8F08300BF44
:105A100040E60008A40F00206BE6000871E60008CD
:105A20004DE00008B80F002075E600080AD7233CB7
:105A30003CE6000838E60008D5E5000884E60008E2
:105A40008AE6000898D200087DE50008A8CB000887
:105A50008FE600089FE60008B9E10008D9E60008D3
:105A60002DE9F047054605F095FA324B0446D3F888
:105A700008809A4690B93048FCF762FC2F4B53F8E7
:105A8000241049B10123A34013EA080F02D02C4887
:105A900000F007FA0134F1E72A4821E028462A49B4
:105AA000224605F07FFA58B92848FCF749FC284CF3
:105AB00054F8041F0029EFD0214800F0F2F9F7E76D
:105AC0002B7800262D2B03BF013504F1FF344FF056
:105AD00001094FF00009194B53F8267027B91D48EA
:105AE000BDE8F047FCF72CBC28463946224605F0B5
:105AF00059FAE8B90120B040020601D51648EFE78F
:105B0000830501D51548EBE7B9F1000F03D0FCF789
:105B1000E6FE134804E040EA0800CAF8080011480D
:105B2000FCF70EFC39461048BDE8F04700F0B9B963
:105B30000136D0E7A40F002001E70008F4D20008E6
:105B4000F0DF0008D5E500085FE3000814E700086F
:105B5000F0D2000829E7000840E7000852E70008F3
:105B600066E7000870E700084DE0000870B50446DD
:105B700005F010FA08B9204830E020461F4905F02A
:105B800083FA00242646254678B12CB1012C06D193
:105B900005F055FA064602E005F051FA05461749A8
:105BA0000020013405F070FAEEE70B2D05D9BDE8B1
:105BB000704013480C2100F074B9012C08DC114B23
:105BC000294633F915201048BDE8704000F069B946
:105BD000A6F57A73B3F57A7F04D90C48BDE8704016
:105BE00000F05FB90A482946324600F05AF9054BE1
:105BF00023F8156070BD00BF79E7000888E1000850
:105C0000B3E70008DC040020D9E70008F1E700084A
:105C100013E80008F0B585B0074605F0BBF9C0B23F
:105C2000E0B90446324B04F11C021B68192003EB57
:105C30008203591D8D785A79454305F561759B7925
:105C40000095C978484300F56170019021462948C4
:105C5000013400F026F9282CE4D146E0384605F05E
:105C6000EEF927283DDC224B00F11C061B68781C4E
:105C700003EB8606202100238DF80F3005F07DF917
:105C8000751D044658B1441C204605F0D8F9152866
:105C900005D870719DF80F3001338DF80F30204614
:105CA000202105F06AF9044658B1441C204605F04D
:105CB000C6F90D2805D89DF80F30687001338DF8AE
:105CC0000F302046A91C0DF10F02FFF7FDFA9DF8D9
:105CD0000F30042B09D028460021042205F019F9C1
:105CE00003E00548282100F0DCF805B0F0BD00BF56
:105CF000340200202CE8000841E8000870B586B0A6
:105D0000054605F047F9C0B208BB044606236343C5
:105D1000444A03F58873126819201344591D4D78BD
:105D20009A7A454305F561755B7900958D786843EE
:105D300000F561700190C878029009793A480391A2
:105D40002146013400F0ADF80C2CDFD168E0284684
:105D500005F075F90B285FDC06267043314B00F522
:105D600088701E68202106440023681C8DF81730B7
:105D700005F003F9741D054658B1451C284605F089
:105D80005EF9032805D89DF81730607101338DF84E
:105D900017302846202105F0F0F8054658B1451C7B
:105DA000284605F04CF90D2805D870719DF817307C
:105DB00001338DF817302846611C0DF11702FFF7EB
:105DC00083FA202105F0D9F8054658B1451C28462C
:105DD00005F035F90C2805D89DF81730E07001332F
:105DE0008DF817302846202105F0C7F850B1013052
:105DF00005F025F90D2805D89DF8173020710133DD
:105E00008DF817309DF81730062B09D02046002159
:105E1000062205F07EF803E004480C2100F041F86A
:105E200006B070BD3402002057E8000841E80008C1
:105E300070B5064600240A4BE518AA8816420AD017
:105E4000E158084800F02DF828460021FFF710FB24
:105E50000548FCF775FA1434B4F5166FEBD170BD34
:105E60001CD4000877E80008D5E50008426A10B5A0
:105E70008469A154416A02690131B1FBF2F402FB69
:105E800014124262426B32B11368DB0708D4BDE8DA
:105E9000104000F0E1BD036DDA6842F08002DA6084
:105EA00010BD0FB42DE9F04F684A89B012AB1668E7
:105EB000674A53F8045B176804939B4629780029C6
:105EC00000F0B880252902D001353046B0E06C786A
:105ED000302C03D002354FF0000903E0AC784FF0CE
:105EE00001090335A4F13003092B4FF000081AD83B
:105EF000A4F13003DAB2092A07D80A2B13DC0A22EC
:105F000002FB083815F8014BF2E7A4F16103052BF9
:105F100002D8A4F15703F0E7A4F14103052B02D8FE
:105F2000A4F13703E9E76C2C03BF2C78012201357B
:105F30000022632C66D006D8252C77D0582C3FD071
:105F4000002C77D0BAE7732C63D002D8642C11D020
:105F5000B4E7752C02D0782C32D0AFE70BF1040AED
:105F600005ACDBF800000A2112B10022234613E041
:105F7000234620E00BF1040A05ACDBF8000072B107
:105F8000002806DA2D238DF8143040420DF1150358
:105F900000E023460A210022FCF732FC0DE0002835
:105FA00006DA2D238DF8143040420DF1150300E080
:105FB00023460A210022FCF7FBFBD34600941AE09B
:105FC0000BF1040303930DF1140ADBF80000102118
:105FD00032B1583C624262415346FCF711FC06E084
:105FE000B4F158035A425A415346FCF7E1FBDDF83D
:105FF0000CB0CDF800A03046394642464B46FCF77F
:106000003BFC5BE730469BF800100BF10404B847FB
:106010000AE0DBF800303046009339464246002360
:106020000BF10404FCF728FCA34647E73046214661
:10603000B84743E7074B186803681B69984700286F
:10604000F8D009B0BDE8F04F04B070470C0500204F
:106050000805002020090020F0B5142285B007466D
:106060000E461648002104F054FF154B00241A7AFE
:10607000E0B2013412B1511E0A40F9E71C7DD1B2E1
:10608000013214B1611E0C40F9E7421A002A0DDDFD
:1060900093E8070001AD85E807000A4C94E8070083
:1060A00083E8070095E8070084E80700034A3846BC
:1060B000314605B0BDE8F040FBF7C2BED409002070
:1060C000100000201C0000200E4B1A78552A16D113
:1060D0005A88B2F5D26F12D11A79BE2A0FD193F82D
:1060E0008C260020EF2A0CD113F8012B5040064AD1
:1060F0009342F9D1D0F1010038BF00207047002051
:106100007047704700F8000890FE00084A4B55227F
:106110002DE9F3411A704FF4D2625A80BE221A71EF
:10612000EF2283F88C26002283F88D2611461E4626
:10613000B35C0132B2F5D26F81EA0301F8D13E4B74
:106140003E4A83F88D163E4B04275A6002F188328E
:106150005A600020013F17F0FF075DD0384B342212
:10616000384CDA60C4F309037BB1331903F1784387
:10617000A3F57843D3F800804FF400500023019337
:1061800000F062FD0428E5D11BE04FF4302000F060
:106190005BFD0428DED12A4D4FF430202B6943F0FB
:1061A00002032B616C612B6943F040032B6100F00B
:1061B0004BFD2A6941F6FD73134004282B61D4D0AE
:1061C000C8E71F4D4FF400502B6943F001032B61CA
:1061D0001FFA88F3238000F037FD042812D1A31C96
:1061E0000193019B4FEA1848A3F800804FF4005038
:1061F00000F02AFD2B6941F6FE721A4004282A613C
:1062000006D0A7E72B6941F6FE721A402A61A1E782
:106210000D4B04349C42A5D1094B04281A6942F065
:1062200080021A6102D1FFF74FFF10B90A20FBF775
:10623000CFFF02B0BDE8F081A40F00202301674525
:106240000020024000F8000890FE000813B501226B
:1062500004460021006800F057F9236801A81A8855
:1062600092B242F001021A80637B00228DF8043062
:1062700001238DF805308DF806208DF80730FFF7E3
:1062800087F802B010BD10B50848FCF759F8084B64
:106290001C68236820461B69984718B90A20FBF739
:1062A0004EFFF6E7034A044BDA6010BD81E80008B0
:1062B000600500200400FA0500ED00E008B5044880
:1062C000FCF73EF8FFF722FFBDE80840DBE700BF20
:1062D0008DE800083F4A2DE9F84F916840F201131C
:1062E0000B4040F201118B4293460AD13A4B1A7D82
:1062F00093F815905A75B9EB020918BF4FF00109D0
:1063000001E04FF001094FF00008344B5FFA88F4C8
:106310001B78A3425CD9324B324E1B68324F23B9F3
:106320003B685B8926F814304FE03A68072C94BF2D
:1063300012F804A0A246294851469847DBF80830D5
:106340000546DB0509D5B9F1000F06D0274B5046AD
:106350001B6829461B68DB699847A5F2EE2240F2CC
:10636000DC5392B29A4288BF3B68DBF8082088BFB2
:106370005D8942F2010313402BB31D4B1978164B74
:1063800001F0030202EB840293F8760003EB420271
:10639000D5821A4620B9032915D9012183F8761030
:1063A00002EBC403198BDD8A02EB44020D44598BC6
:1063B0009B8B0D441D44ADB2A2F8785004232DB23E
:1063C00095FBF3F5ADB226F8145008F101089CE7EF
:1063D000BDE8F88FA40F0020D4090020D5040020C8
:1063E000BC07002062030020FC0000200002002007
:1063F00068080020094B30B59D68094B05F48055AD
:106400001868084B1C6800230DB1828800E0A28840
:1064100005495A520233182BF6D130BDA40F002083
:10642000EC080020F0080020DC04002008B5074834
:10643000FBF786FF064A00231370064A1360064ADC
:106440001370FFF7D7FFBDE808401CE794E8000889
:1064500028090020240900205B160020F8B500243C
:10646000224BE0B21F78B8420CD2214B33F8101007
:10647000204B53F820301BB10B2801D8DB6898471C
:106480000134EDE71C4B9B685B0304D41B4B4FF4BA
:1064900080421A61F8BD0025194E2B46EAB2BA4275
:1064A000F4D2726854689C4218D02046FCF763FA14
:1064B000EFF31283502282F3128812494FF0280C16
:1064C000A28C0CFB001092B201324262A28ADBB2B3
:1064D00092B242F00102A28283F3118856F8043F7F
:1064E00000221B6801351A802346D7E734160020A6
:1064F0003616002090060020A40F00200010014056
:106500008C060020580E0020254B10B55343254A19
:10651000254C12680139B2FBF3F20388013AA0421C
:1065200089B292B29BB212D004F50064A0420ED0A0
:10653000B0F1804F0BD0A4F59834A04207D004F5F9
:106540008064A04203D004F58064A04202D123F00D
:1065500070039BB2154CA04206D004F58064A042A3
:106560001CBF23F440739BB203800F4B818598427C
:1065700002850FD003F5006398420BD003F540630A
:10658000984207D003F58063984203D003F58063F7
:10659000984201D1002303860123838210BD00BFEE
:1065A00040420F0080000020002C014000100040FD
:1065B0002DE9F74FA24E0C46377805461146006884
:1065C00091469B4622467B1C06F8043BFFF79CFF46
:1065D000AB686868ADF8043018238DF8063001A95F
:1065E00002238DF80730FCF7FDF92B7B3F0106EB0A
:1065F000070A2C680C2B00F2F280DFE813F00D0084
:10660000F000F000F0004D00F000F000F00082001B
:10661000F000F000F000B600238C8A4823F001035C
:106620001B041B0C2384218CA288238B844223F01F
:1066300073034FEA03434FEA134389B292B243F024
:10664000700314D000F50060844210D000F5406063
:1066500084420CD000F58060844208D000F5806050
:10666000844204D021F0020141F0030107E021F04F
:106670000E0122F4407241F0030142F48072A280C4
:106680002383A4F834B02184238B23F008031B0454
:106690001B0C43F0080332E0238C6A4823F01003FC
:1066A0001B041B0C2384218CA288238B844223F49B
:1066B000E6434FEA03434FEA134389B292B243F4ED
:1066C000E04308D000F50060844204D021F02001AE
:1066D00041F0300107E021F0E00122F4406241F096
:1066E000300142F48062A2802383A4F838B0218470
:1066F000238B23F400631B041B0C43F400632383EC
:106700006DE0238C4F4823F480731B041B0C2384FF
:10671000218CA288A38B844223F073034FEA0343A6
:106720004FEA134389B292B243F0700308D000F5E8
:106730000060844204D021F4007141F4407107E00C
:1067400021F4606122F4405241F4407142F48052DD
:10675000A280A383A4F83CB02184A38B23F0080378
:106760001B041B0C43F0080338E0B4F820C0354A82
:106770002CF4805C4FEA0C4C4FEA1C4CA4F820C06F
:10678000B4F820C0A388B4F81C802CF4005C28F472
:10679000E6484FEA08484FEA0C4C4FEA18484FEADF
:1067A0001C4C94429BB248F4E0484CF4405C03D04B
:1067B00002F50062944203D123F4804343F4804302
:1067C000A380A4F81C80A4F840B0A4F820C0A38B38
:1067D00023F400631B041B0C43F40063A383AB7B13
:1067E00043B1B4F844306FEA43436FEA53439BB27A
:1067F000A4F8443023889BB243F0010323802B7B11
:106800000C2B14D8DFE803F0071313130A13131328
:106810000D131313100004F1340307E004F13803DF
:1068200004E004F13C0301E004F14003F35150465D
:10683000AAF80890CAF8044003B0BDE8F08F00BF82
:10684000640A0020002C014070B50546441E14F86F
:10685000011F61B1064E304604F08FFB0028F6D0D0
:10686000861B0448631B304480F81031EFE770BD8D
:1068700041E50008A40F002070B500220646284913
:106880001301585CB04204D00132072AF7D100202E
:1068900070BD244D0B4405F1C404102E0FCB84E8C9
:1068A0000F002B4617D007D8012E0DD0022E34D161
:1068B0001D4B1B689B680BE0202E27D0402E2CD14F
:1068C000194B1B681B6903E0174B1B685B6820E0D2
:1068D000C5F8C8301DE0154A1268127A042A1CD87F
:1068E000DFE802F00A0A030A0A00114AC5F8C820C4
:1068F000C5F8CC20032206E04FF4E132C5F8C820E9
:10690000C5F8CC20012283F8D12006E0064B1B6895
:10691000DB68C5F8CC30204670BD064870BD00BFAE
:106920006CD30008640A0020B8040020FC0000209A
:10693000A0860100280B00200F4970B500230C78B9
:106940001A46D8B2844205D00D7B854208BF01208B
:106950000CD100E000200C2505FB0010074D084E6F
:10696000154495F828510132755D05720133052BE8
:1069700001D0012AE5D970BD10000020A40F00202D
:106980005DDF000830B587B005460C4603A800213E
:106990000C2204F0BEFA2846002101F08FFD20B140
:1069A00028462A4901F0C6FA03E02846274901F0A3
:1069B000BFFA274901F0C6FB01F08AFD054685EACA
:1069C000E570A0EBE57069460A22FBF741FF002362
:1069D0009D420370ACBF20232D2368468DF80C30F8
:1069E00004F0D8FA012807D130238DF80D308DF846
:1069F0000E308DF80F300CE0022805D130238DF8D1
:106A00000D308DF80E3004E0032804BF30238DF8DC
:106A10000D30694603A804F0A3FA03A804F0BAFAFB
:106A20000338C5B22A4603A9204604F0DDFA002344
:106A300063552046074904F093FA03A920462944E8
:106A400004F08EFA204607B030BD00BF6F12033A43
:106A500000007A44C0E80008826A8169436B1144EF
:106A6000D960416A914203D98A1A5A60816204E06E
:106A700001698A1A5A6000228262002280F844204A
:106A80001A6842F001021A6070478A6810B50C6AF1
:106A9000036814430A6923F4FF4314434A6923F04B
:106AA000700314438A691443CA6914434A6A14433D
:106AB0008A6A224313430360CB6843600B68836098
:106AC0004B68C36010BD02684FF6FE73134003604D
:106AD0000023036043608360C3602A4B984222D046
:106AE000294B984229D0294B984230D0284B9842C4
:106AF00037D0284B98423ED0274B984206D153F8C6
:106B0000682C42F4700243F8682C7047234B98427B
:106B100006D153F87C2C42F0706243F87C2C70470D
:106B20001F4B984206D153F8042C42F00F0243F851
:106B3000042C70471B4B984206D153F8182C42F096
:106B4000F00243F8182C7047174B984206D153F8BF
:106B50002C2C42F4706243F82C2C7047134B984253
:106B600006D153F8402C42F4704243F8402C704751
:106B70000F4B984205D153F8542C42F4702243F83D
:106B8000542C7047080002401C00024030000240B4
:106B900044000240580002406C0002408000024065
:106BA000080402401C040240300402404404024035
:106BB000580402401F4B10B55A6802F00C02042A18
:106BC00003D0082A04D01C4A14E01C4A126811E0C1
:106BD0005A685968C2F38342C90302F1020201D420
:106BE000174906E0596811F4003F1449096818BFB5
:106BF00049084A4302605968124AC1F30311545CC0
:106C00000168E14041605C68C4F30224145D21FA2C
:106C100004F484605C68C4F3C224145DE140C16084
:106C20005B68C3F381331A44137CB1FBF3F1016158
:106C300010BD00BF0010024000127A0028000020A2
:106C400000093D004D00002010B50446FAF75BFE38
:106C5000012806D11CB1FAF756FE013CF8E70520E1
:106C600010BD002C08BF052010BD00BF2DE9F0416C
:106C70001D46A04B8CB09842884617465AD19E4C70
:106C80009E4BA26023609E4B20656361C033A3616D
:106C9000C023E36023619B4BA907A364E36403F56E
:106CA000484303F154032363A3F11403D3F8D42F0F
:106CB000636342F48042C3F8D42FD3F8D02F42F05C
:106CC0000102C3F8D02F4FF002038DF803304FF4C8
:106CD0000073ADF800304FF018038DF8023003D583
:106CE00089486946FBF77EFE1C232A078DF802308F
:106CF00003D585486946FBF775FE4FF48063ADF810
:106D0000003048238DF80230EB0703D57E486946F2
:106D1000FBF768FE0E238DF804300022012301A842
:106D20008DF805308DF806208DF80730724CFEF78F
:106D30002FFB52E0754B984240F0D880744B6F4A5D
:106D40009F601A60C022DA601A61724A18655A613F
:106D5000C0329A61704AAE079A64DA646F4BDA699E
:106D600042F40032DA615A6942F001025A614FF08E
:106D700002038DF803304FF00403ADF800304FF0FC
:106D800018038DF8023003D55F486946FBF72AFEE9
:106D90001C232C078DF8023003D55B486946FBF7AE
:106DA00021FE0823ADF80030E8074FF048038DF8C6
:106DB000023003D554486946FBF714FE26238DF8AC
:106DC00004300022012301A88DF805308DF806203B
:106DD0008DF80730FEF7DCFA4D4C0026012384F8CD
:106DE00044302662E661A6626662C4F82C80657152
:106DF000A760A6712046FDF717FD15F0090F31D0E9
:106E0000206B002826D0E36C039601934FF4805347
:106E10000A9380230693E36805960493202309933D
:106E200063690796029308960B96FFF74CFE01A93B
:106E3000206BFFF72AFE236B1A6842F001021A60EA
:106E4000226D918A89B241F0400191825B689BB2C8
:106E5000236407E0236D4FF6DF721A80DA6842F090
:106E60002002DA6015F00A0F2CD0606B28B3A36CF7
:106E7000002601934FF480530A93802306932369DD
:106E80000296049310230393059607960896099695
:106E90000B96FFF718FE606B01A9FFF7F6FD636B19
:106EA0001A6842F002021A605E605E60236D9A8A80
:106EB00092B242F080029A8204E0236DDA6842F0D6
:106EC0008002DA60236D29079A8992B242F4005257
:106ED0009A819A8A03D592B242F0080203E022F026
:106EE00008021204120C9A82204600E000200CB026
:106EF000BDE8F081003801404C0F0020DCD30008D1
:106F0000380B0020043801400008014000440040D4
:106F1000F80E0020B80C002004440040001002408D
:106F200013B5062204466B463B21682000F070FA38
:106F30009DF800209DF8013043EA022323809DF84C
:106F400002209DF8033043EA022363809DF8042069
:106F50009DF8053043EA0223A38002B010BD13B5AB
:106F6000062204466B464321682000F051FA9DF842
:106F700000209DF8013043EA022323809DF802207F
:106F80009DF8033043EA022363809DF804209DF8B6
:106F9000053043EA0223A38002B010BD2DE9F04F73
:106FA00087B099460746884615469DF840B0FFF7DA
:106FB00063FC02AE0446034600F1100E18685968DF
:106FC000324603C2083373451646F7D1237B0BB90B
:106FD00003950495384602A9FFF73EF8044608B920
:106FE000002031E04368586828B1384602A922469B
:106FF000FAF726FFF2E7A36894F800A01E781EB9FE
:10700000CDF800B0124804E0012E1DD11148CDF892
:1070100000B04B4641462A46FFF728FE03460028AB
:10702000DED00D4A067102EB8A02C2F800036268E4
:1070300050600A4842689A4204D002690C309A4271
:1070400018BF00204772184607B0BDE8F08F00BF98
:107050000038014000440040380B002010000020A0
:1070600013B5244B4000C0B283F8080302ACD3F838
:10707000180383F8091304F8012D0021012283F875
:107080000A23C3F80C4383F80B13C3F8104383F8A7
:10709000142383F8152383F8161348B382889205C6
:1070A00015D40288D4050DD447F2305201888905E1
:1070B00002D5013AFAD113E092B1028892B242F4B9
:1070C00080720280828892B242F44072828047F2DB
:1070D000305293F8151311B1013AFAD100E012B908
:1070E00000F086F904E0034B93F8160380F00100EA
:1070F00002B010BD380B002010B5174C23681BB12F
:10710000FDF704FB002323606B2180226820FFF73A
:10711000A7FF6420FBF713F8192100226820FFF76E
:107120009FFF6B2103226820FFF79AFF372102227D
:107130006820FFF795FF094B1A211A786820FFF79E
:107140008FFF1B2118226820FFF78AFFBDE810403F
:1071500068201C21102283E74C0500203D00002000
:1071600037B50622044603216B461E2000F050F975
:107170009DF801309DF80000154D43EA002000B253
:1071800000F08CFF296800F0DDFF01F0A1F99DF807
:10719000033020809DF8020043EA002000B200F096
:1071A0007DFFA96800F0CEFF01F092F99DF805304F
:1071B000A0809DF8040043EA002000B200F06EFFBA
:1071C000696800F0BFFF01F083F9608003B030BD53
:1071D0004000002007B52320FAF7B1FF6820752191
:1071E00001220DF1070300F013F928B19DF8070003
:1071F000B0F168035842584103B05DF804FB00BF8A
:107200002DE9F04F1421012834BF0646012601FB69
:1072100006F3DFF8D8A1DFF8C0B10AEB03025AF891
:1072200003301069CBF80030694B15891E70694B2B
:10723000B2F80A80DC6989B02043546848EA05073F
:10724000D8610222276120468DF80E1003A9019310
:10725000ADF80C708DF80F20FBF7C4FB019B4FF0CD
:1072600008099B46A268154203D10A20FAF75CFF81
:10727000F8E70A206561FAF757FF25610A20FAF757
:1072800053FFB9F10109EDD1C4F814800A20FAF7CF
:107290004BFF65610A20FAF747FF25610A20FAF7DC
:1072A00043FF0222C4F8108020468DF80F2003A966
:1072B0001C228DF80E20ADF80C70FBF793FB464BAB
:1072C000464A1C689442DBF8102008D142F40012B0
:1072D000CBF81020DBF8102022F4001207E042F473
:1072E0008002CBF81020DBF8102022F48002CBF8CB
:1072F0001020A38803A823F440731B041B0CA38055
:1073000023889BB243F001032380A588FFF752FC3A
:1073100025F03F050599324A2D04B1FBF2F22D0C00
:107320001543ADB2A5802388012523F001031B047A
:107330001B0C23802B4B03A8B1FBF3F34FF4967186
:107340004A439BB24FF47A71002B92FBF1F208BFD3
:107350000123013292B243F400432284A3832388A1
:107360009BB243F001032380238823F4816323F03D
:1073700002031B041B0C23804FF48043238114233E
:1073800003FB06A6737B00248DF80C308DF80D40AE
:107390008DF80E408DF80F50FDF7FAFF337B9DF806
:1073A0000F208DF80C308DF80D408DF80E401AB17D
:1073B00003A8FDF7EDFF07E0590903F01F039D4007
:1073C000094A203142F8215009B0BDE8F08F00BFD2
:1073D000540E002000100240500E002000540040C7
:1073E00040420F00804F120000E100E0F4D300089B
:1073F00008B5054B1A88013292B21A80034B1878EF
:10740000FFF7FEFE002008BDBC040020540E002043
:1074100010B54000204CC0B220702048204C0170B4
:10742000204800210170012020701F4C23601F4C58
:1074300023601F4B1A701F4B1F4A107019701F4991
:107440000868194630B383889C0515D40388DB058A
:107450000DD447F230530488A40502D5013BFAD17C
:1074600012E08BB103889BB243F48073038083885E
:107470009BB243F44073838047F23053107810B1CD
:10748000013BFBD100E013B9BDE81040B0E708783C
:1074900080F0010010BD00BF400E0020410E002012
:1074A000430E0020420E0020480E0020440E002013
:1074B0004C0E00204E0E00204D0E0020500E0020DD
:1074C000244A13B513681446998A89B20191019927
:1074D00011F4706F02D0204A01211170019A12F448
:1074E000E06F2AD01A8B9A8822F480621204120C60
:1074F0009A80019A910520D41A8892051DD41A8881
:10750000D0050FD51A88D105FCD41A8892B242F45E
:1075100000721A801A889205FCD4104B1878FFF775
:107520006FFE0AE01A8892B242F400721A809A88BA
:1075300022F440721204120C9A802268938A23F477
:1075400070631B041B0C9382054B00221A7002B05F
:1075500010BD00BF500E00204E0E0020540E002023
:107560004D0E002001480249FBF7C2B90008004057
:10757000D00E002001480249FBF7BAB900040040D0
:10758000A80E00204FF080400149FBF7B1B900BFC1
:10759000800E002001480249FBF7AAB9002C0140E7
:1075A000580E002001480249FBF7A2B9002C014007
:1075B000580E002038B5204CD4F8F0301D88ADB2FC
:1075C000AA0618D5D4F8CC201AB1988880B2904772
:1075D00011E09B88D4F8BC20D4F8B410DBB28B54F3
:1075E000D4F8BC20D4F8AC300132B2FBF3F103FB89
:1075F0001123C4F8BC302B061DD5D4F8C820D4F80C
:10760000C4100D4B8A4210D0D3F8B800D3F8F01054
:10761000805C0132C0B28880D3F8B010B2FBF1F0C8
:1076200001FB1022C3F8C82038BDD3F8F030DA6867
:1076300022F08002DA6038BD580E00200F4BD3F8DC
:1076400044211188090618D5D3F81C11D3F8180164
:1076500081420ED0D3F80C01405C0131C0B2908061
:10766000D3F80421B1FBF2F002FB1011C3F81C1196
:107670007047D36823F08003D3607047580E002012
:107680000C480D4B4FF400525A60D0F828214FF6A9
:10769000FE7311680B401360D0F81821D0F81C312C
:1076A0009A4202D0F430FFF7D7B9012380F838317D
:1076B000704700BF580E002000000240FFF700BFD7
:1076C000FFF7FEBEFDF792BCFDF790BC0F4B1A68AA
:1076D00042F001021A6059680D4A0A405A601A685D
:1076E00022F0847222F480321A601A6822F4802216
:1076F0001A605A6822F4FE025A604FF41F029A6020
:10770000044B4FF000629A60704700BF00100240C7
:107710000000FFF800ED00E0024B1A6801321A6029
:10772000704700BFA00F002008B5084BB3F8D80081
:1077300093F894260023D9B2914204D2044921F847
:1077400013000133F7E7FEF789FEFEE7A00F0020E4
:107750003616002081F0004102E000BF83F00043B4
:1077600030B54FEA41044FEA430594EA050F08BFDC
:1077700090EA020F1FBF54EA000C55EA020C7FEAA0
:10778000645C7FEA655C00F0E2804FEA5454D4EB1D
:107790005555B8BF6D420CDD2C4480EA020281EAE7
:1077A000030382EA000083EA010180EA020281EA1F
:1077B0000303362D88BF30BD11F0004F4FEA013171
:1077C0004FF4801C4CEA113102D0404261EB410180
:1077D00013F0004F4FEA03334CEA133302D0524206
:1077E00063EB430394EA050F00F0A780A4F10104C2
:1077F000D5F1200E0DDB02FA0EFC22FA05F28018FC
:1078000041F1000103FA0EF2801843FA05F35941E1
:107810000EE0A5F120050EF1200E012A03FA0EFC60
:1078200028BF4CF0020C43FA05F3C01851EBE3718A
:1078300001F0004507D54FF0000EDCF1000C7EEBA7
:1078400000006EEB0101B1F5801F1BD3B1F5001FE5
:107850000CD349085FEA30004FEA3C0C04F1010404
:107860004FEA445212F5800F80F09A80BCF1004F2D
:1078700008BF5FEA500C50F1000041EB045141EAAF
:10788000050130BD5FEA4C0C404141EB010111F4B0
:10789000801FA4F10104E9D191F0000F04BF01465B
:1078A0000020B1FA81F308BF2033A3F10B03B3F139
:1078B00020020CDA0C3208DD02F1140CC2F10C02C9
:1078C00001FA0CF021FA02F10CE002F11402D8BF27
:1078D000C2F1200C01FA02F120FA0CFCDCBF41EAF3
:1078E0000C019040E41AA2BF01EB0451294330BDC2
:1078F0006FEA04041F3C1CDA0C340EDC04F114049F
:10790000C4F1200220FA04F001FA02F340EA030075
:1079100021FA04F345EA030130BDC4F10C04C4F1BB
:10792000200220FA02F001FA04F340EA030029469B
:1079300030BD21FA04F0294630BD94F0000F83F4E5
:10794000801306BF81F480110134013D4EE77FEAC8
:10795000645C18BF7FEA655C29D094EA050F08BF14
:1079600090EA020F05D054EA000C04BF19461046F5
:1079700030BD91EA030F1EBF0021002030BD5FEA39
:10798000545C05D14000494128BF41F0004130BD61
:1079900014F580043CBF01F5801130BD01F00045B5
:1079A00045F0FE4141F470014FF0000030BD7FEA28
:1079B000645C1ABF194610467FEA655C1CBF0B4623
:1079C000024650EA013406BF52EA033591EA030F3A
:1079D00041F4002130BD00BF90F0000F04BF002132
:1079E000704730B54FF4806404F132044FF0000565
:1079F0004FF0000150E700BF90F0000F04BF0021DE
:107A0000704730B54FF4806404F1320410F0004543
:107A100048BF40424FF000013EE700BF42004FEA3E
:107A2000E2014FEA31014FEA02701FBF12F07F43BB
:107A300093F07F4F81F06051704792F0000F14BFB8
:107A400093F07F4F704730B54FF4607401F00045FC
:107A500021F0004120E700BF50EA010208BF704753
:107A600030B54FF000050AE050EA010208BF704748
:107A700030B511F0004502D5404261EB41014FF4B1
:107A8000806404F132045FEA915C3FF4DCAE4FF0B5
:107A900003025FEADC0C18BF03325FEADC0C18BF9C
:107AA000033202EBDC02C2F1200300FA03FC20FAED
:107AB00002F001FA03FE40EA0E0021FA02F114443A
:107AC000C1E600BF70B54FF0FF0C4CF4E06C1CEA4F
:107AD00011541DBF1CEA135594EA0C0F95EA0C0FC4
:107AE00000F0DEF82C4481EA030621EA4C5123EA37
:107AF0004C5350EA013518BF52EA033541F4801166
:107B000043F4801338D0A0FB02CE4FF00005E1FB18
:107B100002E506F00042E0FB03E54FF00006E1FB62
:107B200003569CF0000F18BF4EF0010EA4F1FF04A5
:107B3000B6F5007F64F5407404D25FEA4E0E6D41E5
:107B400046EB060642EAC62141EA55514FEAC520F6
:107B500040EA5E504FEACE2EB4F1FD0C88BFBCF572
:107B6000E06F1ED8BEF1004F08BF5FEA500E50F123
:107B7000000041EB045170BD06F0004646EA0101E9
:107B800040EA020081EA0301B4EB5C04C2BFD4EB1B
:107B90000C0541EA045170BD41F480114FF0000E14
:107BA000013C00F3AB8014F1360FDEBF002001F082
:107BB000004170BDC4F10004203C35DA0C341BDCFC
:107BC00004F11404C4F1200500FA05F320FA04F0CE
:107BD00001FA05F240EA020001F0004221F0004102
:107BE00010EBD37021FA04F642EB06015EEA430E75
:107BF00008BF20EAD37070BDC4F10C04C4F12005A5
:107C000000FA04F320FA05F001FA04F240EA020057
:107C100001F0004110EBD37041F100015EEA430E28
:107C200008BF20EAD37070BDC4F1200500FA05F248
:107C30004EEA020E20FA04F301FA05F243EA0203C7
:107C400021FA04F001F0004121FA04F220EA0200D6
:107C500000EBD3705EEA430E08BF20EAD37070BD1C
:107C600094F0000F0FD101F00046400041EB0101FC
:107C700011F4801F08BF013CF7D041EA060195F0DE
:107C8000000F18BF704703F00046520043EB030398
:107C900013F4801F08BF013DF7D043EA0603704785
:107CA00094EA0C0F0CEA135518BF95EA0C0F0CD090
:107CB00050EA410618BF52EA4306D1D181EA0301D6
:107CC00001F000414FF0000070BD50EA410606BFD0
:107CD0001046194652EA430619D094EA0C0F02D115
:107CE00050EA013613D195EA0C0F05D152EA03365A
:107CF0001CBF104619460AD181EA030101F0004178
:107D000041F0FE4141F470014FF0000070BD41F0C0
:107D1000FE4141F4780170BD70B54FF0FF0C4CF49A
:107D2000E06C1CEA11541DBF1CEA135594EA0C0FB9
:107D300095EA0C0F00F0A7F8A4EB050481EA030E06
:107D400052EA03354FEA013100F088804FEA0333ED
:107D50004FF0805545EA131343EA12634FEA0222BB
:107D600045EA111545EA10654FEA00260EF000417C
:107D70009D4208BF964244F1FD0404F5407402D2CE
:107D80005B084FEA3202B61A65EB03055B084FEA5F
:107D900032024FF480104FF4002CB6EB020E75EB5C
:107DA000030E22BFB61A754640EA0C005B084FEA84
:107DB0003202B6EB020E75EB030E22BFB61A754601
:107DC00040EA5C005B084FEA3202B6EB020E75EB4C
:107DD000030E22BFB61A754640EA9C005B084FEAC4
:107DE0003202B6EB020E75EB030E22BFB61A7546D1
:107DF00040EADC0055EA060E18D04FEA051545EAC0
:107E000016754FEA06164FEAC30343EA52734FEA68
:107E1000C2025FEA1C1CC0D111F4801F0BD141EAE1
:107E200000014FF000004FF0004CB6E711F4801F46
:107E300004BF01430020B4F1FD0C88BFBCF5E06F26
:107E40003FF6AFAEB5EB030C04BFB6EB020C5FEA36
:107E5000500C50F1000041EB045170BD0EF0004E8B
:107E60004EEA113114EB5C04C2BFD4EB0C0541EABD
:107E7000045170BD41F480114FF0000E013C90E6BA
:107E800045EA060E8DE60CEA135594EA0C0F08BF7E
:107E900095EA0C0F3FF43BAF94EA0C0F0AD150EA7D
:107EA00001347FF434AF95EA0C0F7FF425AF104610
:107EB00019462CE795EA0C0F06D152EA03353FF438
:107EC000FDAE1046194622E750EA410618BF52EAB5
:107ED00043067FF4C5AE50EA41047FF40DAF52EA89
:107EE00043057FF4EBAE12E74A0011D212F50012FF
:107EF00011D20DD56FF47873B3EB62520ED44FEA02
:107F0000C12343F0004343EA505323FA02F0704781
:107F10004FF00000704750EA013002D14FF0FF30BF
:107F200070474FF00000704780F0004002E000BF53
:107F300081F0004142001FBF5FEA410392EA030F54
:107F40007FEA226C7FEA236C6AD04FEA1262D2EB9E
:107F50001363C1BFD218414048404140B8BF5B42A3
:107F6000192B88BF704710F0004F40F4000020F03C
:107F70007F4018BF404211F0004F41F4000121F052
:107F80007F4118BF494292EA030F3FD0A2F101029C
:107F900041FA03FC10EB0C00C3F1200301FA03F1DA
:107FA00000F0004302D5494260EB4000B0F5000FFD
:107FB00013D3B0F1807F06D340084FEA310102F1BC
:107FC0000102FE2A51D2B1F1004F40EBC25008BF6E
:107FD00020F0010040EA03007047490040EB000038
:107FE00010F4000FA2F10102EDD1B0FA80FCACF167
:107FF000080CB2EB0C0200FA0CF0AABF00EBC25066
:1080000052421843BCBFD0401843704792F0000F53
:1080100081F4000106BF80F400000132013BB5E7A6
:108020004FEA41037FEA226C18BF7FEA236C21D01C
:1080300092EA030F04D092F0000F08BF0846704781
:1080400090EA010F1CBF0020704712F07F4F04D14F
:10805000400028BF40F00040704712F100723CBF62
:1080600000F50000704700F0004343F0FE4040F48C
:10807000000070477FEA226216BF08467FEA23634A
:108080000146420206BF5FEA412390EA010F40F435
:10809000800070474FF0000304E000BF10F0004381
:1080A00048BF40425FEA000C08BF704743F0964368
:1080B00001464FF000001CE050EA010208BF704783
:1080C0004FF000030AE000BF50EA010208BF70470A
:1080D00011F0004302D5404261EB41015FEA010C1F
:1080E00002BF84460146002043F0B64308BFA3F117
:1080F0008053A3F50003BCFA8CF2083AA3EBC253F9
:1081000010DB01FA02FC634400FA02FCC2F1200217
:10811000BCF1004F20FA02F243EB020008BF20F04E
:108120000100704702F1200201FA02FCC2F12002B4
:1081300050EA4C0021FA02F243EB020008BF20EAA9
:10814000DC7070474FF0FF0C1CEAD0521EBF1CEAD7
:10815000D15392EA0C0F93EA0C0F6FD01A4480EAC5
:10816000010C400218BF5FEA41211ED04FF00063AE
:1081700043EA501043EA5111A0FB01310CF00040DA
:10818000B1F5000F3EBF490041EAD3715B0040EA00
:10819000010062F17F02FD2A1DD8B3F1004F40EBD0
:1081A000C25008BF20F00100704790F0000F0CF0A3
:1081B000004C08BF49024CEA502040EA51207F3A67
:1081C000C2BFD2F1FF0340EAC250704740F4000042
:1081D0004FF00003013A5DDC12F1190FDCBF00F033
:1081E00000407047C2F10002410021FA02F1C2F1E1
:1081F000200200FA02FC5FEA310040F1000053EA7D
:108200004C0308BF20EADC70704792F0000F00F0CA
:10821000004C02BF400010F4000F013AF9D040EAD0
:108220000C0093F0000F01F0004C02BF490011F464
:10823000000F013BF9D041EA0C018FE70CEAD15362
:1082400092EA0C0F18BF93EA0C0F0AD030F0004CE2
:1082500018BF31F0004CD8D180EA010000F0004096
:10826000704790F0000F17BF90F0004F084691F054
:10827000000F91F0004F14D092EA0C0F01D142028E
:108280000FD193EA0C0F03D14B0218BF084608D157
:1082900080EA010000F0004040F0FE4040F40000A1
:1082A000704740F0FE4040F4400070474FF0FF0C34
:1082B0001CEAD0521EBF1CEAD15392EA0C0F93EA7B
:1082C0000C0F69D0A2EB030280EA010C49024FEACD
:1082D000402037D04FF0805343EA111143EA101386
:1082E0000CF000408B4238BF5B0042F17D024FF43E
:1082F000000C8B4224BF5B1A40EA0C00B3EB510F19
:1083000024BFA3EB510340EA5C00B3EB910F24BF01
:10831000A3EB910340EA9C00B3EBD10F24BFA3EB86
:10832000D10340EADC001B0118BF5FEA1C1CE0D14E
:10833000FD2A3FF650AF8B4240EBC25008BF20F001
:10834000010070470CF0004C4CEA50207F32C2BF55
:10835000D2F1FF0340EAC250704740F400004FF0F2
:108360000003013A37E792F0000F00F0004C02BF23
:10837000400010F4000F013AF9D040EA0C0093F0ED
:10838000000F01F0004C02BF490011F4000F013B47
:10839000F9D041EA0C0195E70CEAD15392EA0C0FAF
:1083A00008D142027FF47DAF93EA0C0F7FF470AFE7
:1083B000084676E793EA0C0F04D14B023FF44CAF2A
:1083C00008466EE730F0004C18BF31F0004CCAD1BF
:1083D00030F000427FF45CAF31F000437FF43CAFFB
:1083E0005FE700BF4FF0FF3C06E000BF4FF0010C1D
:1083F00002E000BF4FF0010C4DF804CD4FEA4002FF
:108400004FEA41037FEA226C18BF7FEA236C11D048
:1084100001B052EA530C18BF90EA010F58BFB2EBFB
:10842000030088BFC81738BF6FEAE17018BF40F07B
:10843000010070477FEA226C02D15FEA402C05D12F
:108440007FEA236CE4D15FEA412CE1D05DF8040BB4
:10845000704700BF844608466146FFE70FB5FFF747
:10846000C9FF002848BF10F1000F0FBD4DF808EDFF
:10847000FFF7F4FF0CBF012000205DF808FB00BFF0
:108480004DF808EDFFF7EAFF34BF012000205DF84A
:1084900008FB00BF4DF808EDFFF7E0FF94BF012097
:1084A00000205DF808FB00BF4DF808EDFFF7D2FF94
:1084B00094BF012000205DF808FB00BF4DF808EDD7
:1084C000FFF7C8FF34BF012000205DF808FB00BFA4
:1084D0004FEA4002B2F1FE4F0FD34FF09E03B3EBD1
:1084E00012620DD94FEA002343F0004310F0004F11
:1084F00023FA02F018BF404270474FF00000704767
:1085000012F1610F01D1420205D110F0004008BF05
:108510006FF0004070474FF00000704742000ED2ED
:10852000B2F1FE4F0BD34FF09E03B3EB126209D4AE
:108530004FEA002343F0004323FA02F070474FF064
:108540000000704712F1610F01D1420202D14FF0D9
:10855000FF3070474FF00000704700BF73B96AB931
:10856000002908BF0028BCBF00204FF00041C4BF55
:108570006FF000414FF0FF3000F03CB882B0EC46A5
:108580002DE9005000F006F8DDF804E002B00CBC64
:10859000704700BF2DE9704F089E14461D46804667
:1085A000894600F029F804FB01F3A4FB00AB00FBB3
:1085B00005329344B8EB0A0869EB0B09C6E9008958
:1085C000BDE8708F2DE9704F089E14461D46804609
:1085D000894600F061F900FB05F5A0FB04AB04FB44
:1085E0000154A344B8EB0A0869EB0B09C6E90089FA
:1085F000BDE8708F704700BF00292DE9F00FC0F271
:10860000A1800024002BC0F29880154606460F4634
:10861000002B3FD18A4258D9B2FA82F34BB1C3F151
:10862000200201FA03F720FA02F29D4000FA03F655
:108630001743290CB7FBF1F201FB1277A8B200FB3C
:1086400002F34FEA164C4CEA0747BB4209D97F199F
:1086500002F1FF3C80F00581BB4240F20281023A08
:108660002F44FF1AB7FBF1F301FB137100FB03F07A
:10867000B6B246EA0141884208D9491903F1FF37E9
:1086800080F0F180884240F2EE80023B43EA0242F1
:10869000002303E08B420AD900231A4610461946EC
:1086A00014B1404261EB4101BDE8F00F7047B3FAED
:1086B00083F8B8F1000F40F088808B4202D38242E9
:1086C00000F2E28000230122E8E712B90123B3FBA4
:1086D000F2F5B5FA85F2002A3AD17F1B280C1FFA71
:1086E00085FC0123B7FBF0F100FB11770CFB01F2D5
:1086F0004FEA164848EA0747BA4207D97F1901F1FD
:10870000FF3802D2BA4200F2C4804146BF1AB7FB1A
:10871000F0F200FB12700CFB02FCB6B246EA00401D
:10872000844507D9401902F1FF3702D2844500F28F
:10873000AE803A4642EA0142B0E7E443524263EB7C
:10874000430362E7404261EB41014FF0FF3459E7D8
:108750009540C2F1200927FA09F126FA09F9974054
:10876000280CB1FBF0F800FB18111FFA85FC0CFB7C
:1087700008F349EA07094FEA194747EA01418B42E2
:1087800006FA02F608D9491908F1FF327AD28B426B
:1087900078D9A8F102082944C91AB1FBF0F300FB0B
:1087A00013170CFB03F21FFA89F949EA0747BA428B
:1087B00007D97F1903F1FF3160D2BA425ED9023B7B
:1087C0002F44BF1A43EA08438CE7C8F1200225FA78
:1087D00002F103FA08FC27FA02F320FA02F207FA80
:1087E00008F741EA0C0C4FEA1C49B3FBF9F109FB0D
:1087F00011331FFA8CFA0AFB01FB17433A0C42EAC9
:1088000003439B4505FA08F008D913EB0C0301F16B
:10881000FF3235D29B4533D902396344CBEB030396
:10882000B3FBF9F209FB12330AFB02FABFB247EAC3
:108830000347BA4508D917EB0C0702F1FF331BD2E7
:10884000BA4519D9023A674442EA0145A5FB00013D
:10885000CAEB07078F424FF000030AD305D02A4620
:108860001CE76246FDE63B4610E706FA08F686423C
:10887000F5D26A1E002311E71A46E5E70B46A0E78A
:108880001146CBE7904687E74346424606E7023A61
:1088900050E702392F4439E72DE9F00F1446054619
:1088A0000E46002B43D18A4253D9B2FA82F757B110
:1088B000C7F1200620FA06F601FA07F302FA07F4D8
:1088C00000FA07F51E43210CB6FBF1F201FB12661C
:1088D000A0B200FB02F32F0C47EA0646B34209D9C7
:1088E000361902F1FF3780F0FD80B34240F2FA8082
:1088F000023A2644F61AB6FBF1F301FB136100FBC2
:1089000003F0ADB245EA0141884208D9091903F1E3
:10891000FF3680F0E980884240F2E680023B43EA7D
:108920000242002310461946BDE8F00F70478B4203
:108930004CD8B3FA83F6002E4FD18B4202D3824239
:1089400000F2DD80BDE8F00F002301221046194639
:10895000704712B90124B4FBF2F4B4FA84F2002A8D
:1089600040F08280091B260CA7B20123B1FBF6F070
:1089700006FB101107FB00F24FEA154C4CEA0141CF
:108980008A4207D9091900F1FF3C02D28A4200F25B
:10899000C8806046891AB1FBF6F206FB121107FB8C
:1089A00002F7ADB245EA0145AF4208D92C1902F1F0
:1089B000FF3180F09B80A74240F29880023A42EA61
:1089C000004210461946BDE8F00F704700231A46D2
:1089D00010461946BDE8F00F7047C6F1200522FA8F
:1089E00005F703FA06F421FA05F301FA06FB20FA6B
:1089F00005F53C434FEA1448B3FBF8FC08FB1C3375
:108A00001FFA84F909FB0CFA45EA0B0B4FEA1B45E8
:108A100045EA03439A4502FA06F204D91B190CF100
:108A2000FF356FD3AC46CAEB0303B3FBF8F508FB85
:108A3000153309FB05F91FFA8BFB4BEA0347B945D0
:108A400004D93F1905F1FF3362D31D4645EA0C4CAA
:108A5000ACFB0223C9EB07079F424FF000054AD346
:108A600046D062462B465DE79440C2F1200921FAC8
:108A700009FC914020FA09F9260CBCFBF6F806FB2C
:108A800018CCA7B207FB08F349EA01094FEA1941DC
:108A900041EA0C4C634500FA02F509D91CEB040CC1
:108AA00008F1FF323BD2634539D9A8F10208A4444A
:108AB000C3EB0C0CBCFBF6F306FB13C107FB03F284
:108AC0001FFA89F949EA01418A4207D9091903F1D4
:108AD000FF3022D28A4220D9023B2144891A43EA3C
:108AE000084343E73A4605E7334618E70A4666E790
:108AF000B0409042B5D20CF1FF32002312E733466A
:108B000032460FE79A458DD9ACF1020C23448AE72F
:108B1000B9459AD9023D274498E70346DEE79046D7
:108B2000C6E70238214435E74FEA4102B2F1E0439B
:108B300024BFB3F5001CDCF1FE5C0DD901F0004C44
:108B40004FEAC0024CEA5070B2F1004F40EB830094
:108B500008BF20F00100704711F0804F21D113F1C0
:108B60003872BCBF01F00040704741F480114FEAF9
:108B70005252C2F11802C2F1200C10FA0CF320FA82
:108B800002F018BF40F001004FEAC1234FEAD3239F
:108B900003FA0CFC40EA0C0023FA02F34FEA430309
:108BA000CCE77FEA625307D150EA01331EBF4FF092
:108BB000FE4040F44000704701F0004040F0FE40AD
:108BC00040F40000704700BF1C481D490268006067
:108BD0008A4200F01D80002100F004B8194B5B5858
:108BE000435004311848194B42189A42FFF4F6AF2B
:108BF000174A00F003B8002342F8043B154B9A4291
:108C0000FFF4F9AFFEF762FD00F036F8FFF7FEBFA4
:108C1000114E124830601248016821F07061016005
:108C2000410201600F4C182020600F490F48086076
:108C30000F48D0F800D0406800470000F04F0020F7
:108C4000EFBEADDE30F4000800000020F40000208C
:108C5000F8000020701600201810024009000000E3
:108C600004000140140C0140000C01404434434412
:108C700000F0FF1FFFF7FEBF2DE9804893B0F7F724
:108C800047FA914E914CD6F80880002318F0080F4F
:108C90002370374600F0E78063681B7A042B00F2EC
:108CA000E080DFE803F00303058AB100237AD9E00E
:108CB000627A864B002A00F0D48000225A7293F820
:108CC0002020100700F1CD80D97A9A7A01F00700B0
:108CD00042EA00225A621A7B02F03F00400140EA59
:108CE000D1019962597B890041EA92119A7B02F085
:108CF000010041EA8021D962D97B01F00F00C00157
:108D000040EA52021A631A7C02F07F00000140EA36
:108D100011115963597C490041EAD212997C01F042
:108D2000030042EA40229A63DA7C02F01F008001CD
:108D300040EA9101D963197DC90041EA5212997D37
:108D40001A645A7D01F0070042EA00225A64DA7D73
:108D500002F03F00400140EAD1019964197E890088
:108D600041EA92115A7E02F0010041EA8021D96461
:108D7000997E01F00F00C00140EA52021A65DA7EC6
:108D800002F07F00000140EA11115965197F490086
:108D900041EAD212597F01F0030042EA40229A656B
:108DA0009A7F02F01F00800140EA9101D965D97FC6
:108DB000C90041EA52121A6651E094F86420434B0C
:108DC000002A4ED0002283F8642093F86620012AFE
:108DD00047D193F88A20102A84BF102283F88A2072
:108DE00094F88A103A4A0023D8B2884202F102026B
:108DF00035D212F8010C12F8025C40EA052535481C
:108E000040F823500133EFE794F8CC202F4B42B3C6
:108E1000002283F8CC2093F8CD20A82A21D193F802
:108E2000E050F5B9294901EB450393F8D00093F8D8
:108E3000D13003EB0020FEF7CFFD1FA3D3E90023C1
:108E4000FEF76AFF1EA3D3E90023FEF787FCFFF7B6
:108E50004BF8214B43F825000135082DE2D10123C1
:108E600000E00023237018F4804F08D094F80431F8
:108E700023B1164B002283F80421012323702378A9
:108E800043B118F4807F05D0104BD3F808311B682C
:108E90001B689847DFF844802278D8F8003032B950
:108EA0000A4AD2F80C219A1AD243D20F00E00122CA
:108EB000B2B1F9F7DDFDB2E09A9999999999194003
:108EC0000000000000707740A40F0020F800002090
:108ED0006001002084010020DC01002050160020E9
:108EE000D4F810A1A84D0AF10101C4F81011BAF18B
:108EF000000F40F09080D5F81421110740F18F80C9
:108F0000D5F818219A1A002AC0F2898003F5C339CE
:108F100005F58E7009F1A009C5F81891FEF720F942
:108F20009A4B05F58E7001461A78F8F77BFE95F896
:108F3000220105F58E7110F0040F17D0C5F82491A9
:108F40005346FA180025A2F8FE508F4ACD5A02F572
:108F5000947E23F80E5002F5977E23F80E500233CC
:108F6000062BEED120F0040082F8220194F834217F
:108F7000854BA2B1B3F81C01B6F8FE20821AA3F803
:108F80001C21B3F81E01B6F80021821AA3F81E2195
:108F9000B3F82001B6F80221821AA3F82021D4F8F0
:108FA0002431794A002B3AD07948C3EB090981452D
:108FB00002F5947502F5977019D8764BDA6882F449
:108FC0000052DA600023CA5A35F903E017B2BE45F1
:108FD000C4BFDFF8D4E123F80E2030F903E0BE452A
:108FE000BCBF6D4FDA530233062BECD117E00023E0
:108FF000C2F8243135F903E0C15EFA1871444FF02C
:10900000020E734491FBFEF1062BA2F8FE10F1D183
:10901000F9F722FD03E00229C8BFC5F81021F8F7CF
:10902000AFFFB389C8F800002BB1D4F83821821AF9
:10903000002AFFF626AE574F4FF480427A61524F16
:10904000184496F80580D4F84431C4F8380107F57F
:10905000A870D4F83C51CDF81080984707F5A87057
:10906000014694F85621F8F7DDFD4C4B1B88002B88
:1090700000F0B980D7F858314FF000081B7807F599
:10908000AE7903934746454A1288B2F57A7F029239
:10909000434A04D1002142F80810C9F81010414990
:1090A000C85F52F80810014442F80810FEF7F6FFB6
:1090B000D9F8102083460132012AC9F8102007D1BF
:1090C0000022C9F80400C9F80000C9F808202CE003
:1090D000D9F800C061468DE80410FEF729FF009A18
:1090E00082461046FEF7DAFF01465046FFF7DEF8EB
:1090F000DDF804C001466046FEF71CFF024611463B
:10910000C9F8040058460092FEF712FF0146504687
:10911000FFF718F8D9F80810FEF70CFF009AC9F805
:109120000C00C9F80020C9F808001E49029B002263
:1091300001F1540B012B7A5227F80B20DFF85CA0C9
:1091400044D1D9F81000012808DD0138FEF7A6FF48
:109150000146D9F80C00FFF7A9F800E0002002F062
:109160000BFA039B02460BB318460092FEF796FFDC
:10917000009A01461046FFF7A1F9B8B14FF47A738F
:10918000AAF800302FE000BFF80000205A16002097
:109190007FC3C9010010014026020020581600209C
:1091A000900200204802002020020020B54A4FF41F
:1091B0007A7158F802200A2002F5FA7292FBF1F255
:1091C0002BF807200F210122F8F7C3FF0237062FE3
:1091D00008F1040809F114097FF455AF029F07F163
:1091E000FF39AAF800900023A74F07F5A87207F5EA
:1091F000D271985A595A411A99520233062BF3D117
:10920000D7F8143113F0020300F00A83D7F8B03115
:1092100007F5DC70984707F5DC70014697F8BE212A
:10922000F8F700FDB7F8C03107F5DC78002B45D022
:109230000022D7F8C4011346934F38F902C0B7F89B
:10924000C01107F5E47EB1F5C87F04BF00214EF8D8
:1092500003105EF803108C4F61444EF80310043382
:1092600000210C2B28F80210815202F10202E3D1F6
:10927000B7F8C031012B1CD1D7F8C8314FF4C872F0
:10928000C83393FBF2F30380D7F8CC31C83393FB98
:10929000F2F34380D7F8D031C83393FBF2F27B4B23
:1092A0001B88D21A8280A5F85410A5F85610F9F739
:1092B000D3FBB4F8C031013BA4F8C031B3685A07FE
:1092C00079D5B4F8D421704B322A13D1D3F8C42104
:1092D0001188A3F8D61151889288A3F8D811A3F861
:1092E000DA21B5F85420A3F8DC21B5F85620A3F80C
:1092F000DE2101E0002A3CD00021D4F8C4610A46F6
:10930000614838F901E0B0F8D43100F5F077322B3C
:1093100004BF0023BB50B8585B4B7044B8500432B4
:1093200000200C2A28F80100705201F10201E7D157
:10933000B3F8D421012A17D183F8ED21052283F84F
:10934000EE21B3F8D62183F8EC013280B3F8D821AE
:109350007280B3F8DA21B280B3F8DC21B3F8DE31E1
:10936000A5F85420A5F85630B4F8D431013BA4F840
:10937000D43194F8EF21444BEAB1D3F8E001D3F8AB
:10938000C4113226002290FBF6F083F8EF2108800A
:10939000D3F8E40190FBF6F04880D3F8E83193FB72
:1093A000F6F63A4B1B88F61A8E80A5F85420A5F8DD
:1093B0005620F9F751FBD4F8C431B4F8B8111A8823
:1093C00000268A1AA4F8B821B4F8BA115A88B1460E
:1093D0008A1AA4F8BA219B88B4F8BC21D31AA4F83D
:1093E000BC31F8F7CDFDD4F8F0310546C31A184664
:1093F0000293FEF74FFED4F8F4110390FEF7A2FE9D
:10940000D4F8F881C4F8F05198F800A005903546DA
:109410001F4F785FFEF742FE0599FEF793FE09A9FC
:109420008851BAF1000F35D05046FEF737FE01469D
:109430004FF07E50FEF73AFF0246114607F1AC0BA3
:109440004FF07E500092FEF773FD56F80B10FEF7BA
:1094500079FE07F168018446485FCDF804C0FEF745
:109460001DFE009AB8371146FEF76CFEDDF804C009
:1094700001466046FEF75EFD4BF80600FFF728F850
:1094800078530CE090020020F8000020000000203B
:109490004802002007F1B8026837E95BA952AD4FD6
:1094A0000436EA5F0235062D02FB0299B0D1AA4DBF
:1094B0004FF0640A2A880AFB09F3524393FBF2FA3D
:1094C000AAF1490A07F1080009A91FFA8AFAF8F770
:1094D00075FFBAF13B0FD8F8046010D9B4F91C023B
:1094E000FEF7DCFDD4F8186201463046FEF7E6FFD1
:1094F0009A4F94F8223168B343F008032CE04FF000
:109500007E513046FEF716FD01464FF07E50FEF7C5
:10951000CDFE4FF0000B8246914B304653F81B10A6
:109520000193FEF70FFE024637F90B000092FEF79B
:10953000B5FD009A01461046FEF7FCFC5146FEF7C9
:1095400001FE019B43F81B000BF1020BBBF1060F60
:10955000E2D1C3E723F008033146D4F8140287F8B8
:10956000223102F007F80746C4F82002D4F81002AE
:10957000D4F818B200F10046D4F814020146FEF700
:10958000E1FD594682465846FEF7DCFD014650464D
:10959000FEF7D0FC01F0F0FF0146304601F0EAFF93
:1095A00070490646C4F824023846FEF7CBFD01F0A8
:1095B00015FF6C49A4F828023046FEF7C3FD01F000
:1095C0000DFFD4F81431A4F82A021B0739D56648D8
:1095D00009A9F8F7F3FED8F808904FF07E514846F5
:1095E000FEF7A8FC01464FF07E50FEF75FFE4FF0FD
:1095F000000B8246594D484605F50B7353F81B1076
:109600000193FEF79FFD05F58E71024631F90B00BF
:109610000092FEF743FD009A01461046FEF78AFCD1
:109620005146FEF78FFD019B43F81B000BF1020B27
:10963000BBF1060FDED11846F8F778FFA5F838021F
:1096400040E0DFF814A109A90AF10400F8F7B6FE1A
:109650006868D5F808900146FEF774FD49468346D0
:109660004846FEF76FFD01465846FEF763FCED687D
:10967000814629462846FEF765FD01464846FEF725
:1096800059FC01F079FF00210546FEF7EFFEA0B975
:10969000DAF804002946FEF709FE2946CAF8040054
:1096A000DAF80800FEF702FE2946CAF80800DAF8E0
:1096B0000C00FEF7FBFDCAF80C002C48F8F736FF4B
:1096C000A4F838022A490398FEF73CFD06F100464B
:1096D000054607F10047B4F938020D960C97FEF7DE
:1096E000DDFC244900F10040FEF72CFD0E90B4F99A
:1096F0000802FEF7D3FC0F90B4F90A02FEF7CEFC85
:109700001090B4F90C02FEF7C9FC0CA911900FA837
:10971000F8F754FE98F80130104E012B2ED1164B5D
:109720001B785F070ED4D6F83C32402093FBF0F054
:10973000181AFEF7B3FC1199FEF7FCFBFEF7C8FE02
:10974000C6F83C02054BD3F83C02402390FBF3F0F3
:1097500016E000BF0003002000000020F8000020F9
:10976000080300204C3D0F44240300200400002087
:10977000BD37863535FA8E3C5C160020A94B18881B
:10978000FEF78CFC01461198FEF7D2FBD4F8441288
:1097900011902846FEF7CEFB01462846FEF786FDCF
:1097A000D4F84062054631461198FEF7C1FB0146E8
:1097B0002846FEF7C7FC01463046FEF7BBFB0646CF
:1097C000C4F840020F98D4F8487201F007FED4F8AC
:1097D00054522978F9F774F83844C4F848021098BC
:1097E000D4F84C7201F0FAFD2978F9F769F8384499
:1097F000C4F84C023046D4F8507201F0EFFD69789D
:10980000F9F75EF8884B38441A68029FC4F8500292
:109810003A441A60D4F858320133C4F8583205E09B
:10982000A7F8B831A7F8BA31A7F8BC317F4CB4F823
:109830005031A4F85C32B4F85231A4F85E32049B83
:10984000012B0ED1B4F96222B4F9543103EB420377
:10985000032293FBF2F39BB2A4F86032A4F86232C5
:1098600003E0B4F85431A4F86032F8F789FB704B88
:10987000D4F890521860D4F86432C4F86402C31A61
:109880009BB20293A4F86832B4F970022B89984213
:109890000EDBB0F5FA6FAF7907DAC21A5743A3F5BA
:1098A000FA6397FBF3F7643703E0C7F1640700E05E
:1098B0006427604BD4F83C61B3F81A8193F9EC301B
:1098C00000215B429BB2CDF80C80049334460A46DB
:1098D000594BDDF80CE031F903B0CEEB0B0303F28A
:1098E000F31C40F2E63EF44503D8002BB8BF5B42C0
:1098F00001E04FF4FA73022ADFF830E133D096F832
:109900005DC1BCF1000F04D06345CCBFCCEB0303B9
:1099100000234FF0640C93FBFCF80EEB48096FF04A
:10992000630A0AFB083AB9F894920EEB480EBEF9A6
:1099300096820FFA89FECEEB080E0EFB0AFEDFF8C8
:1099400004819EFBFCFEF14421F8089095F804E0A8
:1099500003FB0EFE394B9EFBF3F363449BB27B4348
:1099600093FBFCFC1CE096F85EC1BCF1000F04D038
:109970006345CCBFCCEB03030023DDF8108003FB71
:1099800008FCAEF8A6C295F805E083EAE37CACEBF0
:10999000E37C0CFB0EFC294B9CFBF3FC0CF1640CF0
:1099A00006EB020E9EF80480254B0CFB08F84FF0E6
:1099B000640E98FBFEF802F8038094F80E9003F111
:1099C00003080CFB09F999FBFEF902F8089094F8DA
:1099D000189003F106080CFB09FC9CFBFEFCDDF86B
:1099E0000CE002F808C0F345A3F2AA2807DA08F24F
:1099F000A22331F803E0CEF1000E21F803E001329A
:109A0000032A01F1020104F101047FF461AF094C62
:109A1000B4F81C31984217DBB0F5FA6FA8BF4FF4C9
:109A2000FA6012E00000002054160020F800002028
:109A300050160020A40F0020620300200CFEFFFF40
:109A4000A20300209A0300201846C01A4FF47A722D
:109A50005043C3F5FA63B0FBF3F3642693FBF6F2CD
:109A600008EB42016FF0630000FB0233B1F8B4125F
:109A700008EB4202B2F9B6020AB2821A534393FBD0
:109A8000F6F6B8F8CC3231445806B04DA8F8A81212
:109A90003DD5B5F8CE32B5F83802C01A00B2FEF79F
:109AA000FDFAAB49FEF74EFB064601F061FC0746A6
:109AB000304601F0D1FC0646B5F9A402FEF7EEFAF5
:109AC0008146B5F9A202FEF7E9FA39468246FEF769
:109AD00039FB314683464846FEF734FB014658467B
:109AE000FEF726FAFEF7F4FC3946A5F8A20248462E
:109AF000FEF728FB314607465046FEF723FB01469A
:109B00003846FEF717FAFEF7E3FCA5F8A402A268B0
:109B100040F602031340002B66D0D8F8D062029BB7
:109B200006211E4498F8D432884D0133DBB2B3FBD2
:109B3000F1F088F8D43201FB103313F0FF07C8F8B6
:109B4000D06251D1910712D5F8F722F995F8D522B4
:109B5000B5F8D632934207D3D5F8D8329B789342E2
:109B60008CBF0023012300E03B4688F8DC32A36869
:109B70001A0536D598F8F132D8F8E01208EB43030D
:109B8000B3F8F402082391FBF3F280B28A1A02447C
:109B900092FBF3F39BB240F6E4415943D8F8D83234
:109BA00040F6FF70B1FBF0F1D888C8F8E022091A3E
:109BB0004FF47A7251439B8891FBF3F14E43654B0E
:109BC00096FBF2F2C8F8FC12D3E90001801841EBD1
:109BD000E271C3E90001604A0023FEF7BFFCC8F848
:109BE00008030023C8F8D032D8F80C33574A13F4CE
:109BF000805318BF012382F81033A36898F8DC6201
:109C000013F4807F554C2CD0D8F8143320781B687F
:109C1000C0F380005B684D4D984758B1012385F82B
:109C20001833D5F814331B68DB68984710B102234A
:109C300085F81833D8F814331B689B68984730B1FF
:109C400023785B0703D4414B022283F81823D8F80A
:109C500014331B689B69984718B13C4B002283F86A
:109C6000182398F81823394B022A02D14C204E2190
:109C700014E0012A06D153204D214C220B46FAF75D
:109C800075FE1FE093F81023012A04D153200146EA
:109C900002464D23F3E726B153204D210A464423C3
:109CA000EDE7B3F8CC22170603D553204D21024629
:109CB000E4E793F8EE211AB11920FAF72DFE01E03E
:109CC00083F819632278550704D5254F4FF40053C4
:109CD0007B616DE0D8F80C33D80703D41F4942F0FC
:109CE00001020A70B8F8C02122B1184AD2F8142132
:109CF000910705D41B4A1288003218BF012200E0E8
:109D0000012242B11648C26882F40052C260227831
:109D100022F00102227098F82221120703D422783F
:109D200022F001022270DB0203D5237823F0010325
:109D3000237023780C4A13F0010F17D00023084931
:109D4000C8F81C334FF400530B611EE0F8000020EC
:109D500035FA8E3CF8030020407E05005C1600209A
:109D6000001001405816002050160020D8F81C138F
:109D7000136851B903F5F4237D4903F590737D4FC2
:109D8000C1F81C334FF400537B61D8F81C331268C0
:109D900073B1D21A002A0BDB764803F5F423C268AC
:109DA00003F5907382F40052C260714AC2F81C330A
:109DB000714B1B781BB1F9F7D3FE00F063BD6F4CFC
:109DC00094F84A30012B40F05785694D2368C5F857
:109DD000B843C5F8BC33664ED6F8BC0335460368B5
:109DE0005B689847002800F04185D6F8BC030368FB
:109DF0009B689847D6F8B83393F84820E2B9B0F199
:109E000024077A427A4183F84820002AE3D15C4B48
:109E10001B785D07DFD4232802D1F9F7A1FEDAE72A
:109E2000D6F8C0331B7D8342D5D1564A564B1A60B3
:109E3000564A574BDA60CEE7012A05D14D2814BFA8
:109E40000022022200F00EBD022A05D13C2814BFD8
:109E50000022032200F006BD032A0BD140284FF058
:109E6000000200F2FF841A71DA71587198710422AD
:109E700000F0F8BC042A07D19A7983F849005040D1
:109E80009871052200F0EEBC052AA4D159791A79FF
:109E90009142997906D941409971511C1971134425
:109EA000187298E7814240F0D98493F84970682F7E
:109EB00000F0648200F218812C2F00F0828448D8D0
:109EC000242F00F063842BD8202F00F04782222F0C
:109ED00000F08D83012F40F09D842C20F8F7CAF903
:109EE0000020F8F798F93846F8F795F90020F8F7C8
:109EF00092F94320F8F78FF94C20F8F78CF94620B7
:109F0000F8F789F94C20F8F786F93846F8F783F91D
:109F10000020F8F780F90020F8F77DF9002662E1CB
:109F2000282F00F03B842A2F00F04584262F40F094
:109F30007184184E0320F8F79DF9B6F9E600F8F79A
:109F40009CF9B6F9E800F8F798F9B6F9EA0000F0DC
:109F50002FBC642F00F06E811ED8342F00F0678371
:109F6000402F00F04984322F40F0548400F03DBC73
:109F7000F8000020001001405B16002018040020AB
:109F80005C160020EFBEADDEF04F00200400FA05A5
:109F900000ED00E0A40F0020662F00F0768100F2B3
:109FA000AB810B20F8F766F9B6F96802F8F765F9A6
:109FB000B6F8C40300B2F8F760F9D6F81431C3F369
:109FC000C000C3F38002800040EA4200C3F34002B5
:109FD0001043C3F3401240EAC20003F010031843D9
:109FE000F8F74BF9B6F8CC2212F0010F0CBF0021A4
:109FF000022112F0020F0CBF0023042312F0040F01
:10A000000CBF0027102712F0400F0CBF4FF00008C4
:10A010004FF0200812F0100F0CBF4FF0000E4FF45D
:10A02000007E039312F0200FD6F80C330CBF0020F3
:10A030004FF4806003F48026029102F0080B03F4D1
:10A0400080110497CDF8148003F4003703F400580E
:10A0500003F4807ACDF818E0079003F4803E03F40F
:10A06000002003F4805903F4004C03F0C00343EADA
:10A070000B0343EA0A0343EA090343EA080343EAFA
:10A080000C0343EA0E033B43334303430B43D249E0
:10A09000039F91F800E00299CEF3800E43EA0E038D
:10A0A0000B43DDF810803B43DDF814E0069843EAEB
:10A0B000080343EA0E03079912F4807F43EA000382
:10A0C0000CBF00254FF400650B4312F4007F43EAF8
:10A0D00005030CBF00224FF400121A43BF4B0020AF
:10A0E00093F8C6630346B9E0732F00F0188351D884
:10A0F0006E2F00F0918110D86C2F00F0578100F284
:10A100006381692F40F0868396F8DD0300264000C6
:10A1100000F0FE00F8F7AEF83CE1702F00F0C981C6
:10A12000C0F0A281722F40F07583AD4F1620F8F772
:10A13000A1F80020F8F7A1F8B7F9D000F8F79DF8DA
:10A14000B7F9D200F8F799F8B7F9D400F8F795F80D
:10A15000D6F83C31B3F9A801F8F78FF80020F8F7EA
:10A160008CF80020F8F7AEF8D6F83C31B3F952007D
:10A170000A2390FBF3F0F8F780F897F80401F8F75A
:10A180004AF897F80601F8F746F897F80501F8F746
:10A1900042F8C2E2782F00F0BB800DD8752F00F096
:10A1A0001A82C0F06D82772F40F0348396F8C60390
:10A1B000F8F760F80026A3E2F02F00F0D982FE2F16
:10A1C00000F0B882A02F40F025830C20F8F752F859
:10A1D000844B1868F8F776F8834B1868F8F772F82C
:10A1E000824B1868D7E2824B1B68985D0136F8F7FE
:10A1F00012F8042EF7D10020F8F73FF800267D4B27
:10A20000985D0136F8F707F80B2EF8D100267A4B47
:10A21000985D0136F7F7FFFF082EF8D10720F7F712
:10A22000FAFF0026754B985D0136F7F7F4FF072E0D
:10A23000F8D172E207206A4EF8F71CF8E620F7F72B
:10A24000EAFF7079F7F7E7FF0020F7F7E4FF96F8E9
:10A250002631002B0CBF04200C209CE2B3420CD210
:10A2600067495F5C012101FA07F7174218BF99405F
:10A2700003F1010318BF0843F0E7F8F723F8584B40
:10A2800093F86C06F7F7C7FFE2E21220F7F7F2FF48
:10A290005C4B1B88B3F5806F21D900275A4BF85EC1
:10A2A000082390FBF3F00237F7F7E7FF062FF5D10D
:10A2B000B6F95C02F7F7E1FFB6F95E02F7F7DDFFEA
:10A2C000B6F96002F7F7D9FFB6F91C01F7F7D5FF29
:10A2D000B6F91E01F7F7D1FFB6F9200168E2B6F929
:10A2E0000802F7F7CAFFB6F90A02F7F7C6FFB6F990
:10A2F0000C02F7F7C2FFDBE71020F7F7BBFF0026E1
:10A30000424B985D0136F7F786FF102EF8D19FE299
:10A310003820F7F7AFFF0027D5F83C3107F12C06BE
:10A32000F6003344B3F90600F7F7A7FFD5F83C3140
:10A3300001373344B3F90800F7F79FFFD5F83C31F4
:10A340003344B3F90A00F7F798FFD5F83C311E44BF
:10A35000307BF7F760FF082FDED179E20820F7F7AE
:10A3600089FF0026D5F83C3103EBC60393F86D0155
:10A370000136F7F750FF082EF4D169E21020F7F705
:10A3800079FF0026224B985D0136F7F744FF102E27
:10A39000F8D15DE295F8DD339E4280F059821D4B85
:10A3A00033F91600F7F769FF0136F3E70620F7F7F0
:10A3B00061FFB6F92802F7F760FFB6F92A02F7F74E
:10A3C0005CFFB6F93802F3E10620F7F753FF0020EF
:10A3D000F7F778FFBAE100BF5C160020F800002014
:10A3E000A40F0020E8F7FF1FECF7FF1FF0F7FF1F97
:10A3F000780000207CDD000888DD000891DD000881
:10A40000BF040020000000200003002062000020A4
:10A4100036160020620300200720F7F72BFF96F87E
:10A42000D502F7F7F8FED6F808034FF6FF77B842E3
:10A43000A8BF384620EAE07000B2F7F71EFFB6F971
:10A44000E003F7F71AFFC24DC24BD5F8FC0293F8B0
:10A450000C310028B8BF40420BB10A235843B84220
:10A46000A8BF384600B2A3E10720F7F703FFD6F8EC
:10A4700090321878F7F7CFFED6F890325878F7F781
:10A48000CAFED6F890321879F7F7C5FED6F89032A2
:10A490005879F7F7C0FED6F890329879F7F7BBFEF7
:10A4A000D6F890329878F7F7B6FED6F89032D8788A
:10A4B000E8E61E20F7F7DEFED6F83C3100261B78D2
:10A4C000022B72D1A24AA449D2F83C31A04F03EB2F
:10A4D0008603586AFDF736FE00F080FFFA28A8BF11
:10A4E000FA2020EAE070C0B2F7F795FED7F83C31C9
:10A4F0009A4903EB8603186BFDF724FE00F06EFF0C
:10A50000FA28A8BFFA2020EAE070C0B2F7F783FE6D
:10A51000D7F83C31924903EB8603D86BFDF712FE66
:10A5200000F05CFF6428A8BF642020EAE070C0B29D
:10A530000136F7F770FE032EC4D1072ED5F83C3153
:10A540001FD1986C8449FDF7FDFD00F047FFFA2804
:10A55000A8BFFA2020EAE070C0B2F7F75CFED5F899
:10A560003C317D49D86CFDF7EDFD00F037FFFA284E
:10A57000A8BFFA2020EAE070C0B2F7F74CFE002036
:10A580000DE033441879F7F746FED5F83C313344F3
:10A59000987BF7F740FED5F83C313344187E0136FE
:10A5A000F7F739FE0A2EC8D152E1D5F83C313344D1
:10A5B0001879F7F730FED5F83C313344987BF7F73C
:10A5C0002AFED5F83C313344187E0136F7F723FED6
:10A5D0000A2EEAD13CE12F20F7F74CFE614E16F827
:10A5E000010F002800F03481F7F715FEF7E7A020EF
:10A5F000F7F740FE0026D5F83C3106F11C0203EBCC
:10A6000082035F1D584A5B790C2101FB0323187AF2
:10A61000F7F701FE7878F7F7FEFDB878F7F7FBFD5E
:10A620000136F878F7F7F7FD282EE4D110E148203D
:10A63000F7F720FE00274FF0060909FB07F9D5F8C8
:10A640003C3109F58879994499F80A00F7F7E3FD58
:10A6500099F80500F7F7DFFD99F80600F7F7DBFD3D
:10A6600099F80700F7F7D7FD99F80800F7F7D3FD39
:10A67000013799F80900F7F7CEFD0C2FDBD1E7E0A1
:10A680004FF000090126002795F8C6339F4224DACF
:10A69000364BF95C0023344A03EB020B9A5C8A4286
:10A6A00004D00C33B3F58A7FF5D114E0DBF8040055
:10A6B00000F070FC80460EB9B24601E081440AE029
:10A6C000C24508DADBF8042012F80A00F7F7A3FD08
:10A6D0000AF1010AF4E70137D6E7002E00F0B8804E
:10A6E0005FFA89F0F7F7C6FD0026CCE71E4A9918F5
:10A6F0009A5C82420DD00C33B3F58A7FF6D10136D5
:10A7000095F8C6339E4280F0A380184BF05C00237E
:10A71000ECE7087AF7F77FFDF1E70020B2E50820C3
:10A72000F7F7A8FD0126F0B20136F7F774FD092E00
:10A73000F9D18DE00820F7F79DFD0020F7F79DFD8A
:10A740000020F7F79AFD0020F7F797FD00202FE093
:10A75000F8000020A40F0020000020410000C842A3
:10A7600000007A4447CA000878CA0008BF040020E5
:10A770000420F7F77FFDD6F83C31B3F95600F7F720
:10A780007CFDD6F83C31B3F9540011E00420F7F712
:10A7900071FDB04B9868F7F795FD59E0AD4E042078
:10A7A000F7F768FDB6F90801F7F767FDB6F90A0192
:10A7B000F7F763FD4CE00120F7F75CFDA54B5879F6
:10A7C00060E5A44E0720F7F755FD96F81801F7F756
:10A7D00022FDB6F91E01F7F750FDB6F91A01F7F799
:10A7E0004CFDB6F91C01F7F748FD0120F7F742FDD3
:10A7F000984B93F8200145E50820F7F73BFD00262C
:10A80000944B334493F810010136F7F704FD082EFA
:10A81000F6D11DE0C82F00F04A8340F24881D02FC6
:10A8200000F0328240F29081D42F00F01D8300F2BC
:10A83000FB82D22F40F0F182874B1B7803F0040398
:10A8400003F0FF06002B00F0DD820020F7F712FD79
:10A85000824BD3F8B8339879F7F7DDFC7F4B0022B1
:10A86000D3F8B83383F84820FFF7B5BA96F8FC332D
:10A8700013B17B4A7B4BDA60DFF8FC814C344445F2
:10A880007FF49EAA754CD4F8483113B104F2FE301F
:10A890009847D4F81431714A13F0080F6D4E38D030
:10A8A000B2F8A61201F145039BB28A2B2DD8B2F85B
:10A8B000CC325F0729D5B2F83802B2F8E23394F807
:10A8C0002251C21A92B293B218B2B330BCBF02F591
:10A8D000B4739BB21AB2B32AC4BFA3F5B4739BB2CC
:10A8E0002D0796F8EC005D4A13D540B24042434331
:10A8F000D2F83C011BB2007B43436FF01D0093FB79
:10A90000F0F31944A2F8A61203E0B4F83832A4F820
:10A91000E233D4F83C71514D97F86491B9F1000FCE
:10A9200051D0B5F8CC329A074DD0D5F81002D5F8F1
:10A9300014320146D5F81882B5F8A8A20193FDF7A4
:10A9400001FC019B834619461846FDF7FBFB0146B7
:10A950005846FDF7EFFA414683464046FDF7F2FBC5
:10A9600001465846FDF7E6FA00F006FE014640466D
:10A97000FDF79CFC3C498046FDF78CFDF8B940464C
:10A9800000F0A8FDD5F80014FDF7DCFB00F026FD73
:10A99000B0F5617FA8BF4FF46170FDF77FFB3349CD
:10A9A000FDF784FC00F058FD05464846FDF776FBB0
:10A9B0002946FDF7C7FB00F011FD80B200E0002042
:10A9C0005044A4F8A8022A4B381D1D68D4F89012F0
:10A9D00007F15403B6F8F620A847F9F777FBD4F847
:10A9E0000434002B5FD01D4B93F80834013B142B2B
:10A9F00054D8DFE803F00B5353275653531F5353D8
:10AA0000535353435353535353274300D4F80C34F5
:10AA10005B782BB1174B00205989F7F7C9FF42E04B
:10AA20000D4B1B7803F0040303F0FF00002BF1D162
:10AA30000146F2E70F4C0020E188F7F7B9FF01204B
:10AA40002189EAE70B4C00202189F7F7B1FF0120AB
:10AA50006189E2E7A40F00205C160020F8000020C6
:10AA60000400FA0500ED00E08FC2753CEFB6B0447B
:10AA70007400002062000020B0040020C04C0020C0
:10AA8000E188F7F795FF01202189F7F791FF022070
:10AA90006189F7F78DFF0320A189BEE7B3689B06A4
:10AAA00001D5F7F791FFFBF7D9FCFEF7EAB82B2F9A
:10AAB00007D10020F7F7DEFBF7F7AEF9B14B58717D
:10AAC000C3E636D8252F10D1AE4E0020F7F7D2FBC3
:10AAD0000023B360F7F7AAF90746F7F7A7F9B368B9
:10AAE00007EB00400343B360AFE650D8212F00F0DE
:10AAF000EC81232F40F0F681F7F78EF927281ED836
:10AB0000D6F83C3100F11C0703EB8707F7F784F90F
:10AB10009D4B7E1D03F58A72197A814203D00C3356
:10AB20009342F9D10BE01B787B71F7F775F97070E0
:10AB300026E0352F6AD1F7F76FF90B284AD90120A3
:10AB40000021F7F779FB80E6CD2F00F0A98000F215
:10AB50000981CA2F00F0AE80CC2F40F0C381D6F817
:10AB60009062F7F759F93070F7F756F97070F7F708
:10AB700053F93071F7F750F97071F7F74DF9B0717B
:10AB8000F7F74AF9B070F7F747F9F0705DE6272F4D
:10AB900010D10020F7F76EFBF7F748F9794EA6F8C9
:10ABA000E600F7F743F9A6F8E800F7F73FF9A6F84B
:10ABB000EA004AE6292F40F095810020F7F75AFB7A
:10ABC000F7F734F96F4EA6F80801F7F72FF9A6F852
:10ABD0000A013AE606277843D6F83C7100F58870FA
:10ABE0000744F7F719F90328A9D8B872F7F714F949
:10ABF0007871F7F711F9B871F7F70EF9F871F7F7FF
:10AC00000BF93872F7F708F978721EE622D82D2F63
:10AC100014D10020F7F72EFBF7F7FEF8594E86F80F
:10AC20001801F7F703F9A6F81E01F7F7FFF8A6F8E1
:10AC30001A01F7F7FBF8A6F81C0106E6332F40F0DF
:10AC400051810020F7F716FBF7F7E6F84D4B83F834
:10AC50002001FAE5412F0DD10020F7F70BFB00266C
:10AC6000F7F7DAF8474B33440136082E83F8100122
:10AC7000F6D1EAE5442F40F035810020F7F7FAFAE3
:10AC8000012386F8FC33E0E5404B1B7858073FF57D
:10AC9000DCADF9F777F8FBF739FAF8F769FCD4E59A
:10ACA0003A4B1B7859073FF5D0AD4FF4C873A6F85F
:10ACB000C031CAE5D6F83C713B78022B42D1002660
:10ACC000F7F7AAF8FDF7E6F93149FDF7EFFA7862F0
:10ACD000F7F7A2F8FDF7DEF92E49FDF7E7FA38633A
:10ACE000F7F79AF8FDF7D6F92B49FDF7DFFA0136A9
:10ACF000032EF86307F10407E2D1072ED5F83C7163
:10AD000012D1F7F789F8FDF7C5F92149FDF7CEFA19
:10AD1000B864F7F781F8FDF7BDF91D49FDF7C6FAEC
:10AD2000F864F7F779F809E0F7F776F837443871FF
:10AD3000F7F772F8B873F7F76FF8387601360A2E1E
:10AD4000DBD182E5013F0026F7F766F8013738715D
:10AD5000F7F762F8B873F7F75FF801360A2E38761E
:10AD6000F2D172E5CE2F19D1084B1B785A073FF567
:10AD70006CAD96F8223143F0040386F8223164E585
:10AD800062000020A40F002078CA00085C16002092
:10AD9000000020410000C84200007A44CF2F40F05C
:10ADA000A180F7F743F8F7F741F8514FA7F8D00023
:10ADB000F7F73CF8A7F8D200F7F738F8D6F83C6177
:10ADC000A7F8D400F7F732F8A6F8A801F7F72EF89D
:10ADD000F7F72CF8F7F72AF8F7F728F800EB8000D8
:10ADE0004000A6F85200F7F717F887F80401F7F7C4
:10ADF00013F887F80601F7F70FF887F80501F7F75A
:10AE00000BF822E5F7F708F8394B022883F86C06AF
:10AE10007FF641AF83F86C663DE7D32F62D1F7F739
:10AE200005F8A6F8E20310E5EF2F0AD1D6F83C6149
:10AE3000F6F7FCFFA6F85600F6F7F8FFA6F8540060
:10AE400003E5FA2F05D12B4B1B785B077FF523AF6A
:10AE500048E0D62F46D10026F6F7E8FF264B985358
:10AE60000236102EF8D1F0E40027D5F83C61F6F751
:10AE7000DDFF06EBC706A6F86601F6F7D7FFA6F8D2
:10AE80006801F6F7D3FFA0F57A7307289BB298BF45
:10AE900086F86D01B3F57A7F98BFA6F86A01F6F7D8
:10AEA000BBFF0137082F86F86C01DED1CDE4002608
:10AEB000F6F7BCFF114B03F26A2290530236102EB4
:10AEC000F6D1012283F80421BFE40026D5F83C71B5
:10AED000F6F7A2FF07EBC6070136082E87F86D01CB
:10AEE000F4D1B2E401200021F7F7A6F9B0E400BFE5
:10AEF000A40F00205C160020DC040020F8000020D5
:10AF000010B50023934203D0CC5CC4540133F9E75D
:10AF100010BD02440346934202D003F8011BFAE736
:10AF2000704700000D4B70B51D680022845C2B1922
:10AF30005B7803F00303012B8B5C08BF2034EE1811
:10AF4000767806F00306012E08BF2033E41A02D1FA
:10AF50000132002BEAD1204670BD00BF88000020DE
:10AF600010B50446224613780134002BFAD1CC5C8C
:10AF7000D4540133002CFAD110BDC9B2024610F8E6
:10AF8000013B1BB18B42F9D1104670470029FBD021
:10AF900018467047034613F8012B002AFBD1181AF4
:10AFA000013870470F4BF0B51E680023934215D04F
:10AFB000C55C7419647804F00304012CCC5C08BFF0
:10AFC000203537197F7807F00307012F08BF203499
:10AFD0002D1B04D10133002CE8D100E000252846C8
:10AFE000F0BD00BF8800002010B5034632B111F853
:10AFF000014B013A03F8014B002CF7D11A4493425C
:10B0000003D0002103F8011BF9E710BD30B5037828
:10B010000BB1044604E00B78002B18BF002030BDB4
:10B0200022461078013438B10023C85C28B1D55CC1
:10B030008542F5D10133F8E730BD104630BD00211F
:10B040000A2200F001B92DE9F04E82468B461F46D8
:10B05000144612B90020BDE8F08E002BFAD000266D
:10B06000A642F7D2A5196D0807FB05B95046494617
:10B07000089B9847002802DB03D06E1C25462C460F
:10B08000EEE74846BDE8F08E174B2DE9F0411D680C
:10B090000646AC6D0F46FCB9502000F0E3F8A865F9
:10B0A0008460AB6D046044601C61DC60AB6D9C61CE
:10B0B0005C61AB6DDC629C62AB6D5C631C63AB6D11
:10B0C000DC639C63AB6D5C641C64AB6DDC649C6492
:10B0D000AB6D1C77AB6D5C6230463946AA6D0123BF
:10B0E000BDE8F04100F002B8EC000020F0B508B96E
:10B0F000106828B3044614F8015B0F4617F8016B7B
:10B100003EB1B542FAD10BB12046F3E714600370AB
:10B11000F0BD4DB915602846F0BD17F8016BAE4281
:10B1200007D0002EF9D11C46234613F8015B0F46C9
:10B13000F3E715B10021217000E02B461360F0BD4C
:10B14000F0BD000084463F482DE9F04FD0F8008064
:10B150000E46344614F8015B08EB0500407800F019
:10B16000080000F0FF0708B12646F2E72D2D03D1B5
:10B17000B41C7578012703E02B2D04BF7578B41C2F
:10B1800033F010000DD1302D08D1207800F0DF0011
:10B19000582851D165781023023402E0002B08BFF3
:10B1A0000A23002F0CBF6FF0004A4FF0004ABAFB91
:10B1B000F3F903FB19AA0026304608EB050B9BF8B0
:10B1C00001B01BF0040F01D0303D0BE01BF0030B6E
:10B1D0001BD0BBF1010F14BF4FF0570B4FF0370BD3
:10B1E000CBEB05059D4210DAB6F1FF3F0AD048458A
:10B1F00006D801D1554503DC03FB0050012601E0D0
:10B200004FF0FF3614F8015BD7E7731C0CD1002F09
:10B210004FF022030CBF6FF000404FF00040CCF81D
:10B2200000302AB9BDE8F08F07B1404242B106B103
:10B23000611E1160BDE8F08F002B08BF0823B0E746
:10B24000BDE8F08F8800002030B51346044A05465B
:10B250000C46106829462246BDE83040FFF772BF11
:10B26000EC000020024B0146186800F003B800BF54
:10B27000EC00002070B5CD1C25F0030508350C2D21
:10B2800038BF0C25002D06463FDB8D423DD3214BB8
:10B290001C6818462146A1B10B685B1B0ED40B2B12
:10B2A00003D90B60CC18CD501FE08C4202D16268EC
:10B2B00002601AE04B6863600C4616E00C46496871
:10B2C000E9E7154C23681BB9304600F027F82060E9
:10B2D0002946304600F022F8431C014615D0C41C14
:10B2E00024F0030484420AD1256004F10B00231DDD
:10B2F00020F00700C31A0BD05A42E25070BD30460E
:10B30000611A00F00BF80130EED10C2333600020FD
:10B3100070BD00BF641600206016002038B5064CD2
:10B32000002305460846236000F008F8431C02D1BC
:10B33000236803B12B6038BD6C160020094A1368DE
:10B3400063B118446946884202D8106018467047B5
:10B35000054B0C221A604FF0FF307047034B13600F
:10B36000EFE700BF681600206C1600207016002062
:10B3700000B5194A20F00043934283B0014617DD1F
:10B38000B3F1FF4F04DBFCF7D3FD03B05DF804FB22
:10B39000694600F037FB00F00302012A009801998A
:10B3A00011D0022A0AD09AB1012201F0EFF8ECE79D
:10B3B000002100F0EFFC03B05DF804FB00F0EAFCB4
:10B3C00000F10040E1E701F0E1F800F10040DCE7C6
:10B3D00000F0E0FCD9E700BFD80F493F30B5C0F31B
:10B3E000C754A4F17F031E2B83B0014620DC581CF8
:10B3F0001BDB162B4FEAD17509DDC1F3160040F4B3
:10B400000000963CA04005B1404203B030BD114B56
:10B4100053F825402046FCF78DFD01900198214608
:10B42000FCF786FD20F0004333B9002003B030BDA7
:10B43000FDF74EF803B030BDC0F31604C0F3C7509B
:10B4400044F40004C0F1960024FA00F0002DDCD092
:10B45000DAE700BF1CF0000800B51D4A20F00043E9
:10B46000934283B0014618DDB3F1FF4F04DBFCF7D4
:10B470005FFD03B05DF804FB694600F0C3FA00F01D
:10B480000300012818D002280ED0D0B100980199ED
:10B4900000F080FC00F10040EBE70021002201F009
:10B4A00075F803B05DF804FB00980199012201F0E2
:10B4B0006DF800F10040DCE70098019900F06AFCAB
:10B4C000D7E700980199012201F060F8D1E700BFA9
:10B4D000D80F493F70B58AB0054600F09BF8224C62
:10B4E000064694F90030013303D0284601F02CFAC7
:10B4F00010B930460AB070BD284601F0DBF94FF0B4
:10B500007E51FCF7DBFF0028F3D01849012200230D
:10B510002846009208930191FCF780FA02460B46F8
:10B520001348CDE90423CDE9022301F0A7F894F9EB
:10B530000030CDE90601022B0BD0684601F09CF8E3
:10B5400038B1089B53B9DDE90601FDF7EDFA0AB001
:10B5500070BD01F073FA21230360F2E701F06EFA87
:10B56000089B0360EFE700BFF000002024F0000814
:10B570002CF0000800F0B6B970B58AB0054600F0AE
:10B58000B5FB224C064694F90030013308D028461A
:10B5900001F0DAF920B128460021FCF771FF10B95B
:10B5A00030460AB070BD1A49012200232846019195
:10B5B00000920893FCF732FA2478CDE90401CDE932
:10B5C00002017CB900220023CDE90623684601F080
:10B5D00053F888B1089BA3B9DDE90601FDF7A4FA89
:10B5E0000AB070BD0020002102460B46FCF794FB18
:10B5F000022CCDE90601E9D101F020FA21230360F4
:10B60000E8E701F01BFA089B0360E5E7F000002083
:10B6100030F00008F8B520F00043B3F17E5F044637
:10B6200010D008DCB3F17C5F11DAB3F10C5F00F3EA
:10B6300084809D48F8BD0146FCF77AFC0146FCF782
:10B6400035FEF8BD002840F3CD800020F8BD00286D
:10B65000C0F2CA8001464FF07E50FCF769FC4FF003
:10B660007C51FCF76FFD044600F040FB8F49064615
:10B670002046FCF767FD8E49FCF75CFC2146FCF791
:10B6800061FD8C49FCF754FC2146FCF75BFD8A49BF
:10B69000FCF750FC2146FCF755FD8849FCF748FCB7
:10B6A0002146FCF74FFD8649FCF744FC2146FCF798
:10B6B00049FD844905462046FCF744FD8249FCF7D4
:10B6C00037FC2146FCF73EFD8049FCF733FC214660
:10B6D000FCF738FD7E49FCF72BFC2146FCF732FDD8
:10B6E0004FF07E51FCF726FC01462846FCF7DEFDB4
:10B6F0003146FCF727FD26F47F6525F00F05074648
:10B7000029462846FCF71EFD01462046FCF710FCA2
:10B71000294604463046FCF70DFC01462046FCF75E
:10B72000C5FD01463846FCF705FC01462846FCF7F6
:10B7300001FC0146FCF7FEFBF8BD0146FCF702FDEB
:10B740005A490546FCF7FEFC5949FCF7F3FB29462C
:10B75000FCF7F8FC5749FCF7EBFB2946FCF7F2FC39
:10B760005549FCF7E7FB2946FCF7ECFC5349FCF78D
:10B77000DFFB2946FCF7E6FC5149FCF7DBFB2946D9
:10B78000FCF7E0FC4F4906462846FCF7DBFC4E4937
:10B79000FCF7CEFB2946FCF7D5FC4C49FCF7CAFB6D
:10B7A0002946FCF7CFFC4A49FCF7C2FB2946FCF7C7
:10B7B000C9FC4FF07E51FCF7BDFB01463046FCF75B
:10B7C00075FD01462046FCF7BDFC01464148FCF7EB
:10B7D000AFFB01462046FCF7ABFB01463E48FCF7B9
:10B7E000A7FBF8BD3D48F8BD4FF07E51FCF7A2FB2A
:10B7F0004FF07C51FCF7A6FC2C490446FCF7A2FC58
:10B800002B49FCF797FB2146FCF79CFC2949FCF7E8
:10B810008FFB2146FCF796FC2749FCF78BFB214662
:10B82000FCF790FC2549FCF783FB2146FCF78AFCDA
:10B830002349FCF77FFB2146FCF784FC06462046A3
:10B8400000F054FA1F4905462046FCF77BFC1E49D0
:10B85000FCF76EFB2146FCF775FC1C49FCF76AFB04
:10B860002146FCF76FFC1A49FCF762FB2146FCF706
:10B8700069FC4FF07E51FCF75DFB01463046FCF75A
:10B8800015FD2946FCF75EFC1249FCF751FB014609
:10B890002846FCF74FFB0146FCF74CFB01461048DD
:10B8A000FCF746FBF8BD00BFDB0FC93F08EF1138BE
:10B8B000047F4F3A4611243DA80A4E3E90B0A63E62
:10B8C000ABAA2A3E2EC69D3D6133303F2D57014025
:10B8D00039D119406821A233DA0FC93FDB0F494043
:10B8E000DA0F494021F00042B2F1FF4FF8B50446AB
:10B8F00014DC20F00045B5F1FF4F06460EDCB1F137
:10B900007E5F3AD08F1707F0020747EAD07755B924
:10B91000022F2FD0032F2FD13148F8BD08462146E2
:10B92000FCF708FBF8BDFAB1B2F1FF4F29D0B5F131
:10B93000FF4F19D0AA1AD2153C2A19DC002938DB8E
:10B940002046FCF7B3FC00F0B5FF00F09DFE012F90
:10B950002CD0022F22D0002F2FD02249FCF7EAFA58
:10B960002149FCF7E5FAF8BD002E15DB1F48F8BDAC
:10B970001E48ECE71C48F8BDF8BDBDE8F84000F0F3
:10B9800083BEB5F1FF4F19D0022FF3D0032FC3D0E0
:10B99000012F1BD00020F8BD1548F8BD1149FCF758
:10B9A000C9FA01461048FCF7C3FAF8BD00F100409F
:10B9B000F8BD3C32C4DA0020C9E7F8BD022F0CD034
:10B9C000032F08D0012F04D00A48F8BD4FF00040E3
:10B9D000F8BD0948F8BD0948F8BD0948F8BD00BFE1
:10B9E000DB0F49C02EBDBB33DB0F4940DB0FC93F26
:10B9F000DB0FC9BFDB0F493FDB0F49BFE4CB16C0EC
:10BA0000E4CB16402DE9F04FAB4A20F000449442BD
:10BA100089B006460D4664DDA84A94421CDC002825
:10BA2000A74940F3EC80FCF783FAA64B24F00F04FF
:10BA30009C42064664D0A449FCF77AFA0146286085
:10BA40003046FCF775FAA049FCF772FA01236860EA
:10BA5000184609B0BDE8F08F9C4A944262DDB4F10B
:10BA6000FF4F46DAE715863FA4EBC7542046FCF7A4
:10BA70002FFDFCF713FB0346014620460593FCF718
:10BA800057FA4FF08741FCF75DFB8046FCF720FD3D
:10BA9000FCF704FB0146044640460694FCF748FACE
:10BAA0004FF08741FCF74EFB00210790FCF7DEFCCE
:10BAB000002800F0C58020460021FCF7D7FC0028B4
:10BAC00014BF0123022382480221019000913A46CB
:10BAD00005A8294600F022FA002EC0F2A7800346EE
:10BAE00003E00022286000234A60184609B0BDE840
:10BAF000F08F0146FCF71CFA002368602860F4E729
:10BB00007449FCF715FA74490446FCF711FA01462A
:10BB100028602046FCF70CFA6F49FCF709FA01236C
:10BB20006860E2E700F0C6FE6C490746FCF70AFBD6
:10BB30004FF07C51FCF7FEF9FCF7CAFC8246FCF79B
:10BB4000ADFA5F498346FCF7FDFA01463846FCF73B
:10BB5000EFF95D4980465846FCF7F4FABAF11F0F39
:10BB600081464946404618DC5D4B0AF1FF3253F8E6
:10BB7000223024F0FF029A420FD0FCF7D9F9074691
:10BB80002F6039464046FCF7D3F94946FCF7D0F917
:10BB9000002E686056DB5346A7E7FCF7C9F9E315AA
:10BBA000C0F3C7529A1A082A0746E9DD49495846A0
:10BBB0000393FCF7C7FA074639464046FCF7B8F945
:10BBC000044621464046FCF7B3F93946FCF7B0F984
:10BBD000414907465846FCF7B5FA3946FCF7A8F93B
:10BBE000814649462046FCF7A3F9039BC0F3C752A0
:10BBF0009B1A192B074641DC2860A046C1E7FCF7D9
:10BC000099F9304B24F00F049C42064623D02E496C
:10BC1000FCF790F9014628603046FCF789F92A497B
:10BC2000FCF788F94FF0FF3368605EE795E80C0099
:10BC300003F1004102F1004243422A60696054E787
:10BC4000032340E707F1004700F100402F606860E0
:10BC5000CAF1000349E71F49FCF76CF91E49044685
:10BC6000FCF768F9014628602046FCF761F91A499B
:10BC7000FCF760F94FF0FF33686036E71949584622
:10BC8000FCF760FA074639462046FCF751F9804632
:10BC900041462046FCF74CF93946FCF749F9124970
:10BCA00004465846FCF74EFA2146FCF741F9814616
:10BCB0004946404661E700BFD80F493FE3CB1640F5
:10BCC000800FC93FD00FC93F43443537800F4943E8
:10BCD000B8F000080044353708A3852E84F9223FC8
:10BCE00038F0000800A3852E32318D2420F0004268
:10BCF000B2F1FF4FF8B5044603462DD25AB30028DF
:10BD00003DDBB2F5000F4FEAE0502CD37F38C3F390
:10BD10001603C20743F4000348BF5B00002740102E
:10BD20005B003E4619244FF08072B5189D4202DC3C
:10BD30005B1BAE181744013C4FEA43034FEA520223
:10BD4000F3D113B107F001031F447F1007F17C57B3
:10BD500007EBC050F8BDF8BD0146FCF7F3F92146EA
:10BD6000FCF7E8F8F8BD14F400020FD15B001902EB
:10BD700002F10102FAD5C2F101021044C6E7014600
:10BD8000FCF7D6F80146FCF791FAF8BD0122104401
:10BD9000BCE700BF2DE9F84320F00046B6F1485F4C
:10BDA00005460F4649DAFCF793FB002800F09D801A
:10BDB00029462846FCF7C6F94E490446FCF7C2F965
:10BDC0004D49FCF7B7F82146FCF7BCF94B49FCF7A5
:10BDD000AFF82146FCF7B6F94949FCF7ABF8214624
:10BDE000FCF7B0F94749FCF7A3F82146FCF7AAF99C
:10BDF0004549FCF79FF82146FCF7A4F98046204608
:10BE00004FF07C51FCF79EF9414606462046FCF770
:10BE100099F9394604462846FCF794F9014620462C
:10BE2000FCF786F801463046FCF782F801464FF0F1
:10BE30007E50FCF77DF8BDE8F8830146FCF782F9F7
:10BE40002C490446FCF77EF92B49FCF773F8214690
:10BE5000FCF778F92949FCF76BF82146FCF772F9F1
:10BE60002749FCF767F82146FCF76CF92549FCF7F0
:10BE70005FF82146FCF766F92349FCF75BF8214699
:10BE8000FCF760F9214B80469E42B8DD204B9E4274
:10BE900027DC06F17F4631464FF07E50FCF748F82C
:10BEA000814620464FF07C51FCF74CF93146FCF7B7
:10BEB0003FF8414606462046FCF744F93946044619
:10BEC0002846FCF73FF901462046FCF731F80146C9
:10BED0003046FCF72DF801464846FCF729F8BDE846
:10BEE000F883DFF834900B4EDBE74FF07E50BDE86F
:10BEF000F88300BF4ED747ADF6740F317CF2933410
:10BF0000010DD037610BB63AABAA2A3D9999993EFB
:10BF10000000483F0000903E0000383F2DE9F04F00
:10BF2000DFB00B93013B0293D31E48BF131DB84CE7
:10BF300006466898DB1054F8204023EAE3730C931C
:10BF4000DB4302EBC30308940693089C029B0C9A04
:10BF50001D190991C3EB02071DD4699C3D4404EBF4
:10BF6000870901354FF0000822AC0AE059F80800B3
:10BF7000FCF794F80137AF4244F8080008F10408D0
:10BF800009D0002FF2DA01370020AF4244F8080050
:10BF900008F10408F5D1089A002AC0F2DF82089A55
:10BFA0000B9B02F101089C0022AF4FEA880827444E
:10BFB0000025029A002AC0F2F28105EB070B4FF030
:10BFC00000094FF0000A56F809005BF8041DFCF761
:10BFD000B9F801465046FBF7ADFF09F10409A14548
:10BFE0008246F0D14AA840F805A004354545E0D185
:10BFF000089A0EAB03EB82030D9391464FEA890337
:10C000000793079A5EAB1344B9F1000F53F850AC95
:10C0100023DD0DF134084AAF174490440DAD4FF0C5
:10C020006E515046FCF78EF8FCF752FAFCF736F8E2
:10C030004FF087418346FCF785F801465046FBF7F1
:10C0400077FFFCF745FA594645F8040F57F8040DF9
:10C05000FBF770FF45458246E1D15046069900F056
:10C060008DFC4FF078510546FCF76CF800F026FC8B
:10C070004FF08241FCF766F801462846FBF758FF6F
:10C080000546FCF725FA8246FCF708F801462846E3
:10C09000FBF74EFF069A8046002A40F3678109F1BC
:10C0A000FF310EA850F82130C2F1080043FA00F227
:10C0B00002FA00F01B1A06989244C0F1070743FAEF
:10C0C00007F70EA840F82130002F32DDB9F1000F3C
:10C0D0000AF1010A40F375810EAB079A1946114423
:10C0E000002507E0C2F5807012B143F8040C012569
:10C0F0008B420BD053F8042B002DF3D0C2F1FF027A
:10C100008B4243F8042C4FF00105F3D1069B002B22
:10C110000DDD012B00F03281022B08D109F1FF3334
:10C120000EA951F8232002F03F0241F82320022FEC
:10C1300070D040460021FCF799F9002800F0838078
:10C14000089A09F1FF35AA420DDC079A0EAB0D984B
:10C150001344002253F8041D834242EA0102F9D13C
:10C16000002A40F0E481089B0EA85A1E50F82230A5
:10C17000002B40F0F18100EB8202012352F8041DF4
:10C1800001330029FAD04B4499450A933DDADDF892
:10C190002CA022AACA44DDF8308002EB8A02C844EF
:10C1A000C9EB0309131D03920593699A079B4FEA94
:10C1B00089094AAF02EB8808CDF810901F4400258A
:10C1C00058F8040FFBF76AFF029B039A002B5051AB
:10C1D0004FF0000B13DBDDF814A04FF00009AA4468
:10C1E00056F809005AF8041DFBF7ACFF0146584603
:10C1F000FBF7A0FE09F10409A1458346F0D1049A9A
:10C200000435954247F804BFDAD1DDF82890F5E609
:10C21000D0F3000841464FF07E50FBF789FE804680
:10C22000002D86D006994FF07E5000F0A7FB014606
:10C230004046FBF77DFE804640460021FCF716F99C
:10C2400000287FF47DAF069B40465942CDF808A0F8
:10C2500000F094FB4FF087410446FCF725F90028D5
:10C2600000F07F814FF06E512046FBF76BFFFCF72B
:10C270002FF9FBF713FF4FF087410546FBF762FFED
:10C2800001462046FBF754FEFCF722F90EAB43F8BB
:10C2900029002846FCF71CF9069C09F10105083421
:10C2A0000EA9069441F8250006994FF07E5000F043
:10C2B00065FB002D04464FDB6E1C4FEA8508C6EB7C
:10C2C000867A0DF138094AABC1444FEA8A0A98448C
:10C2D0004FF0000B59F80B00FBF7E0FE2146FBF78F
:10C2E00031FF4FF06E5148F80B002046FBF72AFF54
:10C2F000ABF1040BD3450446ECD1DFF88C92DDF8AA
:10C3000020A00024B34603950497BAF1000FB8BFEC
:10C31000002515DB00263746002501E0A7420FDC8B
:10C3200058F8061059F80600FBF70CFF014628469E
:10C33000FBF700FE0137BA45054606F10406EDDAC3
:10C340005EA800EB84030134A345A8F1040843F878
:10C35000A05CDAD1039D049F689C032C00F29880B6
:10C36000DFE814F0CB009C009C00310010D109F1F3
:10C37000FF330EA951F823703F12A5E609F1FF33F0
:10C380000EA850F8232002F07F0240F82320CEE6CA
:10C390004FF07C51FCF788F858B90746C9E64FF0D2
:10C3A000000A4AA840F805A0043545457FF401AECF
:10C3B0001EE6B9F1000F4FF002070AF1010A3FF73C
:10C3C0008BAE0025A2E6002D40F3DC804FEA850B02
:10C3D0005EAB36AE05F1FF3A5B4406EB8A0A53F8D2
:10C3E000A08C54465B4635AABB462F4600E0C846A3
:10C3F00054F804594146284601920093FBF79AFDF0
:10C40000814649462846FBF793FD4146FBF792FDDE
:10C41000019AC4F804909442A060009BE7D13D4685
:10C42000012D5F469B4640F3AD805EAB9B445BF8BD
:10C43000A04C00E044465AF8049921464846FBF7D0
:10C4400079FD804641464846FBF772FD2146FBF7E1
:10C4500071FD5645CAF80480CAF80800EAD16C1C80
:10C4600006EB84040020083654F8041DFBF762FD37
:10C47000B442F9D1002F7ED0369A379B099C00F147
:10C48000004002F1004203F10043A06022606360BB
:10C49000029A02F007005FB0BDE8F08F002DB8BF30
:10C4A00000200ADB36AE6C1C002006EB840454F836
:10C4B000041DFBF73FFDB442F9D1002F35D000F148
:10C4C0000043099C014623603698FBF731FD002D9F
:10C4D00008DD36AC04EB850554F8041FFBF72AFD94
:10C4E000AC42F9D10FB100F10040099A5060029AB4
:10C4F00002F007005FB0BDE8F08F002D39DB6C1C47
:10C5000036AE002006EB840454F8041DFBF712FD40
:10C51000B442F9D10FB100F10040099A1060029ABB
:10C5200002F007005FB0BDE8F08F0346C9E7069A46
:10C530000EAC54F82530083ACDF808A00692002B2E
:10C540007FF4B2AE04EB850353F8041D013D083AB5
:10C550000029F9D00692A7E6012314E60B9B9C0064
:10C5600046E52046FBF7B4FF0EAA4D4642F82900E7
:10C570009AE60020CEE7099C369A379BA06022609D
:10C58000636085E7002075E7DCF300082DE9F843D8
:10C5900020F00043B3F1485F04460F46904603DAAB
:10C5A000FBF796FF002857D021462046FBF7CAFD2F
:10C5B00021460546FBF7C6FD294906462846FBF7F6
:10C5C000C1FD2849FBF7B4FC2946FBF7BBFD264912
:10C5D000FBF7B0FC2946FBF7B5FD2449FBF7A8FCA7
:10C5E0002946FBF7AFFD2249FBF7A4FC8146B8F1D1
:10C5F000000F22D038464FF07C51FBF7A3FD49468F
:10C6000080463046FBF79EFD01464046FBF790FC16
:10C610002946FBF797FD3946FBF78AFC1549054685
:10C620003046FBF78FFD01462846FBF783FC0146A9
:10C630002046FBF77DFCBDE8F88349462846FBF71A
:10C6400081FD0C49FBF774FC3146FBF77BFD21466D
:10C65000FBF770FCBDE8F8832046BDE8F88300BF17
:10C66000D3C92E2F342FD7321BEF3836010D503956
:10C670008988083CABAA2A3E002070470020014967
:10C68000704700BF0000F87F2DE9F04120F0004521
:10C69000B5F1A14F0446064608DBB5F1FF4F6FDC4C
:10C6A000002840F3A0806F48BDE8F0816E4B9D42AA
:10C6B00077DCB5F1445F68DB4FF0FF372146204659
:10C6C000FBF740FD01468046FBF73CFD6749054608
:10C6D000FBF738FD6649FBF72DFC2946FBF732FDD9
:10C6E0006449FBF727FC2946FBF72CFD6249FBF761
:10C6F00021FC2946FBF726FD6049FBF71BFC294678
:10C70000FBF720FD5E49FBF715FC4146FBF71AFDE0
:10C710005C4980462846FBF715FD5B49FBF708FCA2
:10C720002946FBF70FFD5949FBF702FC2946FBF7A9
:10C7300009FD5749FBF7FCFB2946FBF703FD55496B
:10C74000FBF7F6FB2946FBF7FDFC7B1C0146404648
:10C750004CD0FBF7EFFB2146FBF7F4FC4E4B4F4D63
:10C7600053F82710FBF7E4FB2146FBF7E1FB0146FA
:10C7700055F82700FBF7DCFB002E30DBBDE8F0812D
:10C780000146FBF7D7FBBDE8F0814549FBF7D2FB3B
:10C790004FF07E51FBF792FE00288DD02046BDE879
:10C7A000F08100F087F83F4B04469D4229DCA3F559
:10C7B000D0039D4244DC0146FBF7BCFB4FF07E51A9
:10C7C000FBF7B6FB4FF0804105462046FBF7B2FB76
:10C7D00001462846FBF76AFD002704466EE700F194
:10C7E0000040BDE8F0813048BDE8F081FBF7A2FBD6
:10C7F0002146FBF7A7FC01462046FBF799FBBDE865
:10C80000F0812A4B9D4214DC4FF07F51FBF790FBE7
:10C810004FF07F5105462046FBF794FC4FF07E51C8
:10C82000FBF788FB01462846FBF740FD022704463C
:10C8300044E701461E48FBF739FD032704463DE760
:10C840004FF07E51FBF774FB4FF07E5105462046BA
:10C85000FBF770FB01462846FBF728FD012704463D
:10C860002CE700BFDB0FC93FFFFFDF3ED769853CE8
:10C8700059DA4B3D356B883D6E2EBA3D2549123E47
:10C88000ABAAAA3E21A215BD6BF16E3D95879D3DD9
:10C89000388EE33DCDCC4C3E08F4000818F4000877
:10C8A000CAF24971FFFF973FDB0FC9BFFFFF1B4073
:10C8B000000080BF20F00040704700BF2DE9F0412C
:10C8C00020F00047FD0D7F3D162D064613DC002DA0
:10C8D00080461BDB194F2F41074214D01849FBF744
:10C8E00029FB0021FBF7EAFD68B1002E1BDB28EADB
:10C8F0000700BDE8F081B7F1FF4F04D30146FBF715
:10C9000019FBBDE8F0813046BDE8F0810C49FBF72A
:10C9100011FB0021FBF7D2FD0028F4D0002E08DB2C
:10C920000020BDE8F0814FF4000343FA05F5A84468
:10C93000DDE7002FE7D00348BDE8F081FFFF7F006F
:10C94000CAF24971000080BF30F0004001D10220DE
:10C950007047A0F50003B3F1FE4F01D204207047E9
:10C96000054B421E9A4201D803207047B0F1FF43A5
:10C9700058425841704700BFFEFF7F0038B530F085
:10C980000044024603460D4614D0B4F1FF4F0DD2C9
:10C99000B4F5000F0FD3E40D2C44FE2C2EDC002C3C
:10C9A0001DDD23F0FF4343EAC45038BD0146FBF7C9
:10C9B000C1FA38BD38BD4FF09841FBF7C3FB194BA6
:10C9C00002469D4207DBC0F3C7540346193CE3E728
:10C9D000154800F02DF81449FBF7B4FB38BD14F1ED
:10C9E000160F13DA4CF250339D421146F0DD0F481A
:10C9F00000F01EF80D49FBF7A5FB38BD11460B48AA
:10CA000000F016F80949FBF79DFB38BD04F1190049
:10CA100023F0FF4343EAC0504FF04C51FBF792FB29
:10CA200038BD00BFB03CFFFF6042A20DCAF24971A1
:10CA300001F0004120F0004008437047014B1868A6
:10CA4000704700BFEC000020524F4C4C3B50495403
:10CA500043483B5941573B414C543B506F733B500B
:10CA60006F73523B4E6176523B4C4556454C3B4DA5
:10CA700041473B56454C3B00000000009EDD00084E
:10CA80000000000001000000A3DD0008010000001C
:10CA900002000000AADD0008020000000300000000
:10CAA000B3DD00080300000004000000B9DD000849
:10CAB0000500000005000000BEDD000806000000C3
:10CAC00006000000C8DD00080700000007000000A5
:10CAD000D1DD00080800000008000000DADD0008D1
:10CAE0000900000009000000E3DD00080A00000062
:10CAF0000A000000EDDD00080B0000000B00000044
:10CB0000F7DD00080C0000000C00000001DE00084A
:10CB10000D0000000D00000009DE00080E000000FE
:10CB20000E00000011DE00080F0000000F000000E2
:10CB300019DE0008100000001000000022DE0008CE
:10CB4000110000001100000029DE000812000000A2
:10CB50001200000033DE0008130000001300000084
:10CB60003BDE0008140000001400000046DE000850
:10CB7000150000001500000050DE0008160000003F
:10CB80001600000000000000FF00000091DD00081A
:10CB900088DD00087CDD0008001001400020100244
:10CBA00000100140004010020000000000000000E2
:10CBB0000301000000D1000804000000C0D00008FC
:10CBC0000400000080D000080201000060D00008CE
:10CBD00000010000000000000600000000D0000876
:10CBE00006000000A0CF00080101000000000000C6
:10CBF0000400000060CF00080600000000CF00081D
:10CC00000800000080CE00080800000000CE0008E8
:10CC10000800000080CD00080101000000000000B5
:10CC20000001000000000000000100000000000002
:10CC30000400000040CD000806000000E0CC000821
:10CC4000000100000000000002010000C0CC00084C
:10CC500001010000000000000000000000000000D2
:10CC6000A8CC00089CCC00089ACC000898CC0008FE
:10CC70002D170008E9160008C51600089D160008C3
:10CC80008D1600081526000819170008351600082B
:10CC90000D170008FF160008FFFFFFFF0001060345
:10CCA0000D0307030C03FFFF00020102020203024F
:10CCB0000802090206030D0307030C03FFFF00002F
:10CCC0000000803F0000000000000000000080BF66
:10CCD0000000803F00000000000000000000803FD6
:10CCE0000000803F000080BF0000803F000080BF48
:10CCF0000000803F000080BF000080BF0000803F38
:10CD00000000803F0000803F0000803F0000803F27
:10CD10000000803F0000803F000080BF000080BF17
:10CD20000000803F00000000000000000000000044
:10CD30000000803F00000000000000000000000034
:10CD40000000803F000000000000803F0000803FA6
:10CD50000000803F000080BF000080BF0000000096
:10CD60000000803F000000000000803F000080BF06
:10CD70000000803F0000803F000080BF0000008076
:10CD80000000803F0000803F000000BF0000803FA7
:10CD90000000803F000000BF000080BF0000803F17
:10CDA0000000803F000080BF0000003F0000803F87
:10CDB0000000803F0000003F0000803F0000803FF7
:10CDC0000000803F0000003F000080BF000080BFE7
:10CDD0000000803F000080BF000000BF000080BF57
:10CDE0000000803F000000BF0000803F000080BFC7
:10CDF0000000803F0000803F0000003F000080BF37
:10CE00000000803FF704353FF70435BF0000803F46
:10CE10000000803FF70435BFF70435BF0000803FB6
:10CE20000000803FF70435BFF704353F0000803F26
:10CE30000000803FF704353FF704353F0000803F96
:10CE40000000803F00000000000080BF000080BFA5
:10CE50000000803F000080BF00000000000080BF95
:10CE60000000803F000000000000803F000080BF05
:10CE70000000803F0000803F00000000000080BFF5
:10CE80000000803F000080BF0000803F000080BFA6
:10CE90000000803F000080BF000080BF0000803F96
:10CEA0000000803F0000803F0000803F0000803F86
:10CEB0000000803F0000803F000080BF000080BF76
:10CEC0000000803F000080BF0000803F0000803FE6
:10CED0000000803F000080BF000080BF000080BFD6
:10CEE0000000803F0000803F0000803F000080BFC6
:10CEF0000000803F0000803F000080BF0000803FB6
:10CF00000000803F000000BFD0B35D3F0000803FC5
:10CF10000000803F000000BFD0B35DBF0000803F35
:10CF20000000803F0000003FD0B35D3F000080BFA5
:10CF30000000803F0000003FD0B35DBF000080BF15
:10CF40000000803F000080BF00000000000080BFA4
:10CF50000000803F0000803F000000000000803F94
:10CF60000000803F000000000000803F000080BF04
:10CF70000000803F000080BF000080BF0000000074
:10CF80000000803F000000000000803F0000803F64
:10CF90000000803F0000803F000080BF00000000D4
:10CFA0000000803FD0B35DBF0000003F0000803F25
:10CFB0000000803FD0B35DBF000000BF000080BF15
:10CFC0000000803FD0B35D3F0000003F0000803F85
:10CFD0000000803FD0B35D3F000000BF000080BF75
:10CFE0000000803F00000000000080BF0000803F84
:10CFF0000000803F000000000000803F000080BF74
:10D000000000803F00000000A8AAAA3F0000803F67
:10D010000000803F000080BFB0AA2ABF000080BF90
:10D020000000803F0000803FB0AA2ABF000080BF00
:10D030000000803F00000000A8AAAA3F000080BFB7
:10D040000000803F000080BFB0AA2ABF0000803FE0
:10D050000000803F0000803FB0AA2ABF0000803F50
:10D060000000803F0000803F000000000000000042
:10D070000000803F000080BF0000000000000000B2
:10D080000000803F000080BF0000803F000080BFA4
:10D090000000803F000080BF000080BF0000803F94
:10D0A0000000803F0000803F0000803F0000803F84
:10D0B0000000803F0000803F000080BF000080BF74
:10D0C0000000803F000000000000803F000080BFA3
:10D0D0000000803F000080BF000000000000803F93
:10D0E0000000803F0000803F000000000000803F03
:10D0F0000000803F00000000000080BF000080BFF3
:10D100000000803F00000000A8AAAA3F0000000025
:10D110000000803F000080BFB0AA2ABF00000000CE
:10D120000000803F0000803FB0AA2ABF000000003E
:10D13000000000008025000000C201000600000081
:10D14000010000008025000000C20100070000006F
:10D1500001000102000103000104000105000106B5
:10D1600000010700010800010900010A00010B008D
:10D17000010C01031DE2000822E2000826E200087B
:10D1800039E200082BE2000831E2000835E200082D
:10D1900000000000B9E10008D9E10008E1E1000861
:10D1A000E9E10008F1E10008F8E1000803E2000805
:10D1B0000BE2000813E2000818E20008000000007B
:10D1C00043E200084CE20008FD5C000870E2000841
:10D1D00074E20008155C00088AE200088FE200088B
:10D1E000D1570008D0E10008A3E20008B1400008D0
:10D1F000C0E20008C5E20008E5380008F4E20008D3
:10D20000B9E100082D640008F9E2000801E3000814
:10D21000615A000815E3000819E300083D550008AD
:10D220002CE30008B9E100084535000831E30008A7
:10D2300035E300082D5700089DE2000851E300087F
:10D24000D153000864E300086AE300086D5B00083E
:10D25000C9EC000885E300089938000894E3000849
:10D2600085E3000815340008A0E30008A5E30008E2
:10D27000BD62000886E60008B5E30008995500087D
:10D28000E3E30008D7E300086D3400088FEA0008E4
:10D29000B9E10008E533000893E4000897E40008CA
:10D2A0009DE40008A3E40008A6E40008ADE400083B
:10D2B000B0E40008B5E40008C1E40008C4E40008D4
:10D2C000CAE40008D1E40008DBE40008E5E4000853
:10D2D000EEE40008FCE4000808E500080FE500089B
:10D2E00015E5000822E500082DE500083AE50008EC
:10D2F00000000000EAE30008F1E30008F6E300089C
:10D3000007E4000811E400081CE4000827E4000812
:10D3100031E2000832E400082BE200083BE4000898
:10D3200045E4000853E4000856E4000866E40008F9
:10D330006DE4000876E4000880E4000888E4000852
:10D34000000000001E1E6464646464649001C800F0
:10D35000C800C800C800C800C800C800C8006400F1
:10D360000000C800C800C800C80032000200000069
:10D370008025000000C20100000000002000000025
:10D380008025000000C201000100000040000000F4
:10D390008025000000C20100000000000100000024
:10D3A0008025000000C20100000000001000000005
:10D3B0008025000000C201000003000004000000FE
:10D3C00080250000004B0000000000000800000065
:10D3D00000E1000000E10000000400006D5E0008B4
:10D3E0006B1700083917000815490008871700084F
:10D3F0001149000800540040000C0140400080002A
:10D400001F2000000000200000580040000C0140D8
:10D41000000400082122000000004000C2E80008CB
:10D4200044000000B00F002000000000282300008E
:10D43000CBE8000841000000B20F0020000000000F
:10D4400001000000D9E8000844000000BE100020E0
:10D45000B0040000A4060000E0E80008440000005A
:10D46000C010002000000000D0070000EAE800081B
:10D4700044000000C210002000000000D00700009F
:10D48000F4E8000842000000C41000200000000082
:10D490001200000001E9000842000000C510002051
:10D4A00001000000FF0000000CE90008420000003D
:10D4B000C6100020000000000100000021E9000863
:10D4C000440000007410002000000000D00700009D
:10D4D0002EE9000844000000761000200000000043
:10D4E000D00700003BE9000844000000781000204D
:10D4F00000000000D007000047E9000844000000D9
:10D500007A10002000000000D007000057E9000852
:10D51000440000007C10002000000000D007000044
:10D5200068E90008440000007E10002000000000B0
:10D53000D007000073E900084400000080100020BC
:10D5400000000000D007000088E900084400000047
:10D550008210002032000000007D000097E90008E2
:10D56000440000008410002032000000F20100009E
:10D57000A6E9000841000000C710002000000000DC
:10D5800001000000B3E9000841000000C8100020BD
:10D590000000000001000000C6E900084100000092
:10D5A000C910002000000000B4000000D2E900080B
:10D5B00041000000CA1000200000000064000000CC
:10D5C000DEE9000842000000CB100020FFFFFFFF53
:10D5D00001000000F4E9000841000000CC10002028
:10D5E00000000000090000000BEA000841000000F4
:10D5F000CD100020000000000900000022EA000811
:10D6000041000000E0100020300000007E0000001B
:10D6100033EA000850000000D0100020B0040000E1
:10D6200000C2010040EA000850000000D4100020B1
:10D63000B004000000C201004DEA000841000000F3
:10D64000BC10002000000000030000005FEA00089A
:10D6500041000000E4100020000000000300000072
:10D6600072EA000841000000E51000200000000000
:10D670000100000083EA000841000000E6100020DD
:10D68000000000000100000097EA000860000000B0
:10D69000E8100020A6FFFFFF5A000000AFEA0008D4
:10D6A00060000000EC1000204CFFFFFFB400000001
:10D6B000C7EA000841000000F01000200000000050
:10D6C00001000000E0EA000841000000F110002025
:10D6D0000000000001000000EBEA00084400000028
:10D6E000B210002000000000204E0000FCEA0008FC
:10D6F00041000000A810002000000000FF00000012
:10D7000007EB000841000000A91000200A000000FB
:10D71000320000001DEB000841000000AA100020AC
:10D720000A0000003200000033EB00084400000053
:10D73000AC100020010000001027000047EB00089B
:10D7400044000000AE10002000000000720600003F
:10D750005CEB000841000000B01000200000000059
:10D76000010000007AEB0008410000008610002054
:10D77000000000000800000085EB000841000000E8
:10D780008710002000000000080000008FEB000858
:10D790004100000088100020000000000800000088
:10D7A00099EB0008480000008A1000204CFFFFFFA2
:10D7B00068010000AAEB0008480000008C1000205F
:10D7C0004CFFFFFF68010000BCEB000848000000B0
:10D7D0008E1000204CFFFFFF68010000CCEB00081A
:10D7E000440000009A100020640000008403000040
:10D7F000E2EB00084400000092100020000000004E
:10D8000000010000EBEB0008410000009810002030
:10D810000000000080000000FBEB00084400000056
:10D820009410002064000000E80300000CEC0008E5
:10D83000440000009610002064000000E80300008F
:10D840001EEC0008810000005312002001000000BF
:10D85000FA00000030EC00088100000054120020A3
:10D86000000000000100000027EC0008810000001B
:10D8700051120020000000002000000045EC0008CC
:10D88000810000005212002000000000640000002F
:10D8900052EC000881000000581200200000000037
:10D8A000960000006CEC0008840000005612002076
:10D8B000010000008403000086EC00084200000024
:10D8C00090100020FFFFFFFF010000009CEC00080B
:10D8D00082000000A2120020FFFFFFFF01000000F5
:10D8E000AAEC000882000000A31200200000000043
:10D8F00001000000BCEC0008810000004411002081
:10D900000000000002000000D1EC0008010100004E
:10D910001216002000000000FA000000D9EC0008F8
:10D920000101000013160020000000006400000048
:10D93000E1EC0008010100001416002000000000C6
:10D9400064000000E9EC0008010100001516002049
:10D950000000000064000000F2EC0008010100007B
:10D9600016160020000000006400000002ED000810
:10D9700001010000171600200000000064000000F4
:10D980000BED000801010000181600200000000047
:10D990006400000014ED0008040100001A160020C5
:10D9A000E8030000D007000023ED0008810000001C
:10D9B0009A12002000000000C800000032ED0008AC
:10D9C000810000009B12002000000000C800000041
:10D9D00045ED0008840000009C120020E8030000D0
:10D9E000D007000057ED0008840000009E120020C0
:10D9F00064000000D007000069ED0008840000000A
:10DA0000A012002064000000B80B00007BED0008AD
:10DA100081000000A412002000000000FF000000B0
:10DA200088ED000841000000911000200000000077
:10DA30000900000095ED0008810000004C11002055
:10DA400000000000FA000000A4ED000881000000C2
:10DA5000541100200000000064000000B3ED000835
:10DA6000810000005511002000000000640000004B
:10DA7000C1ED0008A00000005011002001000000CE
:10DA800014000000D1ED00088100000068110020A2
:10DA90000000000001000000E0ED00088800000028
:10DAA0004A110020D4FEFFFF2C010000EFED00081A
:10DAB0008800000048110020D4FEFFFF2C01000068
:10DAC000FDED00088100000058110020000000005A
:10DAD000300000000BEE0008A00000005C110020E8
:10DAE00000000000010000001AEE0008A000000085
:10DAF00060110020000000000100000026EE000878
:10DB0000A0000000641100200000000001000000DF
:10DB100032EE00088800000046110020B0B9FFFF77
:10DB20005046000042EE000881000000F410002082
:10DB3000000000000200000051EE0008810000001B
:10DB4000F910002000000000C800000059EE000895
:10DB5000810000000311002000000000C800000048
:10DB6000B4EB0008810000000D110020000000004F
:10DB7000C800000061EE000881000000F8100020DD
:10DB800000000000C800000068EE000881000000EE
:10DB90000211002000000000C8000000A3EB0008F4
:10DBA000810000000C11002000000000C8000000EF
:10DBB0006FEE000881000000FA1000200000000055
:10DBC000C800000075EE000881000000041100206C
:10DBD00000000000C8000000C6EB00088100000043
:10DBE0000E11002000000000C80000007BEE0008BD
:10DBF000A00000001C1100200000000064000000D4
:10DC000084EE0008A00000002811002000000000A1
:10DC1000640000008DEE0008A00000003411002018
:10DC2000000000006400000096EE0008A000000064
:10DC30001811002000000000640000009EEE0008A3
:10DC4000A00000002411002000000000640000007B
:10DC5000A6EE0008A0000000301100200000000027
:10DC600064000000AEEE0008A000000020110020BB
:10DC70000000000064000000B5EE0008A0000000F5
:10DC80002C1100200000000064000000BCEE000821
:10DC9000A000000038110020000000006400000017
:10DCA000C3EE0008A00000004011002000000000AA
:10DCB0000A000000D1EE0008A00000003C11002086
:10DCC000000000000A000000DDEE000881000000F6
:10DCD000FB10002000000000C8000000E3EE000878
:10DCE000810000000511002000000000C8000000B5
:10DCF000E9EE0008810000000F1100200000000084
:10DD0000C8000000EFEE000881000000FF100020B6
:10DD100000000000C8000000F7EE000881000000CD
:10DD20000911002000000000C8000000FFEE0008FC
:10DD3000810000001311002000000000C800000056
:10DD400007EF000881000000011100200000000022
:10DD5000C80000000DEF0008810000000B1100203A
:10DD600000000000C800000013EF00088100000060
:10DD70001511002000000000C80000004465632069
:10DD8000203720323031340032323A31343A3039AF
:10DD9000003232376238396500434A4D3100415212
:10DDA0004D3B00414E474C453B00484F52495A4F6E
:10DDB0004E3B004241524F3B004D41473B004845DE
:10DDC0004144465245453B004845414441444A3B55
:10DDD0000043414D535441423B0043414D5452494D
:10DDE000473B0047505320484F4D453B0047505359
:10DDF00020484F4C443B0050415353544852553BEC
:10DE0000004245455045523B004C45444D41583B2E
:10DE1000004C45444C4F573B004C4C4947485453E9
:10DE20003B0043414C49423B00474F5645524E4F01
:10DE3000523B004F53442053573B0054454C454DF3
:10DE4000455452593B004155544F54554E453B00A3
:10DE5000534F4E41523B000000000040000801407B
:10DE600001000000001C00280000004000080140E4
:10DE700002000000041C00280000004000080140CF
:10DE800004000000081C00280000004000080140B9
:10DE9000080000000C1C002800040040000801409D
:10DEA00040000000001D0028000400400008014060
:10DEB00080000000041D002800040040000C014008
:10DEC00001000000081D002800040040000C014073
:10DED000020000000C1D0028002C01400008014039
:10DEE00000010000001B0128002C01400008014037
:10DEF000000800000C1B012800080040000C014035
:10DF000040000000001E002800080040000C0140F6
:10DF100080000000041E002800080040000C0140A2
:10DF200000010000081E002800080040000C01400D
:10DF3000000200000C1E00283031323334353637F1
:10DF400038394142434445464748494A4B4C4D4E77
:10DF50004F505152535455565758595A00004F205C
:10DF600010044302400108436C65616E666C69678A
:10DF700068742F2573202573202F202573202825D2
:10DF80007329007261746570726F66696C65202513
:10DF9000640D0A0053797374656D20557074696D52
:10DFA000653A202564207365636F6E64732C205678
:10DFB0006F6C746167653A202564202A20302E3109
:10DFC0005620282564532062617474657279290D86
:10DFD0000A004350552025644D487A2C206465740E
:10DFE00065637465642073656E736F72733A2000A5
:10DFF0002573200041434348573A202573002E25BE
:10E0000063004379636C652054696D653A2025642B
:10E010002C20493243204572726F72733A20256476
:10E020002C20636F6E6669672073697A653A2025D4
:10E03000640D0A00417661696C61626C6520636FF2
:10E040006D6D616E64733A0D0A0025730925730DB9
:10E050000A006D6173746572007261746573000DFE
:10E060000A232076657273696F6E0D0A000D0A230C
:10E070002064756D70206D61737465720D0A000DFA
:10E080000A23206D697865720D0A006D69786572E2
:10E090002025730D0A00636D697820256400636D87
:10E0A000697820256420302030203020300D0A008F
:10E0B0000D0A0D0A2320666561747572650D0A00EC
:10E0C00066656174757265202D25730D0A0066659D
:10E0D00061747572652025730D0A000D0A0D0A23FF
:10E0E000206D61700D0A006D61702025730D0A00AE
:10E0F0000D0A232064756D702070726F66696C65FF
:10E100000D0A000D0A232070726F66696C650D0A96
:10E11000000D0A23206175780D0A000D0A23206185
:10E12000646A72616E67650D0A000D0A23206475CA
:10E130006D702072617465730D0A000D0A232072E0
:10E1400061746570726F66696C650D0A000D0A4531
:10E150006E746572696E6720434C49204D6F64652B
:10E160002C20747970652027657869742720746F76
:10E170002072657475726E2C206F72202768656C32
:10E1800070270D0A000D0A2320000D1B5B4B001B9E
:10E190005B324A1B5B313B314800556E6B6E6F77CB
:10E1A0006E20636F6D6D616E642C20747279202710
:10E1B00068656C70270008200800414554523132D0
:10E1C000333400526573657474696E6720746F2010
:10E1D00064656661756C7473004144584C33343522
:10E1E000004D505536303530004D4D41383435787E
:10E1F00000424D41323830004C534D333033444CA3
:10E200004843004D505536303030004D505536356E
:10E2100030300046414B45004E6F6E650047595205
:10E220004F00414343004241524F00534F4E415231
:10E2300000475053004750532B4D414700434A4D30
:10E2400043550061646A72616E67650073686F7739
:10E250002F7365742061646A7573746D656E7420C4
:10E2600072616E6765732073657474696E6773009D
:10E270006175780073686F772F73657420617578A6
:10E280002073657474696E677300636D69780064E8
:10E29000657369676E20637573746F6D206D69783F
:10E2A000657200726573657420746F2064656661C1
:10E2B000756C747320616E64207265626F6F740098
:10E2C00064756D70007072696E7420636F6E66693C
:10E2D00067757261626C652073657474696E6773CB
:10E2E00020696E2061207061737461626C652066C4
:10E2F0006F726D006578697400666561747572652A
:10E30000006C697374206F72202D76616C206F72BF
:10E310002076616C006765740067657420766172B1
:10E320006961626C652076616C75650068656C700A
:10E33000006D6170006D617070696E67206F66209E
:10E340007263206368616E6E656C206F72646572C3
:10E35000006D69786572206E616D65206F72206C4A
:10E36000697374006D6F746F72006765742F7365E5
:10E3700074206D6F746F72206F7574707574207671
:10E38000616C756500696E64657820283020746F53
:10E39000203229007261746570726F66696C650065
:10E3A00073617665007361766520616E64207265C5
:10E3B000626F6F74006E616D653D76616C7565208E
:10E3C0006F7220626C616E6B206F72202A20666F04
:10E3D00072206C6973740073686F7720737973743B
:10E3E000656D207374617475730052585F50504DA1
:10E3F000005642415400494E464C494748545F41FB
:10E4000043435F43414C0052585F53455249414C8E
:10E41000004D4F544F525F53544F50005345525686
:10E420004F5F54494C5400534F4654534552494151
:10E430004C004641494C534146450054454C454DDE
:10E44000455452590043555252454E545F4D455420
:10E4500045520033440052585F504152414C4C45A4
:10E460004C5F50574D0052585F4D5350005253531C
:10E47000495F414443004C45445F53545249500066
:10E48000444953504C4159004F4E4553484F543125
:10E4900032350054524900515541445000515541C4
:10E4A00044580042490047494D42414C005936000A
:10E4B0004845583600464C59494E475F57494E47E4
:10E4C000005934004845583658004F43544F583887
:10E4D000004F43544F464C415450004F43544F4615
:10E4E0004C41545800414952504C414E450048451A
:10E4F0004C495F3132305F4343504D0048454C49F1
:10E500005F39305F44454700565441494C34004818
:10E51000455836480050504D5F544F5F5345525652
:10E520004F004455414C434F505445520053494EBF
:10E53000474C45434F5054455200435553544F4D5B
:10E5400000414552543132333435363738616263D5
:10E5500064656667680043757272656E74206D69E4
:10E560007865723A2025730D0A00417661696C6105
:10E57000626C65206D69786572733A2000496E7629
:10E58000616C6964206D6978657220747970650DBD
:10E590000A004D697865722073657420746F2025B8
:10E5A000730D0A0020256420256400556E6B6E6F84
:10E5B000776E207661726961626C65206E616D654F
:10E5C0000D0A0043757272656E7420736574746908
:10E5D0006E67733A200D0A002573207365742074EA
:10E5E0006F200056616C75652061737369676E6D8D
:10E5F000656E74206F7574206F662072616E67653A
:10E600000D0A004D75737420626520616E79206F6C
:10E6100072646572206F6620414554523132333442
:10E620000D0A0043757272656E74206173736967B9
:10E630006E6D656E743A20004E4709004F4B09001D
:10E64000437573746F6D206D697865723A200D0A99
:10E650004D6F746F720954687209526F6C6C095077
:10E6600069746368095961770D0A002325643A09C2
:10E67000002573090053616E6974792063686563CE
:10E680006B3A09007265736574006C6F6164004CCD
:10E690006F61646564202573206D69780D0A0057E9
:10E6A000726F6E67206E756D626572206F66206195
:10E6B0007267756D656E74732C206E65656473206A
:10E6C0006964782074687220726F6C6C2070697451
:10E6D0006368207961770D0A004D6F746F72206E48
:10E6E000756D626572206D75737420626520626558
:10E6F000747765656E203120616E642025640D0A93
:10E7000000456E61626C6564206665617475726552
:10E71000733A2000417661696C61626C65206665C0
:10E720006174757265733A2000496E76616C696434
:10E730002066656174757265206E616D650D0A00F5
:10E7400047505320756E617661696C61626C650D2E
:10E750000A00534F4E415220756E617661696C61BB
:10E76000626C650D0A0044697361626C6564200027
:10E77000456E61626C6564200055736167653A0D92
:10E780000A6D6F746F7220696E646578205B7661C4
:10E790006C75655D202D2073686F77205B6F72202C
:10E7A0007365745D206D6F746F722076616C756532
:10E7B0000D0A004E6F2073756368206D6F746F7261
:10E7C0002C207573652061206E756D626572205B0B
:10E7D000302C2025645D0D0A004D6F746F7220256A
:10E7E00064206973207365742061742025640D0AA8
:10E7F00000496E76616C6964206D6F746F7220766B
:10E80000616C75652C20313030302E2E3230303036
:10E810000D0A0053657474696E67206D6F746F72B2
:10E8200020256420746F2025640D0A00617578200E
:10E8300025752025752025752025752025750D0A3F
:10E8400000696E6465783A206D7573742062652086
:10E850003C2025750D0A0061646A72616E6765204F
:10E8600025752025752025752025752025752025E1
:10E87000752025750D0A00736574202573203D20D1
:10E88000000D0A5265626F6F74696E67005361769E
:10E89000696E67000D0A4C656176696E6720434CAE
:10E8A00049206D6F64652C20756E736176656420F8
:10E8B0006368616E676573206C6F73742E0D0A0058
:10E8C0002E006C6F6F7074696D6500656D665F61B9
:10E8D000766F6964616E6365006D69645F72630081
:10E8E0006D696E5F636865636B006D61785F636817
:10E8F00065636B00727373695F6368616E6E656CEC
:10E9000000727373695F7363616C6500696E707523
:10E91000745F66696C746572696E675F6D6F64655C
:10E92000006D696E5F7468726F74746C65006D6100
:10E93000785F7468726F74746C65006D696E5F6384
:10E940006F6D6D616E640033645F64656164626104
:10E950006E645F6C6F770033645F646561646261ED
:10E960006E645F686967680033645F6E65757472B2
:10E97000616C0033645F6465616462616E645F74DE
:10E9800068726F74746C65006D6F746F725F70770E
:10E990006D5F7261746500736572766F5F70776D1D
:10E9A0005F726174650072657461726465645F6151
:10E9B000726D0064697361726D5F6B696C6C5F731B
:10E9C000776974636800736D616C6C5F616E676C0E
:10E9D0006500666C6170735F73706565640066697D
:10E9E00078656477696E675F616C74686F6C645F8B
:10E9F0006469720073657269616C5F706F72745FD5
:10EA0000315F7363656E6172696F0073657269610E
:10EA10006C5F706F72745F325F7363656E61726991
:10EA20006F007265626F6F745F63686172616374B7
:10EA30006572006D73705F62617564726174650008
:10EA4000636C695F6261756472617465007365729D
:10EA500069616C72785F70726F7669646572007458
:10EA6000656C656D657472795F70726F76696465E7
:10EA7000720074656C656D657472795F7377697423
:10EA800063680074656C656D657472795F696E7634
:10EA9000657273696F6E006672736B795F64656629
:10EAA00061756C745F6C617474697475646500661B
:10EAB00072736B795F64656661756C745F6C6F6EA1
:10EAC000676974756465006672736B795F636F6FF5
:10EAD0007264696E617465735F666F726D617400F4
:10EAE0006672736B795F756E6974006261747465C8
:10EAF00072795F63617061636974790076626174D1
:10EB00005F7363616C6500766261745F6D61785FED
:10EB100063656C6C5F766F6C7461676500766261CB
:10EB2000745F6D696E5F63656C6C5F766F6C74614A
:10EB300067650063757272656E745F6D657465728A
:10EB40005F7363616C650063757272656E745F6D8F
:10EB5000657465725F6F6666736574006D756C745D
:10EB6000697769695F63757272656E745F6D6574EC
:10EB700065725F6F757470757400616C69676E5F44
:10EB80006779726F00616C69676E5F6163630061D2
:10EB90006C69676E5F6D616700616C69676E5F626B
:10EBA0006F6172645F726F6C6C00616C69676E5F3D
:10EBB000626F6172645F706974636800616C696739
:10EBC0006E5F626F6172645F796177006D61785F1B
:10EBD000616E676C655F696E636C696E6174696FA5
:10EBE0006E006779726F5F6C7066006D6F726F6E2A
:10EBF0005F7468726573686F6C64006779726F5FC9
:10EC0000636D70665F666163746F72006779726FBF
:10EC10005F636D70666D5F666163746F7200616CD7
:10EC2000745F686F6C645F6465616462616E6400E8
:10EC3000616C745F686F6C645F666173745F636856
:10EC4000616E6765007961775F6465616462616EBA
:10EC500064007468726F74746C655F636F72726560
:10EC60006374696F6E5F76616C7565007468726F4E
:10EC700074746C655F636F7272656374696F6E5FE5
:10EC8000616E676C65007961775F636F6E74726F38
:10EC90006C5F646972656374696F6E007961775F38
:10ECA000646972656374696F6E007472695F756E12
:10ECB00061726D65645F736572766F00646566612D
:10ECC000756C745F726174655F70726F66696C6594
:10ECD0000072635F726174650072635F6578706F64
:10ECE000007468725F6D6964007468725F65787043
:10ECF0006F00726F6C6C5F70697463685F726174CF
:10ED000065007961775F72617465007470615F722C
:10ED1000617465007470615F627265616B706F69C8
:10ED20006E74006661696C736166655F64656C61D1
:10ED300079006661696C736166655F6F66665F64C2
:10ED4000656C6179006661696C736166655F7468A2
:10ED5000726F74746C65006661696C736166655F7F
:10ED60006D696E5F75736563006661696C7361667A
:10ED7000655F6D61785F757365630067696D62617A
:10ED80006C5F666C616773006163635F6861726486
:10ED900077617265006163635F6C70665F66616373
:10EDA000746F720061636378795F64656164626146
:10EDB0006E64006163637A5F6465616462616E645E
:10EDC000006163637A5F6C70665F6375746F66661B
:10EDD000006163635F756E61726D656463616C0091
:10EDE0006163635F7472696D5F7069746368006109
:10EDF00063635F7472696D5F726F6C6C00626172E5
:10EE00006F5F7461625F73697A65006261726F5FE0
:10EE10006E6F6973655F6C7066006261726F5F63CD
:10EE2000665F76656C006261726F5F63665F616CDE
:10EE300074006D61675F6465636C696E6174696FAE
:10EE40006E007069645F636F6E74726F6C6C657274
:10EE500000705F706974636800695F7069746368EB
:10EE600000705F726F6C6C00695F726F6C6C007029
:10EE70005F79617700695F79617700705F706974AD
:10EE800063686600695F70697463686600645F70D8
:10EE9000697463686600705F726F6C6C6600695FAE
:10EEA000726F6C6C6600645F726F6C6C6600705F92
:10EEB0007961776600695F7961776600645F79617F
:10EEC0007766006C6576656C5F686F72697A6F6EE5
:10EED000006C6576656C5F616E676C6500705F6184
:10EEE0006C7400695F616C7400645F616C740070C5
:10EEF0005F6C6576656C00695F6C6576656C006457
:10EF00005F6C6576656C00705F76656C00695F7636
:10EF1000656C00645F76656C000020202020202056
:10EF200020202028282828282020202020202020B9
:10EF300020202020202020202020881010101010B9
:10EF40001010101010101010101004040404040409
:10EF500004040404101010101010104141414141EC
:10EF60004101010101010101010101010101010151
:10EF700001010101011010101010104242424242E2
:10EF80004202020202020202020202020202020221
:10EF90000202020202101010102000000000000007
:10EFA0000000000000000000000000000000000061
:10EFB0000000000000000000000000000000000051
:10EFC0000000000000000000000000000000000041
:10EFD0000000000000000000000000000000000031
:10EFE0000000000000000000000000000000000021
:10EFF0000000000000000000000000000000000011
:10F000000000000000000000000000000000000000
:10F010000000000000000000000000000000004BA5
:10F02000000000CB61636F73660000000000000009
:10F030007371727466000000000FC93F000F4940F1
:10F0400000CB9640000FC9400053FB4000CB164157
:10F0500000ED2F41000F49410031624100537B41D7
:10F06000003A8A4100CB9641005CA34100EDAF41DC
:10F07000007EBC41000FC94100A0D5410031E241F2
:10F0800000C2EE410053FB4100F20342003A0A4243
:10F090000083104200CB164200141D42005C234244
:10F0A00000A5294200ED2F4200363642007E3C4248
:10F0B00000C74242000F4942A2000000F9000000D0
:10F0C000830000006E0000004E00000044000000BD
:10F0D0001500000029000000FC00000027000000CF
:10F0E00057000000D1000000F500000034000000CF
:10F0F000DD000000C0000000DB0000006200000036
:10F1000095000000990000003C0000004300000052
:10F110009000000041000000FE00000051000000CF
:10F1200063000000AB000000DE000000BB00000038
:10F13000C500000061000000B700000024000000CE
:10F140006E0000003A000000420000004D00000088
:10F15000D2000000E00000000600000049000000AE
:10F160002E000000EA00000009000000D1000000AD
:10F17000920000001C000000FE0000001D000000C6
:10F18000EB0000001C000000B1000000290000009E
:10F19000A70000003E000000E80000008200000020
:10F1A00035000000F50000002E000000BB0000004C
:10F1B0004400000084000000E90000009C00000002
:10F1C0007000000026000000B40000005F00000096
:10F1D0007E000000410000003900000091000000A6
:10F1E000D60000003900000083000000530000003A
:10F1F00039000000F40000009C00000084000000C2
:10F200005F0000008B000000BD000000F90000005E
:10F21000280000003B0000001F000000F800000074
:10F2200097000000FF000000DE0000000500000065
:10F23000980000000F000000EF0000002F00000009
:10F24000110000008B0000005A0000000A000000BE
:10F250006D0000001F0000006D000000360000007F
:10F260007E000000CF00000027000000CB0000005F
:10F2700009000000B70000004F0000004600000039
:10F280003F000000660000009E0000005F000000DC
:10F29000EA0000002D0000007500000027000000BB
:10F2A000BA000000C7000000EB000000E50000000D
:10F2B000F10000007B0000003D000000070000009E
:10F2C00039000000F70000008A0000005200000032
:10F2D00092000000EA0000006B000000FB0000004C
:10F2E0005F000000B10000001F0000008D00000062
:10F2F0005D00000008000000560000000300000050
:10F300003000000046000000FC0000007B00000010
:10F310006B000000AB000000F0000000CF00000018
:10F32000BC000000200000009A000000F400000073
:10F33000360000001D000000A9000000E3000000EE
:10F3400091000000610000005E000000E600000087
:10F350001B0000000800000065000000990000008C
:10F36000850000005F00000014000000A000000005
:10F3700068000000400000008D000000FF00000059
:10F38000D8000000800000004D0000007300000065
:10F390002700000031000000060000000600000009
:10F3A0001500000056000000CA00000073000000B5
:10F3B000A8000000C900000060000000E20000009A
:10F3C0007B000000C00000008C0000006B0000000B
:10F3D0000400000007000000090000000000C93F11
:10F3E0000000F0390000DA370000A2330000842E5C
:10F3F0000000502B0000C2270000D0220000C41FD4
:10F400000000C61B000044176937AC316821223365
:10F41000B40F14336821A2333863ED3EDA0F493F4D
:08F420005E987B3FDA0FC93F43
:08F42800D091FF7F01000000FC
:10F43000000100000000803F00000000000000000C
:10F4400000000000000000000000000001000000BB
:10F45000000000000000000000127A000000000020
:10F460000000000001020304060708090103000070
:10F470000000803F0000803F0000803F010000004E
:10F48000000102030401020304060708090204063E
:10F490000800DC05DC05DC05DC05DC05DC05DC053D
:10F4A000DC050000F949000899DD000803000000B0
:10F4B00000A24A043DE2000819EF00080000000025
:10F4C000000000000000000000000000000000003C
:10F4D00000000000000000000000000024E200081E
:10F4E000000000000000000000000000000000001C
:10F4F000000000000000000000000000000000000C
:10F5000000000000000000000000000000000000FB
:10F510000000000000000000000000008C0000203F
:04F5200001000000E6
:0400000508000000EF
:00000001FF
